Component: ARM Compiler 5.06 update 6 (build 750) Tool: armlink [4d35ed]

==============================================================================

Section Cross References

    gd32f1x0_it.o(i.USART0_IRQHandler_Process) refers to gd32f1x0_usart.o(i.usart_interrupt_flag_get) for usart_interrupt_flag_get
    gd32f1x0_it.o(i.USART0_IRQHandler_Process) refers to gd32f1x0_usart.o(i.usart_data_receive) for usart_data_receive
    gd32f1x0_it.o(i.USART0_IRQHandler_Process) refers to gd32f1x0_usart.o(i.usart_interrupt_disable) for usart_interrupt_disable
    gd32f1x0_it.o(i.USART0_IRQHandler_Process) refers to uip_kernel_message.o(i.UIP_SendMessage) for UIP_SendMessage
    gd32f1x0_it.o(i.USART0_IRQHandler_Process) refers to gd32f1x0_usart.o(i.usart_data_transmit) for usart_data_transmit
    gd32f1x0_it.o(i.USART0_IRQHandler_Process) refers to main.o(.data) for rxcount
    gd32f1x0_it.o(i.USART0_IRQHandler_Process) refers to main.o(.bss) for receiver_buffer
    main.o(i.fputc) refers to gd32f1x0_usart.o(i.usart_data_transmit) for usart_data_transmit
    main.o(i.fputc) refers to gd32f1x0_usart.o(i.usart_flag_get) for usart_flag_get
    main.o(i.main) refers to demo.o(i.uipEnterKernel) for uipEnterKernel
    app_cfg.o(.data) refers to app_cfg.o(.bss) for AppMsgBuf
    app_cfg.o(.data) refers to demo.o(i.TASK_0) for TASK_0
    app_cfg.o(.data) refers to demo.o(i.TASK_1) for TASK_1
    app_cfg.o(.data) refers to demo.o(i.TASK_2) for TASK_2
    app_cfg.o(.data) refers to demo.o(i.TASK_3) for TASK_3
    app_cfg.o(.data) refers to demo.o(i.TASK_4) for TASK_4
    app_cfg.o(.data) refers to demo.o(i.AppIdleTask) for AppIdleTask
    app_int_cfg.o(.data) refers to app_int_cfg.o(i.Chip_GD32F1X0_USART0_ISR_Handler_Callback) for Chip_GD32F1X0_USART0_ISR_Handler_Callback
    app_int_cfg.o(.data) refers to gd32f1x0_it.o(i.USART0_IRQHandler_Process) for USART0_IRQHandler_Process
    demo.o(i.TASK_0) refers to gd32f1x0_misc.o(i.nvic_irq_enable) for nvic_irq_enable
    demo.o(i.TASK_0) refers to gd32f1x0_eval.o(i.gd_eval_com_init) for gd_eval_com_init
    demo.o(i.TASK_0) refers to gd32f1x0_usart.o(i.usart_interrupt_enable) for usart_interrupt_enable
    demo.o(i.TASK_0) refers to uip_kernel_event.o(i.UIP_WaitEvent) for UIP_WaitEvent
    demo.o(i.TASK_0) refers to uip_kernel_event.o(i.UIP_ClearEvent) for UIP_ClearEvent
    demo.o(i.TASK_1) refers to uip_kernel_event.o(i.UIP_WaitEvent) for UIP_WaitEvent
    demo.o(i.TASK_1) refers to uip_kernel_event.o(i.UIP_ClearEvent) for UIP_ClearEvent
    demo.o(i.TASK_1) refers to gd32f1x0_usart.o(i.usart_interrupt_enable) for usart_interrupt_enable
    demo.o(i.TASK_2) refers to uip_kernel_event.o(i.UIP_WaitEvent) for UIP_WaitEvent
    demo.o(i.TASK_2) refers to uip_kernel_event.o(i.UIP_ClearEvent) for UIP_ClearEvent
    demo.o(i.TASK_2) refers to uip_kernel_resource.o(i.UIP_GetResource) for UIP_GetResource
    demo.o(i.TASK_2) refers to uip_kernel_resource.o(i.UIP_ReleaseResource) for UIP_ReleaseResource
    demo.o(i.TASK_3) refers to uip_kernel_resource.o(i.UIP_GetResource) for UIP_GetResource
    demo.o(i.TASK_3) refers to uip_kernel_event.o(i.UIP_SetEvent) for UIP_SetEvent
    demo.o(i.TASK_3) refers to uip_kernel_resource.o(i.UIP_ReleaseResource) for UIP_ReleaseResource
    demo.o(i.TASK_4) refers to uip_kernel_message.o(i.UIP_ReceiveMessage) for UIP_ReceiveMessage
    demo.o(i.TASK_4) refers to gd32f1x0_usart.o(i.usart_interrupt_enable) for usart_interrupt_enable
    demo.o(i.TASK_4) refers to uip_kernel_task.o(i.UIP_TerminateTask) for UIP_TerminateTask
    demo.o(i.TASK_4) refers to demo.o(.bss) for appBuf
    demo.o(i.uipAppInitialize) refers to uip_kernel_common.o(i.uipTaskInitialize) for uipTaskInitialize
    demo.o(i.uipAppInitialize) refers to uip_kernel_common.o(i.uipAlarmInitialize) for uipAlarmInitialize
    demo.o(i.uipAppInitialize) refers to uip_kernel_common.o(i.uipResInitialize) for uipResInitialize
    demo.o(i.uipAppInitialize) refers to uip_kernel_common.o(i.uipMsgInitialize) for uipMsgInitialize
    demo.o(i.uipAppInitialize) refers to hardware_init.o(i.Kernel_System_Tick_Init) for Kernel_System_Tick_Init
    demo.o(i.uipAppInitialize) refers to app_cfg.o(.data) for AppTaskNumber
    demo.o(i.uipEnterKernel) refers to system_gd32f1x0.o(i.SystemInit) for SystemInit
    demo.o(i.uipEnterKernel) refers to uip_kernel_common.o(i.StartOS) for StartOS
    demo.o(i.uipEnterKernel) refers to uip_kernel_common.o(.data) for uipIdleTaskID
    system_gd32f1x0.o(i.SystemCoreClockUpdate) refers to system_gd32f1x0.o(.data) for SystemCoreClock
    system_gd32f1x0.o(i.SystemInit) refers to system_gd32f1x0.o(i.system_clock_config) for system_clock_config
    system_gd32f1x0.o(i.system_clock_config) refers to system_gd32f1x0.o(i.system_clock_72m_hxtal) for system_clock_72m_hxtal
    startup_gd32f1x0.o(RESET) refers to startup_gd32f1x0.o(STACK) for __initial_sp
    startup_gd32f1x0.o(RESET) refers to startup_gd32f1x0.o(.text) for Reset_Handler
    startup_gd32f1x0.o(RESET) refers to gd32f1x0_it.o(i.NMI_Handler) for NMI_Handler
    startup_gd32f1x0.o(RESET) refers to gd32f1x0_it.o(i.HardFault_Handler) for HardFault_Handler
    startup_gd32f1x0.o(RESET) refers to gd32f1x0_it.o(i.MemManage_Handler) for MemManage_Handler
    startup_gd32f1x0.o(RESET) refers to gd32f1x0_it.o(i.BusFault_Handler) for BusFault_Handler
    startup_gd32f1x0.o(RESET) refers to gd32f1x0_it.o(i.UsageFault_Handler) for UsageFault_Handler
    startup_gd32f1x0.o(RESET) refers to gd32f1x0_it.o(i.SVC_Handler) for SVC_Handler
    startup_gd32f1x0.o(RESET) refers to gd32f1x0_it.o(i.DebugMon_Handler) for DebugMon_Handler
    startup_gd32f1x0.o(RESET) refers to uip_kernel_isr_cm.o(CODE) for uipPendSVHandler
    startup_gd32f1x0.o(RESET) refers to uip_kernel_time.o(i.uipSystemCounterHandler) for uipSystemCounterHandler
    startup_gd32f1x0.o(RESET) refers to chip_uip_interrupt.o(i.WWDGT_IRQHandler) for WWDGT_IRQHandler
    startup_gd32f1x0.o(RESET) refers to chip_uip_interrupt.o(i.LVD_IRQHandler) for LVD_IRQHandler
    startup_gd32f1x0.o(RESET) refers to chip_uip_interrupt.o(i.RTC_IRQHandler) for RTC_IRQHandler
    startup_gd32f1x0.o(RESET) refers to chip_uip_interrupt.o(i.FMC_IRQHandler) for FMC_IRQHandler
    startup_gd32f1x0.o(RESET) refers to chip_uip_interrupt.o(i.RCU_IRQHandler) for RCU_IRQHandler
    startup_gd32f1x0.o(RESET) refers to chip_uip_interrupt.o(i.EXTI0_1_IRQHandler) for EXTI0_1_IRQHandler
    startup_gd32f1x0.o(RESET) refers to chip_uip_interrupt.o(i.EXTI2_3_IRQHandler) for EXTI2_3_IRQHandler
    startup_gd32f1x0.o(RESET) refers to chip_uip_interrupt.o(i.EXTI4_15_IRQHandler) for EXTI4_15_IRQHandler
    startup_gd32f1x0.o(RESET) refers to chip_uip_interrupt.o(i.TSI_IRQHandler) for TSI_IRQHandler
    startup_gd32f1x0.o(RESET) refers to chip_uip_interrupt.o(i.DMA_Channel0_IRQHandler) for DMA_Channel0_IRQHandler
    startup_gd32f1x0.o(RESET) refers to chip_uip_interrupt.o(i.DMA_Channel1_2_IRQHandler) for DMA_Channel1_2_IRQHandler
    startup_gd32f1x0.o(RESET) refers to chip_uip_interrupt.o(i.DMA_Channel3_4_IRQHandler) for DMA_Channel3_4_IRQHandler
    startup_gd32f1x0.o(RESET) refers to chip_uip_interrupt.o(i.ADC_CMP_IRQHandler) for ADC_CMP_IRQHandler
    startup_gd32f1x0.o(RESET) refers to chip_uip_interrupt.o(i.TIMER0_BRK_UP_TRG_COM_IRQHandler) for TIMER0_BRK_UP_TRG_COM_IRQHandler
    startup_gd32f1x0.o(RESET) refers to chip_uip_interrupt.o(i.TIMER0_Channel_IRQHandler) for TIMER0_Channel_IRQHandler
    startup_gd32f1x0.o(RESET) refers to chip_uip_interrupt.o(i.TIMER1_IRQHandler) for TIMER1_IRQHandler
    startup_gd32f1x0.o(RESET) refers to chip_uip_interrupt.o(i.TIMER2_IRQHandler) for TIMER2_IRQHandler
    startup_gd32f1x0.o(RESET) refers to chip_uip_interrupt.o(i.TIMER5_DAC_IRQHandler) for TIMER5_DAC_IRQHandler
    startup_gd32f1x0.o(RESET) refers to chip_uip_interrupt.o(i.TIMER13_IRQHandler) for TIMER13_IRQHandler
    startup_gd32f1x0.o(RESET) refers to chip_uip_interrupt.o(i.TIMER14_IRQHandler) for TIMER14_IRQHandler
    startup_gd32f1x0.o(RESET) refers to chip_uip_interrupt.o(i.TIMER15_IRQHandler) for TIMER15_IRQHandler
    startup_gd32f1x0.o(RESET) refers to chip_uip_interrupt.o(i.TIMER16_IRQHandler) for TIMER16_IRQHandler
    startup_gd32f1x0.o(RESET) refers to chip_uip_interrupt.o(i.I2C0_EV_IRQHandler) for I2C0_EV_IRQHandler
    startup_gd32f1x0.o(RESET) refers to chip_uip_interrupt.o(i.I2C1_EV_IRQHandler) for I2C1_EV_IRQHandler
    startup_gd32f1x0.o(RESET) refers to chip_uip_interrupt.o(i.SPI0_IRQHandler) for SPI0_IRQHandler
    startup_gd32f1x0.o(RESET) refers to chip_uip_interrupt.o(i.SPI1_IRQHandler) for SPI1_IRQHandler
    startup_gd32f1x0.o(RESET) refers to chip_uip_interrupt.o(i.USART0_IRQHandler) for USART0_IRQHandler
    startup_gd32f1x0.o(RESET) refers to chip_uip_interrupt.o(i.USART1_IRQHandler) for USART1_IRQHandler
    startup_gd32f1x0.o(RESET) refers to chip_uip_interrupt.o(i.CEC_IRQHandler) for CEC_IRQHandler
    startup_gd32f1x0.o(RESET) refers to chip_uip_interrupt.o(i.I2C0_ER_IRQHandler) for I2C0_ER_IRQHandler
    startup_gd32f1x0.o(RESET) refers to chip_uip_interrupt.o(i.I2C1_ER_IRQHandler) for I2C1_ER_IRQHandler
    startup_gd32f1x0.o(RESET) refers to chip_uip_interrupt.o(i.I2C2_EV_IRQHandler) for I2C2_EV_IRQHandler
    startup_gd32f1x0.o(RESET) refers to chip_uip_interrupt.o(i.I2C2_ER_IRQHandler) for I2C2_ER_IRQHandler
    startup_gd32f1x0.o(RESET) refers to chip_uip_interrupt.o(i.USBD_LP_IRQHandler) for USBD_LP_IRQHandler
    startup_gd32f1x0.o(RESET) refers to chip_uip_interrupt.o(i.USBD_HP_IRQHandler) for USBD_HP_IRQHandler
    startup_gd32f1x0.o(RESET) refers to chip_uip_interrupt.o(i.USBDWakeUp_IRQHandler) for USBDWakeUp_IRQHandler
    startup_gd32f1x0.o(RESET) refers to chip_uip_interrupt.o(i.CAN0_TX_IRQHandler) for CAN0_TX_IRQHandler
    startup_gd32f1x0.o(RESET) refers to chip_uip_interrupt.o(i.CAN0_RX0_IRQHandler) for CAN0_RX0_IRQHandler
    startup_gd32f1x0.o(RESET) refers to chip_uip_interrupt.o(i.CAN0_RX1_IRQHandler) for CAN0_RX1_IRQHandler
    startup_gd32f1x0.o(RESET) refers to chip_uip_interrupt.o(i.CAN0_SCE_IRQHandler) for CAN0_SCE_IRQHandler
    startup_gd32f1x0.o(RESET) refers to chip_uip_interrupt.o(i.SLCD_IRQHandler) for SLCD_IRQHandler
    startup_gd32f1x0.o(RESET) refers to chip_uip_interrupt.o(i.DMA_Channel5_6_IRQHandler) for DMA_Channel5_6_IRQHandler
    startup_gd32f1x0.o(RESET) refers to chip_uip_interrupt.o(i.SPI2_IRQHandler) for SPI2_IRQHandler
    startup_gd32f1x0.o(RESET) refers to chip_uip_interrupt.o(i.CAN1_TX_IRQHandler) for CAN1_TX_IRQHandler
    startup_gd32f1x0.o(RESET) refers to chip_uip_interrupt.o(i.CAN1_RX0_IRQHandler) for CAN1_RX0_IRQHandler
    startup_gd32f1x0.o(RESET) refers to chip_uip_interrupt.o(i.CAN1_RX1_IRQHandler) for CAN1_RX1_IRQHandler
    startup_gd32f1x0.o(RESET) refers to chip_uip_interrupt.o(i.CAN1_SCE_IRQHandler) for CAN1_SCE_IRQHandler
    startup_gd32f1x0.o(.text) refers to system_gd32f1x0.o(i.SystemInit) for SystemInit
    startup_gd32f1x0.o(.text) refers to entry.o(.ARM.Collect$$$$00000000) for __main
    gd32f1x0_adc.o(i.adc_deinit) refers to gd32f1x0_rcu.o(i.rcu_periph_reset_enable) for rcu_periph_reset_enable
    gd32f1x0_adc.o(i.adc_deinit) refers to gd32f1x0_rcu.o(i.rcu_periph_reset_disable) for rcu_periph_reset_disable
    gd32f1x0_cec.o(i.cec_deinit) refers to gd32f1x0_rcu.o(i.rcu_periph_reset_enable) for rcu_periph_reset_enable
    gd32f1x0_cec.o(i.cec_deinit) refers to gd32f1x0_rcu.o(i.rcu_periph_reset_disable) for rcu_periph_reset_disable
    gd32f1x0_dac.o(i.dac_deinit) refers to gd32f1x0_rcu.o(i.rcu_periph_reset_enable) for rcu_periph_reset_enable
    gd32f1x0_dac.o(i.dac_deinit) refers to gd32f1x0_rcu.o(i.rcu_periph_reset_disable) for rcu_periph_reset_disable
    gd32f1x0_fmc.o(i.fmc_halfword_program) refers to gd32f1x0_fmc.o(i.fmc_ready_wait) for fmc_ready_wait
    gd32f1x0_fmc.o(i.fmc_mass_erase) refers to gd32f1x0_fmc.o(i.fmc_ready_wait) for fmc_ready_wait
    gd32f1x0_fmc.o(i.fmc_page_erase) refers to gd32f1x0_fmc.o(i.fmc_ready_wait) for fmc_ready_wait
    gd32f1x0_fmc.o(i.fmc_ready_wait) refers to gd32f1x0_fmc.o(i.fmc_state_get) for fmc_state_get
    gd32f1x0_fmc.o(i.fmc_wait_state_disable) refers to gd32f1x0_fmc.o(i.fmc_unlock) for fmc_unlock
    gd32f1x0_fmc.o(i.fmc_wait_state_disable) refers to gd32f1x0_fmc.o(i.fmc_lock) for fmc_lock
    gd32f1x0_fmc.o(i.fmc_wait_state_enable) refers to gd32f1x0_fmc.o(i.fmc_unlock) for fmc_unlock
    gd32f1x0_fmc.o(i.fmc_wait_state_enable) refers to gd32f1x0_fmc.o(i.fmc_lock) for fmc_lock
    gd32f1x0_fmc.o(i.fmc_word_program) refers to gd32f1x0_fmc.o(i.fmc_ready_wait) for fmc_ready_wait
    gd32f1x0_fmc.o(i.ob_data_program) refers to gd32f1x0_fmc.o(i.fmc_ready_wait) for fmc_ready_wait
    gd32f1x0_fmc.o(i.ob_erase) refers to gd32f1x0_fmc.o(i.ob_obstat_plevel_get) for ob_obstat_plevel_get
    gd32f1x0_fmc.o(i.ob_erase) refers to gd32f1x0_fmc.o(i.fmc_ready_wait) for fmc_ready_wait
    gd32f1x0_fmc.o(i.ob_security_protection_config) refers to gd32f1x0_fmc.o(i.fmc_ready_wait) for fmc_ready_wait
    gd32f1x0_fmc.o(i.ob_security_protection_config) refers to gd32f1x0_fmc.o(i.ob_obstat_plevel_get) for ob_obstat_plevel_get
    gd32f1x0_fmc.o(i.ob_user_write) refers to gd32f1x0_fmc.o(i.fmc_ready_wait) for fmc_ready_wait
    gd32f1x0_fmc.o(i.ob_write_protection_enable) refers to gd32f1x0_fmc.o(i.fmc_ready_wait) for fmc_ready_wait
    gd32f1x0_gpio.o(i.gpio_deinit) refers to gd32f1x0_rcu.o(i.rcu_periph_reset_enable) for rcu_periph_reset_enable
    gd32f1x0_gpio.o(i.gpio_deinit) refers to gd32f1x0_rcu.o(i.rcu_periph_reset_disable) for rcu_periph_reset_disable
    gd32f1x0_i2c.o(i.i2c_clock_config) refers to gd32f1x0_rcu.o(i.rcu_clock_freq_get) for rcu_clock_freq_get
    gd32f1x0_i2c.o(i.i2c_deinit) refers to gd32f1x0_rcu.o(i.rcu_periph_reset_enable) for rcu_periph_reset_enable
    gd32f1x0_i2c.o(i.i2c_deinit) refers to gd32f1x0_rcu.o(i.rcu_periph_reset_disable) for rcu_periph_reset_disable
    gd32f1x0_pmu.o(i.pmu_deinit) refers to gd32f1x0_rcu.o(i.rcu_periph_reset_enable) for rcu_periph_reset_enable
    gd32f1x0_pmu.o(i.pmu_deinit) refers to gd32f1x0_rcu.o(i.rcu_periph_reset_disable) for rcu_periph_reset_disable
    gd32f1x0_pmu.o(i.pmu_to_deepsleepmode) refers to gd32f1x0_pmu.o(.bss) for reg_snap
    gd32f1x0_rcu.o(i.rcu_osci_stab_wait) refers to gd32f1x0_rcu.o(i.rcu_flag_get) for rcu_flag_get
    gd32f1x0_rtc.o(i.rtc_deinit) refers to gd32f1x0_rtc.o(i.rtc_init_mode_enter) for rtc_init_mode_enter
    gd32f1x0_rtc.o(i.rtc_deinit) refers to gd32f1x0_rtc.o(i.rtc_register_sync_wait) for rtc_register_sync_wait
    gd32f1x0_rtc.o(i.rtc_init) refers to gd32f1x0_rtc.o(i.rtc_init_mode_enter) for rtc_init_mode_enter
    gd32f1x0_rtc.o(i.rtc_init) refers to gd32f1x0_rtc.o(i.rtc_init_mode_exit) for rtc_init_mode_exit
    gd32f1x0_rtc.o(i.rtc_init) refers to gd32f1x0_rtc.o(i.rtc_register_sync_wait) for rtc_register_sync_wait
    gd32f1x0_rtc.o(i.rtc_refclock_detection_disable) refers to gd32f1x0_rtc.o(i.rtc_init_mode_enter) for rtc_init_mode_enter
    gd32f1x0_rtc.o(i.rtc_refclock_detection_disable) refers to gd32f1x0_rtc.o(i.rtc_init_mode_exit) for rtc_init_mode_exit
    gd32f1x0_rtc.o(i.rtc_refclock_detection_enable) refers to gd32f1x0_rtc.o(i.rtc_init_mode_enter) for rtc_init_mode_enter
    gd32f1x0_rtc.o(i.rtc_refclock_detection_enable) refers to gd32f1x0_rtc.o(i.rtc_init_mode_exit) for rtc_init_mode_exit
    gd32f1x0_rtc.o(i.rtc_second_ajust) refers to gd32f1x0_rtc.o(i.rtc_register_sync_wait) for rtc_register_sync_wait
    gd32f1x0_spi.o(i.i2s_psc_config) refers to gd32f1x0_rcu.o(i.rcu_clock_freq_get) for rcu_clock_freq_get
    gd32f1x0_spi.o(i.spi_i2s_deinit) refers to gd32f1x0_rcu.o(i.rcu_periph_reset_enable) for rcu_periph_reset_enable
    gd32f1x0_spi.o(i.spi_i2s_deinit) refers to gd32f1x0_rcu.o(i.rcu_periph_reset_disable) for rcu_periph_reset_disable
    gd32f1x0_syscfg.o(i.syscfg_deinit) refers to gd32f1x0_rcu.o(i.rcu_periph_reset_enable) for rcu_periph_reset_enable
    gd32f1x0_syscfg.o(i.syscfg_deinit) refers to gd32f1x0_rcu.o(i.rcu_periph_reset_disable) for rcu_periph_reset_disable
    gd32f1x0_timer.o(i.timer_deinit) refers to gd32f1x0_rcu.o(i.rcu_periph_reset_enable) for rcu_periph_reset_enable
    gd32f1x0_timer.o(i.timer_deinit) refers to gd32f1x0_rcu.o(i.rcu_periph_reset_disable) for rcu_periph_reset_disable
    gd32f1x0_timer.o(i.timer_external_clock_mode0_config) refers to gd32f1x0_timer.o(i.timer_external_trigger_config) for timer_external_trigger_config
    gd32f1x0_timer.o(i.timer_external_clock_mode1_config) refers to gd32f1x0_timer.o(i.timer_external_trigger_config) for timer_external_trigger_config
    gd32f1x0_timer.o(i.timer_external_trigger_as_external_clock_config) refers to gd32f1x0_timer.o(i.timer_input_trigger_source_select) for timer_input_trigger_source_select
    gd32f1x0_timer.o(i.timer_input_capture_config) refers to gd32f1x0_timer.o(i.timer_channel_input_capture_prescaler_config) for timer_channel_input_capture_prescaler_config
    gd32f1x0_timer.o(i.timer_input_pwm_capture_config) refers to gd32f1x0_timer.o(i.timer_channel_input_capture_prescaler_config) for timer_channel_input_capture_prescaler_config
    gd32f1x0_timer.o(i.timer_internal_trigger_as_external_clock_config) refers to gd32f1x0_timer.o(i.timer_input_trigger_source_select) for timer_input_trigger_source_select
    gd32f1x0_tsi.o(i.tsi_deinit) refers to gd32f1x0_rcu.o(i.rcu_periph_reset_enable) for rcu_periph_reset_enable
    gd32f1x0_tsi.o(i.tsi_deinit) refers to gd32f1x0_rcu.o(i.rcu_periph_reset_disable) for rcu_periph_reset_disable
    gd32f1x0_usart.o(i.usart_baudrate_set) refers to gd32f1x0_rcu.o(i.rcu_clock_freq_get) for rcu_clock_freq_get
    gd32f1x0_usart.o(i.usart_deinit) refers to gd32f1x0_rcu.o(i.rcu_periph_reset_enable) for rcu_periph_reset_enable
    gd32f1x0_usart.o(i.usart_deinit) refers to gd32f1x0_rcu.o(i.rcu_periph_reset_disable) for rcu_periph_reset_disable
    gd32f1x0_wwdgt.o(i.wwdgt_deinit) refers to gd32f1x0_rcu.o(i.rcu_periph_reset_enable) for rcu_periph_reset_enable
    gd32f1x0_wwdgt.o(i.wwdgt_deinit) refers to gd32f1x0_rcu.o(i.rcu_periph_reset_disable) for rcu_periph_reset_disable
    gd32f1x0_eval.o(i.gd_eval_com_init) refers to gd32f1x0_rcu.o(i.rcu_periph_clock_enable) for rcu_periph_clock_enable
    gd32f1x0_eval.o(i.gd_eval_com_init) refers to gd32f1x0_gpio.o(i.gpio_af_set) for gpio_af_set
    gd32f1x0_eval.o(i.gd_eval_com_init) refers to gd32f1x0_gpio.o(i.gpio_mode_set) for gpio_mode_set
    gd32f1x0_eval.o(i.gd_eval_com_init) refers to gd32f1x0_gpio.o(i.gpio_output_options_set) for gpio_output_options_set
    gd32f1x0_eval.o(i.gd_eval_com_init) refers to gd32f1x0_usart.o(i.usart_deinit) for usart_deinit
    gd32f1x0_eval.o(i.gd_eval_com_init) refers to gd32f1x0_usart.o(i.usart_baudrate_set) for usart_baudrate_set
    gd32f1x0_eval.o(i.gd_eval_com_init) refers to gd32f1x0_usart.o(i.usart_transmit_config) for usart_transmit_config
    gd32f1x0_eval.o(i.gd_eval_com_init) refers to gd32f1x0_usart.o(i.usart_receive_config) for usart_receive_config
    gd32f1x0_eval.o(i.gd_eval_com_init) refers to gd32f1x0_usart.o(i.usart_enable) for usart_enable
    gd32f1x0_eval.o(i.gd_eval_com_init) refers to gd32f1x0_eval.o(.data) for COM_CLK
    gd32f1x0_eval.o(i.gd_eval_key_init) refers to gd32f1x0_rcu.o(i.rcu_periph_clock_enable) for rcu_periph_clock_enable
    gd32f1x0_eval.o(i.gd_eval_key_init) refers to gd32f1x0_gpio.o(i.gpio_mode_set) for gpio_mode_set
    gd32f1x0_eval.o(i.gd_eval_key_init) refers to gd32f1x0_misc.o(i.nvic_irq_enable) for nvic_irq_enable
    gd32f1x0_eval.o(i.gd_eval_key_init) refers to gd32f1x0_syscfg.o(i.syscfg_exti_line_config) for syscfg_exti_line_config
    gd32f1x0_eval.o(i.gd_eval_key_init) refers to gd32f1x0_exti.o(i.exti_init) for exti_init
    gd32f1x0_eval.o(i.gd_eval_key_init) refers to gd32f1x0_exti.o(i.exti_interrupt_flag_clear) for exti_interrupt_flag_clear
    gd32f1x0_eval.o(i.gd_eval_key_init) refers to gd32f1x0_eval.o(.data) for KEY_CLK
    gd32f1x0_eval.o(i.gd_eval_key_state_get) refers to gd32f1x0_gpio.o(i.gpio_input_bit_get) for gpio_input_bit_get
    gd32f1x0_eval.o(i.gd_eval_key_state_get) refers to gd32f1x0_eval.o(.data) for KEY_PIN
    gd32f1x0_eval.o(i.gd_eval_led_init) refers to gd32f1x0_rcu.o(i.rcu_periph_clock_enable) for rcu_periph_clock_enable
    gd32f1x0_eval.o(i.gd_eval_led_init) refers to gd32f1x0_gpio.o(i.gpio_mode_set) for gpio_mode_set
    gd32f1x0_eval.o(i.gd_eval_led_init) refers to gd32f1x0_gpio.o(i.gpio_output_options_set) for gpio_output_options_set
    gd32f1x0_eval.o(i.gd_eval_led_init) refers to gd32f1x0_eval.o(.data) for GPIO_CLK
    gd32f1x0_eval.o(i.gd_eval_led_off) refers to gd32f1x0_eval.o(.data) for GPIO_PIN
    gd32f1x0_eval.o(i.gd_eval_led_on) refers to gd32f1x0_eval.o(.data) for GPIO_PIN
    gd32f1x0_eval.o(i.gd_eval_led_toggle) refers to gd32f1x0_eval.o(.data) for GPIO_PORT
    chip_uip_interrupt.o(i.ADC_CMP_IRQHandler) refers to uip_kernel_isr_engine.o(i.uipInterruptServiceEngine) for uipInterruptServiceEngine
    chip_uip_interrupt.o(i.ADC_CMP_IRQHandler) refers to uip_kernel_common.o(.data) for uipIntTableID
    chip_uip_interrupt.o(i.CAN0_RX0_IRQHandler) refers to uip_kernel_isr_engine.o(i.uipInterruptServiceEngine) for uipInterruptServiceEngine
    chip_uip_interrupt.o(i.CAN0_RX0_IRQHandler) refers to uip_kernel_common.o(.data) for uipIntTableID
    chip_uip_interrupt.o(i.CAN0_RX1_IRQHandler) refers to uip_kernel_isr_engine.o(i.uipInterruptServiceEngine) for uipInterruptServiceEngine
    chip_uip_interrupt.o(i.CAN0_RX1_IRQHandler) refers to uip_kernel_common.o(.data) for uipIntTableID
    chip_uip_interrupt.o(i.CAN0_SCE_IRQHandler) refers to uip_kernel_isr_engine.o(i.uipInterruptServiceEngine) for uipInterruptServiceEngine
    chip_uip_interrupt.o(i.CAN0_SCE_IRQHandler) refers to uip_kernel_common.o(.data) for uipIntTableID
    chip_uip_interrupt.o(i.CAN0_TX_IRQHandler) refers to uip_kernel_isr_engine.o(i.uipInterruptServiceEngine) for uipInterruptServiceEngine
    chip_uip_interrupt.o(i.CAN0_TX_IRQHandler) refers to uip_kernel_common.o(.data) for uipIntTableID
    chip_uip_interrupt.o(i.CAN1_RX0_IRQHandler) refers to uip_kernel_isr_engine.o(i.uipInterruptServiceEngine) for uipInterruptServiceEngine
    chip_uip_interrupt.o(i.CAN1_RX0_IRQHandler) refers to uip_kernel_common.o(.data) for uipIntTableID
    chip_uip_interrupt.o(i.CAN1_RX1_IRQHandler) refers to uip_kernel_isr_engine.o(i.uipInterruptServiceEngine) for uipInterruptServiceEngine
    chip_uip_interrupt.o(i.CAN1_RX1_IRQHandler) refers to uip_kernel_common.o(.data) for uipIntTableID
    chip_uip_interrupt.o(i.CAN1_SCE_IRQHandler) refers to uip_kernel_isr_engine.o(i.uipInterruptServiceEngine) for uipInterruptServiceEngine
    chip_uip_interrupt.o(i.CAN1_SCE_IRQHandler) refers to uip_kernel_common.o(.data) for uipIntTableID
    chip_uip_interrupt.o(i.CAN1_TX_IRQHandler) refers to uip_kernel_isr_engine.o(i.uipInterruptServiceEngine) for uipInterruptServiceEngine
    chip_uip_interrupt.o(i.CAN1_TX_IRQHandler) refers to uip_kernel_common.o(.data) for uipIntTableID
    chip_uip_interrupt.o(i.CEC_IRQHandler) refers to uip_kernel_isr_engine.o(i.uipInterruptServiceEngine) for uipInterruptServiceEngine
    chip_uip_interrupt.o(i.CEC_IRQHandler) refers to uip_kernel_common.o(.data) for uipIntTableID
    chip_uip_interrupt.o(i.Chip_UIP_InterruptInit) refers to chip_uip_interrupt.o(i.Chip_UIP_InterruptRegisterHandler) for Chip_UIP_InterruptRegisterHandler
    chip_uip_interrupt.o(i.Chip_UIP_InterruptInit) refers to app_int_cfg.o(.data) for UIP_Exc_VectorTable
    chip_uip_interrupt.o(i.Chip_UIP_InterruptInit) refers to chip_uip_interrupt.o(i.Chip_UIP_InterruptNullHandler) for Chip_UIP_InterruptNullHandler
    chip_uip_interrupt.o(i.Chip_UIP_InterruptRegisterHandler) refers to app_int_cfg.o(.data) for UIP_Exc_VectorTable
    chip_uip_interrupt.o(i.Chip_UIP_InterruptRemoveHandler) refers to chip_uip_interrupt.o(i.Chip_UIP_InterruptRegisterHandler) for Chip_UIP_InterruptRegisterHandler
    chip_uip_interrupt.o(i.Chip_UIP_InterruptRemoveHandler) refers to chip_uip_interrupt.o(i.Chip_UIP_InterruptNullHandler) for Chip_UIP_InterruptNullHandler
    chip_uip_interrupt.o(i.Chip_UIP_Kernel_Tick_ISR_Handler) refers to uip_kernel_time.o(i.uipSystemCounterHandler) for uipSystemCounterHandler
    chip_uip_interrupt.o(i.DMA_Channel0_IRQHandler) refers to uip_kernel_isr_engine.o(i.uipInterruptServiceEngine) for uipInterruptServiceEngine
    chip_uip_interrupt.o(i.DMA_Channel0_IRQHandler) refers to uip_kernel_common.o(.data) for uipIntTableID
    chip_uip_interrupt.o(i.DMA_Channel1_2_IRQHandler) refers to uip_kernel_isr_engine.o(i.uipInterruptServiceEngine) for uipInterruptServiceEngine
    chip_uip_interrupt.o(i.DMA_Channel1_2_IRQHandler) refers to uip_kernel_common.o(.data) for uipIntTableID
    chip_uip_interrupt.o(i.DMA_Channel3_4_IRQHandler) refers to uip_kernel_isr_engine.o(i.uipInterruptServiceEngine) for uipInterruptServiceEngine
    chip_uip_interrupt.o(i.DMA_Channel3_4_IRQHandler) refers to uip_kernel_common.o(.data) for uipIntTableID
    chip_uip_interrupt.o(i.DMA_Channel5_6_IRQHandler) refers to uip_kernel_isr_engine.o(i.uipInterruptServiceEngine) for uipInterruptServiceEngine
    chip_uip_interrupt.o(i.DMA_Channel5_6_IRQHandler) refers to uip_kernel_common.o(.data) for uipIntTableID
    chip_uip_interrupt.o(i.EXTI0_1_IRQHandler) refers to uip_kernel_isr_engine.o(i.uipInterruptServiceEngine) for uipInterruptServiceEngine
    chip_uip_interrupt.o(i.EXTI0_1_IRQHandler) refers to uip_kernel_common.o(.data) for uipIntTableID
    chip_uip_interrupt.o(i.EXTI2_3_IRQHandler) refers to uip_kernel_isr_engine.o(i.uipInterruptServiceEngine) for uipInterruptServiceEngine
    chip_uip_interrupt.o(i.EXTI2_3_IRQHandler) refers to uip_kernel_common.o(.data) for uipIntTableID
    chip_uip_interrupt.o(i.EXTI4_15_IRQHandler) refers to uip_kernel_isr_engine.o(i.uipInterruptServiceEngine) for uipInterruptServiceEngine
    chip_uip_interrupt.o(i.EXTI4_15_IRQHandler) refers to uip_kernel_common.o(.data) for uipIntTableID
    chip_uip_interrupt.o(i.FMC_IRQHandler) refers to uip_kernel_isr_engine.o(i.uipInterruptServiceEngine) for uipInterruptServiceEngine
    chip_uip_interrupt.o(i.FMC_IRQHandler) refers to uip_kernel_common.o(.data) for uipIntTableID
    chip_uip_interrupt.o(i.I2C0_ER_IRQHandler) refers to uip_kernel_isr_engine.o(i.uipInterruptServiceEngine) for uipInterruptServiceEngine
    chip_uip_interrupt.o(i.I2C0_ER_IRQHandler) refers to uip_kernel_common.o(.data) for uipIntTableID
    chip_uip_interrupt.o(i.I2C0_EV_IRQHandler) refers to uip_kernel_isr_engine.o(i.uipInterruptServiceEngine) for uipInterruptServiceEngine
    chip_uip_interrupt.o(i.I2C0_EV_IRQHandler) refers to uip_kernel_common.o(.data) for uipIntTableID
    chip_uip_interrupt.o(i.I2C1_ER_IRQHandler) refers to uip_kernel_isr_engine.o(i.uipInterruptServiceEngine) for uipInterruptServiceEngine
    chip_uip_interrupt.o(i.I2C1_ER_IRQHandler) refers to uip_kernel_common.o(.data) for uipIntTableID
    chip_uip_interrupt.o(i.I2C1_EV_IRQHandler) refers to uip_kernel_isr_engine.o(i.uipInterruptServiceEngine) for uipInterruptServiceEngine
    chip_uip_interrupt.o(i.I2C1_EV_IRQHandler) refers to uip_kernel_common.o(.data) for uipIntTableID
    chip_uip_interrupt.o(i.I2C2_ER_IRQHandler) refers to uip_kernel_isr_engine.o(i.uipInterruptServiceEngine) for uipInterruptServiceEngine
    chip_uip_interrupt.o(i.I2C2_ER_IRQHandler) refers to uip_kernel_common.o(.data) for uipIntTableID
    chip_uip_interrupt.o(i.I2C2_EV_IRQHandler) refers to uip_kernel_isr_engine.o(i.uipInterruptServiceEngine) for uipInterruptServiceEngine
    chip_uip_interrupt.o(i.I2C2_EV_IRQHandler) refers to uip_kernel_common.o(.data) for uipIntTableID
    chip_uip_interrupt.o(i.InterruptHandler) refers to uip_kernel_common.o(.data) for uipIntTableID
    chip_uip_interrupt.o(i.InterruptHandler) refers to app_int_cfg.o(.data) for UIP_Exc_VectorTable
    chip_uip_interrupt.o(i.LVD_IRQHandler) refers to uip_kernel_isr_engine.o(i.uipInterruptServiceEngine) for uipInterruptServiceEngine
    chip_uip_interrupt.o(i.LVD_IRQHandler) refers to uip_kernel_common.o(.data) for uipIntTableID
    chip_uip_interrupt.o(i.RCU_IRQHandler) refers to uip_kernel_isr_engine.o(i.uipInterruptServiceEngine) for uipInterruptServiceEngine
    chip_uip_interrupt.o(i.RCU_IRQHandler) refers to uip_kernel_common.o(.data) for uipIntTableID
    chip_uip_interrupt.o(i.RTC_IRQHandler) refers to uip_kernel_isr_engine.o(i.uipInterruptServiceEngine) for uipInterruptServiceEngine
    chip_uip_interrupt.o(i.RTC_IRQHandler) refers to uip_kernel_common.o(.data) for uipIntTableID
    chip_uip_interrupt.o(i.SLCD_IRQHandler) refers to uip_kernel_isr_engine.o(i.uipInterruptServiceEngine) for uipInterruptServiceEngine
    chip_uip_interrupt.o(i.SLCD_IRQHandler) refers to uip_kernel_common.o(.data) for uipIntTableID
    chip_uip_interrupt.o(i.SPI0_IRQHandler) refers to uip_kernel_isr_engine.o(i.uipInterruptServiceEngine) for uipInterruptServiceEngine
    chip_uip_interrupt.o(i.SPI0_IRQHandler) refers to uip_kernel_common.o(.data) for uipIntTableID
    chip_uip_interrupt.o(i.SPI1_IRQHandler) refers to uip_kernel_isr_engine.o(i.uipInterruptServiceEngine) for uipInterruptServiceEngine
    chip_uip_interrupt.o(i.SPI1_IRQHandler) refers to uip_kernel_common.o(.data) for uipIntTableID
    chip_uip_interrupt.o(i.SPI2_IRQHandler) refers to uip_kernel_isr_engine.o(i.uipInterruptServiceEngine) for uipInterruptServiceEngine
    chip_uip_interrupt.o(i.SPI2_IRQHandler) refers to uip_kernel_common.o(.data) for uipIntTableID
    chip_uip_interrupt.o(i.TIMER0_BRK_UP_TRG_COM_IRQHandler) refers to uip_kernel_isr_engine.o(i.uipInterruptServiceEngine) for uipInterruptServiceEngine
    chip_uip_interrupt.o(i.TIMER0_BRK_UP_TRG_COM_IRQHandler) refers to uip_kernel_common.o(.data) for uipIntTableID
    chip_uip_interrupt.o(i.TIMER0_Channel_IRQHandler) refers to uip_kernel_isr_engine.o(i.uipInterruptServiceEngine) for uipInterruptServiceEngine
    chip_uip_interrupt.o(i.TIMER0_Channel_IRQHandler) refers to uip_kernel_common.o(.data) for uipIntTableID
    chip_uip_interrupt.o(i.TIMER13_IRQHandler) refers to uip_kernel_isr_engine.o(i.uipInterruptServiceEngine) for uipInterruptServiceEngine
    chip_uip_interrupt.o(i.TIMER13_IRQHandler) refers to uip_kernel_common.o(.data) for uipIntTableID
    chip_uip_interrupt.o(i.TIMER14_IRQHandler) refers to uip_kernel_isr_engine.o(i.uipInterruptServiceEngine) for uipInterruptServiceEngine
    chip_uip_interrupt.o(i.TIMER14_IRQHandler) refers to uip_kernel_common.o(.data) for uipIntTableID
    chip_uip_interrupt.o(i.TIMER15_IRQHandler) refers to uip_kernel_isr_engine.o(i.uipInterruptServiceEngine) for uipInterruptServiceEngine
    chip_uip_interrupt.o(i.TIMER15_IRQHandler) refers to uip_kernel_common.o(.data) for uipIntTableID
    chip_uip_interrupt.o(i.TIMER16_IRQHandler) refers to uip_kernel_isr_engine.o(i.uipInterruptServiceEngine) for uipInterruptServiceEngine
    chip_uip_interrupt.o(i.TIMER16_IRQHandler) refers to uip_kernel_common.o(.data) for uipIntTableID
    chip_uip_interrupt.o(i.TIMER1_IRQHandler) refers to uip_kernel_isr_engine.o(i.uipInterruptServiceEngine) for uipInterruptServiceEngine
    chip_uip_interrupt.o(i.TIMER1_IRQHandler) refers to uip_kernel_common.o(.data) for uipIntTableID
    chip_uip_interrupt.o(i.TIMER2_IRQHandler) refers to uip_kernel_isr_engine.o(i.uipInterruptServiceEngine) for uipInterruptServiceEngine
    chip_uip_interrupt.o(i.TIMER2_IRQHandler) refers to uip_kernel_common.o(.data) for uipIntTableID
    chip_uip_interrupt.o(i.TIMER5_DAC_IRQHandler) refers to uip_kernel_isr_engine.o(i.uipInterruptServiceEngine) for uipInterruptServiceEngine
    chip_uip_interrupt.o(i.TIMER5_DAC_IRQHandler) refers to uip_kernel_common.o(.data) for uipIntTableID
    chip_uip_interrupt.o(i.TSI_IRQHandler) refers to uip_kernel_isr_engine.o(i.uipInterruptServiceEngine) for uipInterruptServiceEngine
    chip_uip_interrupt.o(i.TSI_IRQHandler) refers to uip_kernel_common.o(.data) for uipIntTableID
    chip_uip_interrupt.o(i.USART0_IRQHandler) refers to uip_kernel_isr_engine.o(i.uipInterruptServiceEngine) for uipInterruptServiceEngine
    chip_uip_interrupt.o(i.USART0_IRQHandler) refers to uip_kernel_common.o(.data) for uipIntTableID
    chip_uip_interrupt.o(i.USART1_IRQHandler) refers to uip_kernel_isr_engine.o(i.uipInterruptServiceEngine) for uipInterruptServiceEngine
    chip_uip_interrupt.o(i.USART1_IRQHandler) refers to uip_kernel_common.o(.data) for uipIntTableID
    chip_uip_interrupt.o(i.USBDWakeUp_IRQHandler) refers to uip_kernel_isr_engine.o(i.uipInterruptServiceEngine) for uipInterruptServiceEngine
    chip_uip_interrupt.o(i.USBDWakeUp_IRQHandler) refers to uip_kernel_common.o(.data) for uipIntTableID
    chip_uip_interrupt.o(i.USBD_HP_IRQHandler) refers to uip_kernel_isr_engine.o(i.uipInterruptServiceEngine) for uipInterruptServiceEngine
    chip_uip_interrupt.o(i.USBD_HP_IRQHandler) refers to uip_kernel_common.o(.data) for uipIntTableID
    chip_uip_interrupt.o(i.USBD_LP_IRQHandler) refers to uip_kernel_isr_engine.o(i.uipInterruptServiceEngine) for uipInterruptServiceEngine
    chip_uip_interrupt.o(i.USBD_LP_IRQHandler) refers to uip_kernel_common.o(.data) for uipIntTableID
    chip_uip_interrupt.o(i.WWDGT_IRQHandler) refers to uip_kernel_isr_engine.o(i.uipInterruptServiceEngine) for uipInterruptServiceEngine
    chip_uip_interrupt.o(i.WWDGT_IRQHandler) refers to uip_kernel_common.o(.data) for uipIntTableID
    chip_uip_interrupt.o(i.uipInterruptHandlingCallback) refers to chip_uip_interrupt.o(i.InterruptHandler) for InterruptHandler
    chip_uip_interrupt.o(i.uipInterruptHandlingCallback) refers to uip_kernel_common.o(.data) for uipLowPowerMode
    hardware_init.o(i.Kernel_System_Tick_Init) refers to system_gd32f1x0.o(.data) for SystemCoreClock
    uip_kernel_common.o(i.StartOS) refers to uip_kernel_isr_cm.o(CODE) for uipDisableAllInterrupts
    uip_kernel_common.o(i.StartOS) refers to uip_kernel_common.o(i.uipKernelInitialize) for uipKernelInitialize
    uip_kernel_common.o(i.StartOS) refers to demo.o(i.uipAppInitialize) for uipAppInitialize
    uip_kernel_common.o(i.StartOS) refers to uip_kernel_scheduler.o(.data) for uipSystemMode
    uip_kernel_common.o(i.uipAlarmInfoInit) refers to uip_kernel_common.o(.data) for uipAlarmNumber
    uip_kernel_common.o(i.uipAlarmInitialize) refers to uip_kernel_common.o(.data) for uipAlarmNumber
    uip_kernel_common.o(i.uipKernelInitialize) refers to uip_kernel_common.o(.data) for uipTCBArray
    uip_kernel_common.o(i.uipKernelInitialize) refers to uip_kernel_common.o(.bss) for uipPriorityToTaskID
    uip_kernel_common.o(i.uipKernelInitialize) refers to uip_kernel_scheduler.o(.bss) for uipPrioGrpArray
    uip_kernel_common.o(i.uipKernelInitialize) refers to uip_kernel_scheduler.o(.data) for uipSchedulerLock
    uip_kernel_common.o(i.uipMsgInfoInit) refers to uip_kernel_common.o(.data) for uipMsgNumber
    uip_kernel_common.o(i.uipMsgInitialize) refers to uip_kernel_common.o(.data) for uipMsgNumber
    uip_kernel_common.o(i.uipResInfoInit) refers to uip_kernel_common.o(.data) for uipResNumber
    uip_kernel_common.o(i.uipResInitialize) refers to uip_kernel_common.o(.data) for uipResNumber
    uip_kernel_common.o(i.uipTaskInfoInit) refers to uip_kernel_common.o(.data) for uipTaskNumber
    uip_kernel_common.o(i.uipTaskInitialize) refers to uip_kernel_common.o(i.uipTaskStackInit) for uipTaskStackInit
    uip_kernel_common.o(i.uipTaskInitialize) refers to uip_kernel_common.o(.data) for uipTaskNumber
    uip_kernel_common.o(i.uipTaskInitialize) refers to uip_kernel_common.o(.bss) for uipInitTaskStackPtr
    uip_kernel_common.o(i.uipTaskInitialize) refers to uip_kernel_scheduler.o(.data) for uipPrioGroup
    uip_kernel_common.o(i.uipTaskInitialize) refers to uip_kernel_scheduler.o(.bss) for uipPrioGrpArray
    uip_kernel_event.o(i.UIP_ClearEvent) refers to uip_kernel_isr_cm.o(CODE) for uipDisableAllInterrupts
    uip_kernel_event.o(i.UIP_ClearEvent) refers to uip_kernel_scheduler.o(.data) for uipNestedInterrupts
    uip_kernel_event.o(i.UIP_GetEvent) refers to uip_kernel_isr_cm.o(CODE) for uipDisableAllInterrupts
    uip_kernel_event.o(i.UIP_GetEvent) refers to uip_kernel_scheduler.o(.data) for uipSchedulerLock
    uip_kernel_event.o(i.UIP_GetEvent) refers to uip_kernel_common.o(.data) for uipTCBArray
    uip_kernel_event.o(i.UIP_SetEvent) refers to uip_kernel_isr_cm.o(CODE) for uipDisableAllInterrupts
    uip_kernel_event.o(i.UIP_SetEvent) refers to uip_kernel_scheduler.o(i.uipGetNextPriority) for uipGetNextPriority
    uip_kernel_event.o(i.UIP_SetEvent) refers to uip_kernel_common.o(.data) for uipTCBArray
    uip_kernel_event.o(i.UIP_SetEvent) refers to uip_kernel_scheduler.o(.data) for uipPrioGroup
    uip_kernel_event.o(i.UIP_SetEvent) refers to uip_kernel_scheduler.o(.bss) for uipPrioGrpArray
    uip_kernel_event.o(i.UIP_SetEvent) refers to uip_kernel_common.o(.bss) for uipPriorityToTaskID
    uip_kernel_event.o(i.UIP_WaitEvent) refers to uip_kernel_isr_cm.o(CODE) for uipDisableAllInterrupts
    uip_kernel_event.o(i.UIP_WaitEvent) refers to uip_kernel_scheduler.o(i.uipClearPrioGrpAndArrayBit) for uipClearPrioGrpAndArrayBit
    uip_kernel_event.o(i.UIP_WaitEvent) refers to uip_kernel_scheduler.o(i.uipGetNextTask) for uipGetNextTask
    uip_kernel_event.o(i.UIP_WaitEvent) refers to uip_kernel_scheduler.o(.data) for uipNestedInterrupts
    uip_kernel_isr_cm.o(CODE) refers to uip_kernel_scheduler.o(i.uipPreContexSwitch) for uipPreContexSwitch
    uip_kernel_isr_cm.o(CODE) refers to uip_kernel_scheduler.o(.data) for uipCurrentTaskTCBPtr
    uip_kernel_isr_engine.o(i.uipInterruptServiceEngine) refers to uip_kernel_isr_cm.o(CODE) for uipDisableAllInterrupts
    uip_kernel_isr_engine.o(i.uipInterruptServiceEngine) refers to chip_uip_interrupt.o(i.uipInterruptHandlingCallback) for uipInterruptHandlingCallback
    uip_kernel_isr_engine.o(i.uipInterruptServiceEngine) refers to uip_kernel_scheduler.o(i.uipGetNextTask) for uipGetNextTask
    uip_kernel_isr_engine.o(i.uipInterruptServiceEngine) refers to uip_kernel_scheduler.o(.data) for uipSystemMode
    uip_kernel_isr_engine.o(i.uipInterruptServiceEngine) refers to uip_kernel_common.o(.data) for uipLowPowerMode
    uip_kernel_message.o(i.UIP_GetMessageStatus) refers to uip_kernel_common.o(.data) for uipMsgNumber
    uip_kernel_message.o(i.UIP_ReadFlag) refers to uip_kernel_common.o(.data) for uipMCBArray
    uip_kernel_message.o(i.UIP_ReceiveMessage) refers to uip_kernel_isr_cm.o(CODE) for uipDisableAllInterrupts
    uip_kernel_message.o(i.UIP_ReceiveMessage) refers to uip_kernel_common.o(.data) for uipMsgNumber
    uip_kernel_message.o(i.UIP_ResetFlag) refers to uip_kernel_isr_cm.o(CODE) for uipDisableAllInterrupts
    uip_kernel_message.o(i.UIP_ResetFlag) refers to uip_kernel_common.o(.data) for uipMCBArray
    uip_kernel_message.o(i.UIP_SendMessage) refers to uip_kernel_isr_cm.o(CODE) for uipDisableAllInterrupts
    uip_kernel_message.o(i.UIP_SendMessage) refers to uip_kernel_event.o(i.UIP_SetEvent) for UIP_SetEvent
    uip_kernel_message.o(i.UIP_SendMessage) refers to uip_kernel_task.o(i.UIP_ActivateTask) for UIP_ActivateTask
    uip_kernel_message.o(i.UIP_SendMessage) refers to uip_kernel_common.o(.data) for uipMsgNumber
    uip_kernel_message.o(i.UIP_StartCOM) refers to demo.o(i.uipCOMInit) for uipCOMInit
    uip_kernel_message.o(i.UIP_StopCOM) refers to uip_kernel_common.o(.data) for uipMCBArray
    uip_kernel_resource.o(i.UIP_GetResource) refers to uip_kernel_isr_cm.o(CODE) for uipDisableAllInterrupts
    uip_kernel_resource.o(i.UIP_GetResource) refers to uip_kernel_scheduler.o(.data) for uipNestedInterrupts
    uip_kernel_resource.o(i.UIP_GetResource) refers to uip_kernel_common.o(.data) for uipResNumber
    uip_kernel_resource.o(i.UIP_GetResource) refers to uip_kernel_scheduler.o(.bss) for uipPrioGrpArray
    uip_kernel_resource.o(i.UIP_GetResource) refers to uip_kernel_common.o(.bss) for uipPriorityToTaskID
    uip_kernel_resource.o(i.UIP_ReleaseResource) refers to uip_kernel_isr_cm.o(CODE) for uipDisableAllInterrupts
    uip_kernel_resource.o(i.UIP_ReleaseResource) refers to uip_kernel_scheduler.o(i.uipGetNextPriority) for uipGetNextPriority
    uip_kernel_resource.o(i.UIP_ReleaseResource) refers to uip_kernel_common.o(.data) for uipResNumber
    uip_kernel_resource.o(i.UIP_ReleaseResource) refers to uip_kernel_scheduler.o(.data) for uipCurrentTaskTCBPtr
    uip_kernel_resource.o(i.UIP_ReleaseResource) refers to uip_kernel_scheduler.o(.bss) for uipPrioGrpArray
    uip_kernel_resource.o(i.UIP_ReleaseResource) refers to uip_kernel_common.o(.bss) for uipPriorityToTaskID
    uip_kernel_scheduler.o(i.uipClearPrioGrpAndArrayBit) refers to uip_kernel_scheduler.o(.bss) for uipPrioGrpArray
    uip_kernel_scheduler.o(i.uipClearPrioGrpAndArrayBit) refers to uip_kernel_scheduler.o(.data) for uipPrioGroup
    uip_kernel_scheduler.o(i.uipGetNextPriority) refers to uip_kernel_scheduler.o(.data) for uipPrioGroup
    uip_kernel_scheduler.o(i.uipGetNextPriority) refers to uip_kernel_scheduler.o(.bss) for uipPrioGrpArray
    uip_kernel_scheduler.o(i.uipGetNextTask) refers to uip_kernel_scheduler.o(.data) for uipPrioGroup
    uip_kernel_scheduler.o(i.uipGetNextTask) refers to uip_kernel_scheduler.o(.bss) for uipPrioGrpArray
    uip_kernel_scheduler.o(i.uipGetNextTask) refers to uip_kernel_common.o(.bss) for uipPriorityToTaskID
    uip_kernel_scheduler.o(i.uipGetNextTask) refers to uip_kernel_common.o(.data) for uipTCBArray
    uip_kernel_scheduler.o(i.uipPreContexSwitch) refers to uip_kernel_scheduler.o(i.uipResetPrioGrpAndArrayBit) for uipResetPrioGrpAndArrayBit
    uip_kernel_scheduler.o(i.uipPreContexSwitch) refers to uip_kernel_scheduler.o(.data) for uipNextRunningTaskTCBPtr
    uip_kernel_scheduler.o(i.uipResetPrioGrpAndArrayBit) refers to uip_kernel_scheduler.o(.data) for uipCurrentTaskTCBPtr
    uip_kernel_scheduler.o(i.uipResetPrioGrpAndArrayBit) refers to uip_kernel_scheduler.o(.bss) for uipPrioGrpArray
    uip_kernel_task.o(i.UIP_ActivateTask) refers to uip_kernel_isr_cm.o(CODE) for uipDisableAllInterrupts
    uip_kernel_task.o(i.UIP_ActivateTask) refers to uip_kernel_common.o(.data) for uipTCBArray
    uip_kernel_task.o(i.UIP_ActivateTask) refers to uip_kernel_scheduler.o(.data) for uipPrioGroup
    uip_kernel_task.o(i.UIP_ActivateTask) refers to uip_kernel_scheduler.o(.bss) for uipPrioGrpArray
    uip_kernel_task.o(i.UIP_ChainTask) refers to uip_kernel_isr_cm.o(CODE) for uipDisableAllInterrupts
    uip_kernel_task.o(i.UIP_ChainTask) refers to uip_kernel_scheduler.o(i.uipClearPrioGrpAndArrayBit) for uipClearPrioGrpAndArrayBit
    uip_kernel_task.o(i.UIP_ChainTask) refers to uip_kernel_scheduler.o(i.uipGetNextTask) for uipGetNextTask
    uip_kernel_task.o(i.UIP_ChainTask) refers to uip_kernel_common.o(i.uipTaskStackInit) for uipTaskStackInit
    uip_kernel_task.o(i.UIP_ChainTask) refers to uip_kernel_scheduler.o(.data) for uipNestedInterrupts
    uip_kernel_task.o(i.UIP_ChainTask) refers to uip_kernel_common.o(.data) for uipTCBArray
    uip_kernel_task.o(i.UIP_ChainTask) refers to uip_kernel_scheduler.o(.bss) for uipPrioGrpArray
    uip_kernel_task.o(i.UIP_ChainTask) refers to uip_kernel_common.o(.bss) for uipInitTaskStackPtr
    uip_kernel_task.o(i.UIP_GetTaskID) refers to uip_kernel_scheduler.o(.data) for uipCurrentTaskTCBPtr
    uip_kernel_task.o(i.UIP_GetTaskState) refers to uip_kernel_isr_cm.o(CODE) for uipDisableAllInterrupts
    uip_kernel_task.o(i.UIP_GetTaskState) refers to uip_kernel_common.o(.data) for uipTCBArray
    uip_kernel_task.o(i.UIP_Schedule) refers to uip_kernel_isr_cm.o(CODE) for uipDisableAllInterrupts
    uip_kernel_task.o(i.UIP_Schedule) refers to uip_kernel_scheduler.o(i.uipGetNextPriority) for uipGetNextPriority
    uip_kernel_task.o(i.UIP_Schedule) refers to uip_kernel_scheduler.o(.data) for uipNestedInterrupts
    uip_kernel_task.o(i.UIP_Schedule) refers to uip_kernel_scheduler.o(.bss) for uipPrioGrpArray
    uip_kernel_task.o(i.UIP_Schedule) refers to uip_kernel_common.o(.bss) for uipPriorityToTaskID
    uip_kernel_task.o(i.UIP_Schedule) refers to uip_kernel_common.o(.data) for uipTCBArray
    uip_kernel_task.o(i.UIP_TerminateTask) refers to uip_kernel_isr_cm.o(CODE) for uipDisableAllInterrupts
    uip_kernel_task.o(i.UIP_TerminateTask) refers to uip_kernel_common.o(i.uipTaskStackInit) for uipTaskStackInit
    uip_kernel_task.o(i.UIP_TerminateTask) refers to uip_kernel_scheduler.o(i.uipClearPrioGrpAndArrayBit) for uipClearPrioGrpAndArrayBit
    uip_kernel_task.o(i.UIP_TerminateTask) refers to uip_kernel_scheduler.o(i.uipGetNextTask) for uipGetNextTask
    uip_kernel_task.o(i.UIP_TerminateTask) refers to uip_kernel_scheduler.o(.data) for uipNestedInterrupts
    uip_kernel_task.o(i.UIP_TerminateTask) refers to uip_kernel_common.o(.bss) for uipInitTaskStackPtr
    uip_kernel_task.o(i.UIP_TerminateTask) refers to uip_kernel_scheduler.o(.bss) for uipPrioGrpArray
    uip_kernel_time.o(i.UIP_CancelAlarm) refers to uip_kernel_isr_cm.o(CODE) for uipDisableAllInterrupts
    uip_kernel_time.o(i.UIP_CancelAlarm) refers to uip_kernel_common.o(.data) for uipAlarmNumber
    uip_kernel_time.o(i.UIP_GetAlarm) refers to uip_kernel_isr_cm.o(CODE) for uipDisableAllInterrupts
    uip_kernel_time.o(i.UIP_GetAlarm) refers to uip_kernel_common.o(.data) for uipAlarmNumber
    uip_kernel_time.o(i.UIP_GetAlarmBase) refers to uip_kernel_common.o(.data) for uipAlarmNumber
    uip_kernel_time.o(i.UIP_SetAbsAlarm) refers to uip_kernel_isr_cm.o(CODE) for uipDisableAllInterrupts
    uip_kernel_time.o(i.UIP_SetAbsAlarm) refers to uip_kernel_common.o(.data) for uipAlarmNumber
    uip_kernel_time.o(i.UIP_SetRelAlarm) refers to uip_kernel_isr_cm.o(CODE) for uipDisableAllInterrupts
    uip_kernel_time.o(i.UIP_SetRelAlarm) refers to uip_kernel_common.o(.data) for uipAlarmNumber
    uip_kernel_time.o(i.uipAlarmHandler) refers to uip_kernel_event.o(i.UIP_SetEvent) for UIP_SetEvent
    uip_kernel_time.o(i.uipAlarmHandler) refers to uip_kernel_task.o(i.UIP_ActivateTask) for UIP_ActivateTask
    uip_kernel_time.o(i.uipAlarmHandler) refers to uip_kernel_common.o(.data) for uipACBArray
    uip_kernel_time.o(i.uipGeneralCounterHandler) refers to uip_kernel_time.o(i.uipAlarmHandler) for uipAlarmHandler
    uip_kernel_time.o(i.uipGeneralCounterHandler) refers to uip_kernel_common.o(.data) for uipACBArray
    uip_kernel_time.o(i.uipGetCtrCurrentValue) refers to uip_kernel_isr_cm.o(CODE) for uipDisableAllInterrupts
    uip_kernel_time.o(i.uipGetCtrCurrentValue) refers to uip_kernel_common.o(.data) for uipAlarmNumber
    uip_kernel_time.o(i.uipSystemCounterHandler) refers to uip_kernel_time.o(i.uipAlarmHandler) for uipAlarmHandler
    uip_kernel_time.o(i.uipSystemCounterHandler) refers to uip_kernel_common.o(.bss) for uipSystemCounter
    uip_kernel_time.o(i.uipSystemCounterHandler) refers to uip_kernel_common.o(.data) for uipACBArray
    entry.o(.ARM.Collect$$$$00000000) refers (Special) to entry10a.o(.ARM.Collect$$$$0000000D) for __rt_final_cpp
    entry.o(.ARM.Collect$$$$00000000) refers (Special) to entry11a.o(.ARM.Collect$$$$0000000F) for __rt_final_exit
    entry.o(.ARM.Collect$$$$00000000) refers (Special) to entry7b.o(.ARM.Collect$$$$00000008) for _main_clock
    entry.o(.ARM.Collect$$$$00000000) refers (Special) to entry8b.o(.ARM.Collect$$$$0000000A) for _main_cpp_init
    entry.o(.ARM.Collect$$$$00000000) refers (Special) to entry9a.o(.ARM.Collect$$$$0000000B) for _main_init
    entry.o(.ARM.Collect$$$$00000000) refers (Special) to entry5.o(.ARM.Collect$$$$00000004) for _main_scatterload
    entry.o(.ARM.Collect$$$$00000000) refers (Special) to entry2.o(.ARM.Collect$$$$00000001) for _main_stk
    entry2.o(.ARM.Collect$$$$00000001) refers to entry2.o(.ARM.Collect$$$$00002712) for __lit__00000000
    entry2.o(.ARM.Collect$$$$00002712) refers to startup_gd32f1x0.o(STACK) for __initial_sp
    entry2.o(__vectab_stack_and_reset_area) refers to startup_gd32f1x0.o(STACK) for __initial_sp
    entry2.o(__vectab_stack_and_reset_area) refers to entry.o(.ARM.Collect$$$$00000000) for __main
    entry5.o(.ARM.Collect$$$$00000004) refers to init.o(.text) for __scatterload
    entry9a.o(.ARM.Collect$$$$0000000B) refers to main.o(i.main) for main
    entry9b.o(.ARM.Collect$$$$0000000C) refers to main.o(i.main) for main
    init.o(.text) refers to entry5.o(.ARM.Collect$$$$00000004) for __main_after_scatterload


==============================================================================

Removing Unused input sections from the image.

    Removing gd32f1x0_it.o(.rev16_text), (4 bytes).
    Removing gd32f1x0_it.o(.revsh_text), (4 bytes).
    Removing main.o(.rev16_text), (4 bytes).
    Removing main.o(.revsh_text), (4 bytes).
    Removing main.o(i.fputc), (40 bytes).
    Removing app_int_cfg.o(.rev16_text), (4 bytes).
    Removing app_int_cfg.o(.revsh_text), (4 bytes).
    Removing demo.o(.rev16_text), (4 bytes).
    Removing demo.o(.revsh_text), (4 bytes).
    Removing demo.o(i.uipCOMInit), (4 bytes).
    Removing hook.o(i.COMErrorHook), (2 bytes).
    Removing hook.o(i.ErrorHook), (2 bytes).
    Removing hook.o(i.PostTaskHook), (2 bytes).
    Removing hook.o(i.PreTaskHook), (2 bytes).
    Removing hook.o(i.ShutdownHook), (2 bytes).
    Removing hook.o(i.StuipCOMExtension), (4 bytes).
    Removing hook.o(i.StuipupHook), (2 bytes).
    Removing system_gd32f1x0.o(.rev16_text), (4 bytes).
    Removing system_gd32f1x0.o(.revsh_text), (4 bytes).
    Removing system_gd32f1x0.o(i.SystemCoreClockUpdate), (240 bytes).
    Removing startup_gd32f1x0.o(HEAP), (512 bytes).
    Removing gd32f1x0_adc.o(.rev16_text), (4 bytes).
    Removing gd32f1x0_adc.o(.revsh_text), (4 bytes).
    Removing gd32f1x0_adc.o(i.adc_calibration_enable), (60 bytes).
    Removing gd32f1x0_adc.o(i.adc_channel_length_config), (88 bytes).
    Removing gd32f1x0_adc.o(i.adc_data_alignment_config), (36 bytes).
    Removing gd32f1x0_adc.o(i.adc_deinit), (20 bytes).
    Removing gd32f1x0_adc.o(i.adc_disable), (20 bytes).
    Removing gd32f1x0_adc.o(i.adc_discontinuous_mode_config), (84 bytes).
    Removing gd32f1x0_adc.o(i.adc_dma_mode_disable), (20 bytes).
    Removing gd32f1x0_adc.o(i.adc_dma_mode_enable), (20 bytes).
    Removing gd32f1x0_adc.o(i.adc_enable), (28 bytes).
    Removing gd32f1x0_adc.o(i.adc_external_trigger_config), (84 bytes).
    Removing gd32f1x0_adc.o(i.adc_external_trigger_source_config), (64 bytes).
    Removing gd32f1x0_adc.o(i.adc_flag_clear), (16 bytes).
    Removing gd32f1x0_adc.o(i.adc_flag_get), (20 bytes).
    Removing gd32f1x0_adc.o(i.adc_inserted_channel_config), (144 bytes).
    Removing gd32f1x0_adc.o(i.adc_inserted_channel_offset_config), (48 bytes).
    Removing gd32f1x0_adc.o(i.adc_inserted_data_read), (64 bytes).
    Removing gd32f1x0_adc.o(i.adc_interrupt_disable), (60 bytes).
    Removing gd32f1x0_adc.o(i.adc_interrupt_enable), (60 bytes).
    Removing gd32f1x0_adc.o(i.adc_interrupt_flag_clear), (16 bytes).
    Removing gd32f1x0_adc.o(i.adc_interrupt_flag_get), (108 bytes).
    Removing gd32f1x0_adc.o(i.adc_regular_channel_config), (220 bytes).
    Removing gd32f1x0_adc.o(i.adc_regular_data_read), (12 bytes).
    Removing gd32f1x0_adc.o(i.adc_software_trigger_enable), (44 bytes).
    Removing gd32f1x0_adc.o(i.adc_special_function_config), (128 bytes).
    Removing gd32f1x0_adc.o(i.adc_tempsensor_vrefint_disable), (20 bytes).
    Removing gd32f1x0_adc.o(i.adc_tempsensor_vrefint_enable), (20 bytes).
    Removing gd32f1x0_adc.o(i.adc_vbat_disable), (20 bytes).
    Removing gd32f1x0_adc.o(i.adc_vbat_enable), (20 bytes).
    Removing gd32f1x0_adc.o(i.adc_watchdog_disable), (24 bytes).
    Removing gd32f1x0_adc.o(i.adc_watchdog_group_channel_enable), (84 bytes).
    Removing gd32f1x0_adc.o(i.adc_watchdog_single_channel_enable), (48 bytes).
    Removing gd32f1x0_adc.o(i.adc_watchdog_threshold_config), (16 bytes).
    Removing gd32f1x0_cec.o(.rev16_text), (4 bytes).
    Removing gd32f1x0_cec.o(.revsh_text), (4 bytes).
    Removing gd32f1x0_cec.o(i.cec_data_receive), (12 bytes).
    Removing gd32f1x0_cec.o(i.cec_data_send), (12 bytes).
    Removing gd32f1x0_cec.o(i.cec_deinit), (20 bytes).
    Removing gd32f1x0_cec.o(i.cec_disable), (20 bytes).
    Removing gd32f1x0_cec.o(i.cec_enable), (20 bytes).
    Removing gd32f1x0_cec.o(i.cec_error_config), (56 bytes).
    Removing gd32f1x0_cec.o(i.cec_flag_clear), (16 bytes).
    Removing gd32f1x0_cec.o(i.cec_flag_get), (24 bytes).
    Removing gd32f1x0_cec.o(i.cec_generate_errorbit_config), (32 bytes).
    Removing gd32f1x0_cec.o(i.cec_init), (60 bytes).
    Removing gd32f1x0_cec.o(i.cec_interrupt_disable), (16 bytes).
    Removing gd32f1x0_cec.o(i.cec_interrupt_enable), (16 bytes).
    Removing gd32f1x0_cec.o(i.cec_interrupt_flag_clear), (12 bytes).
    Removing gd32f1x0_cec.o(i.cec_interrupt_flag_get), (40 bytes).
    Removing gd32f1x0_cec.o(i.cec_listen_mode_disable), (20 bytes).
    Removing gd32f1x0_cec.o(i.cec_listen_mode_enable), (20 bytes).
    Removing gd32f1x0_cec.o(i.cec_own_address_config), (36 bytes).
    Removing gd32f1x0_cec.o(i.cec_reception_tolerance_disable), (20 bytes).
    Removing gd32f1x0_cec.o(i.cec_reception_tolerance_enable), (20 bytes).
    Removing gd32f1x0_cec.o(i.cec_sft_config), (28 bytes).
    Removing gd32f1x0_cec.o(i.cec_stop_receive_bre_config), (36 bytes).
    Removing gd32f1x0_cec.o(i.cec_transmission_end), (20 bytes).
    Removing gd32f1x0_cec.o(i.cec_transmission_start), (20 bytes).
    Removing gd32f1x0_cmp.o(.rev16_text), (4 bytes).
    Removing gd32f1x0_cmp.o(.revsh_text), (4 bytes).
    Removing gd32f1x0_cmp.o(i.cmp_deinit), (12 bytes).
    Removing gd32f1x0_cmp.o(i.cmp_disable), (36 bytes).
    Removing gd32f1x0_cmp.o(i.cmp_enable), (36 bytes).
    Removing gd32f1x0_cmp.o(i.cmp_lock_disable), (36 bytes).
    Removing gd32f1x0_cmp.o(i.cmp_lock_enable), (36 bytes).
    Removing gd32f1x0_cmp.o(i.cmp_mode_init), (84 bytes).
    Removing gd32f1x0_cmp.o(i.cmp_output_init), (104 bytes).
    Removing gd32f1x0_cmp.o(i.cmp_output_level_get), (44 bytes).
    Removing gd32f1x0_cmp.o(i.cmp_switch_disable), (20 bytes).
    Removing gd32f1x0_cmp.o(i.cmp_switch_enable), (20 bytes).
    Removing gd32f1x0_cmp.o(i.cmp_window_disable), (20 bytes).
    Removing gd32f1x0_cmp.o(i.cmp_window_enable), (20 bytes).
    Removing gd32f1x0_crc.o(.rev16_text), (4 bytes).
    Removing gd32f1x0_crc.o(.revsh_text), (4 bytes).
    Removing gd32f1x0_crc.o(i.crc_block_data_calculate), (36 bytes).
    Removing gd32f1x0_crc.o(i.crc_data_register_read), (12 bytes).
    Removing gd32f1x0_crc.o(i.crc_data_register_reset), (20 bytes).
    Removing gd32f1x0_crc.o(i.crc_deinit), (24 bytes).
    Removing gd32f1x0_crc.o(i.crc_free_data_register_read), (12 bytes).
    Removing gd32f1x0_crc.o(i.crc_free_data_register_write), (12 bytes).
    Removing gd32f1x0_crc.o(i.crc_init_data_register_write), (12 bytes).
    Removing gd32f1x0_crc.o(i.crc_input_data_reverse_config), (28 bytes).
    Removing gd32f1x0_crc.o(i.crc_reverse_output_data_disable), (20 bytes).
    Removing gd32f1x0_crc.o(i.crc_reverse_output_data_enable), (28 bytes).
    Removing gd32f1x0_crc.o(i.crc_single_data_calculate), (16 bytes).
    Removing gd32f1x0_dac.o(.rev16_text), (4 bytes).
    Removing gd32f1x0_dac.o(.revsh_text), (4 bytes).
    Removing gd32f1x0_dac.o(i.dac0_data_set), (44 bytes).
    Removing gd32f1x0_dac.o(i.dac0_disable), (20 bytes).
    Removing gd32f1x0_dac.o(i.dac0_dma_disable), (20 bytes).
    Removing gd32f1x0_dac.o(i.dac0_dma_enable), (20 bytes).
    Removing gd32f1x0_dac.o(i.dac0_enable), (20 bytes).
    Removing gd32f1x0_dac.o(i.dac0_flag_clear), (20 bytes).
    Removing gd32f1x0_dac.o(i.dac0_flag_get), (24 bytes).
    Removing gd32f1x0_dac.o(i.dac0_interrupt_disable), (20 bytes).
    Removing gd32f1x0_dac.o(i.dac0_interrupt_enable), (20 bytes).
    Removing gd32f1x0_dac.o(i.dac0_interrupt_flag_clear), (20 bytes).
    Removing gd32f1x0_dac.o(i.dac0_interrupt_flag_get), (40 bytes).
    Removing gd32f1x0_dac.o(i.dac0_output_buffer_disable), (20 bytes).
    Removing gd32f1x0_dac.o(i.dac0_output_buffer_enable), (20 bytes).
    Removing gd32f1x0_dac.o(i.dac0_output_value_get), (16 bytes).
    Removing gd32f1x0_dac.o(i.dac0_software_trigger_disable), (20 bytes).
    Removing gd32f1x0_dac.o(i.dac0_software_trigger_enable), (20 bytes).
    Removing gd32f1x0_dac.o(i.dac0_trigger_disable), (20 bytes).
    Removing gd32f1x0_dac.o(i.dac0_trigger_enable), (20 bytes).
    Removing gd32f1x0_dac.o(i.dac0_trigger_source_config), (28 bytes).
    Removing gd32f1x0_dac.o(i.dac_deinit), (20 bytes).
    Removing gd32f1x0_dbg.o(.rev16_text), (4 bytes).
    Removing gd32f1x0_dbg.o(.revsh_text), (4 bytes).
    Removing gd32f1x0_dbg.o(i.dbg_deinit), (16 bytes).
    Removing gd32f1x0_dbg.o(i.dbg_id_get), (12 bytes).
    Removing gd32f1x0_dbg.o(i.dbg_low_power_disable), (16 bytes).
    Removing gd32f1x0_dbg.o(i.dbg_low_power_enable), (16 bytes).
    Removing gd32f1x0_dbg.o(i.dbg_periph_disable), (32 bytes).
    Removing gd32f1x0_dbg.o(i.dbg_periph_enable), (32 bytes).
    Removing gd32f1x0_dma.o(.rev16_text), (4 bytes).
    Removing gd32f1x0_dma.o(.revsh_text), (4 bytes).
    Removing gd32f1x0_dma.o(i.dma_channel_disable), (36 bytes).
    Removing gd32f1x0_dma.o(i.dma_channel_enable), (36 bytes).
    Removing gd32f1x0_dma.o(i.dma_circulation_disable), (36 bytes).
    Removing gd32f1x0_dma.o(i.dma_circulation_enable), (36 bytes).
    Removing gd32f1x0_dma.o(i.dma_deinit), (92 bytes).
    Removing gd32f1x0_dma.o(i.dma_flag_clear), (24 bytes).
    Removing gd32f1x0_dma.o(i.dma_flag_get), (32 bytes).
    Removing gd32f1x0_dma.o(i.dma_init), (276 bytes).
    Removing gd32f1x0_dma.o(i.dma_interrupt_disable), (36 bytes).
    Removing gd32f1x0_dma.o(i.dma_interrupt_enable), (36 bytes).
    Removing gd32f1x0_dma.o(i.dma_interrupt_flag_clear), (24 bytes).
    Removing gd32f1x0_dma.o(i.dma_interrupt_flag_get), (196 bytes).
    Removing gd32f1x0_dma.o(i.dma_memory_address_config), (20 bytes).
    Removing gd32f1x0_dma.o(i.dma_memory_increase_disable), (36 bytes).
    Removing gd32f1x0_dma.o(i.dma_memory_increase_enable), (36 bytes).
    Removing gd32f1x0_dma.o(i.dma_memory_to_memory_disable), (36 bytes).
    Removing gd32f1x0_dma.o(i.dma_memory_to_memory_enable), (36 bytes).
    Removing gd32f1x0_dma.o(i.dma_memory_width_config), (40 bytes).
    Removing gd32f1x0_dma.o(i.dma_periph_address_config), (20 bytes).
    Removing gd32f1x0_dma.o(i.dma_periph_increase_disable), (36 bytes).
    Removing gd32f1x0_dma.o(i.dma_periph_increase_enable), (36 bytes).
    Removing gd32f1x0_dma.o(i.dma_periph_width_config), (40 bytes).
    Removing gd32f1x0_dma.o(i.dma_priority_config), (40 bytes).
    Removing gd32f1x0_dma.o(i.dma_transfer_direction_config), (68 bytes).
    Removing gd32f1x0_dma.o(i.dma_transfer_number_config), (20 bytes).
    Removing gd32f1x0_dma.o(i.dma_transfer_number_get), (20 bytes).
    Removing gd32f1x0_exti.o(.rev16_text), (4 bytes).
    Removing gd32f1x0_exti.o(.revsh_text), (4 bytes).
    Removing gd32f1x0_exti.o(i.exti_deinit), (32 bytes).
    Removing gd32f1x0_exti.o(i.exti_event_disable), (16 bytes).
    Removing gd32f1x0_exti.o(i.exti_event_enable), (16 bytes).
    Removing gd32f1x0_exti.o(i.exti_flag_clear), (12 bytes).
    Removing gd32f1x0_exti.o(i.exti_flag_get), (24 bytes).
    Removing gd32f1x0_exti.o(i.exti_init), (184 bytes).
    Removing gd32f1x0_exti.o(i.exti_interrupt_disable), (16 bytes).
    Removing gd32f1x0_exti.o(i.exti_interrupt_enable), (16 bytes).
    Removing gd32f1x0_exti.o(i.exti_interrupt_flag_clear), (12 bytes).
    Removing gd32f1x0_exti.o(i.exti_interrupt_flag_get), (36 bytes).
    Removing gd32f1x0_exti.o(i.exti_software_interrupt_disable), (16 bytes).
    Removing gd32f1x0_exti.o(i.exti_software_interrupt_enable), (16 bytes).
    Removing gd32f1x0_fmc.o(.rev16_text), (4 bytes).
    Removing gd32f1x0_fmc.o(.revsh_text), (4 bytes).
    Removing gd32f1x0_fmc.o(i.fmc_flag_clear), (12 bytes).
    Removing gd32f1x0_fmc.o(i.fmc_flag_get), (20 bytes).
    Removing gd32f1x0_fmc.o(i.fmc_halfword_program), (64 bytes).
    Removing gd32f1x0_fmc.o(i.fmc_interrupt_disable), (16 bytes).
    Removing gd32f1x0_fmc.o(i.fmc_interrupt_enable), (16 bytes).
    Removing gd32f1x0_fmc.o(i.fmc_lock), (20 bytes).
    Removing gd32f1x0_fmc.o(i.fmc_mass_erase), (68 bytes).
    Removing gd32f1x0_fmc.o(i.fmc_page_erase), (72 bytes).
    Removing gd32f1x0_fmc.o(i.fmc_ready_wait), (34 bytes).
    Removing gd32f1x0_fmc.o(i.fmc_state_get), (48 bytes).
    Removing gd32f1x0_fmc.o(i.fmc_unlock), (36 bytes).
    Removing gd32f1x0_fmc.o(i.fmc_wait_state_disable), (32 bytes).
    Removing gd32f1x0_fmc.o(i.fmc_wait_state_enable), (32 bytes).
    Removing gd32f1x0_fmc.o(i.fmc_word_program), (64 bytes).
    Removing gd32f1x0_fmc.o(i.fmc_wscnt_set), (24 bytes).
    Removing gd32f1x0_fmc.o(i.ob_data_get), (12 bytes).
    Removing gd32f1x0_fmc.o(i.ob_data_program), (68 bytes).
    Removing gd32f1x0_fmc.o(i.ob_erase), (156 bytes).
    Removing gd32f1x0_fmc.o(i.ob_lock), (20 bytes).
    Removing gd32f1x0_fmc.o(i.ob_obstat_plevel_get), (16 bytes).
    Removing gd32f1x0_fmc.o(i.ob_reset), (20 bytes).
    Removing gd32f1x0_fmc.o(i.ob_security_protection_config), (144 bytes).
    Removing gd32f1x0_fmc.o(i.ob_unlock), (36 bytes).
    Removing gd32f1x0_fmc.o(i.ob_user_get), (16 bytes).
    Removing gd32f1x0_fmc.o(i.ob_user_write), (76 bytes).
    Removing gd32f1x0_fmc.o(i.ob_write_protection_enable), (104 bytes).
    Removing gd32f1x0_fmc.o(i.ob_write_protection_get), (12 bytes).
    Removing gd32f1x0_fwdgt.o(.rev16_text), (4 bytes).
    Removing gd32f1x0_fwdgt.o(.revsh_text), (4 bytes).
    Removing gd32f1x0_fwdgt.o(i.fwdgt_config), (104 bytes).
    Removing gd32f1x0_fwdgt.o(i.fwdgt_counter_reload), (16 bytes).
    Removing gd32f1x0_fwdgt.o(i.fwdgt_enable), (16 bytes).
    Removing gd32f1x0_fwdgt.o(i.fwdgt_flag_get), (24 bytes).
    Removing gd32f1x0_fwdgt.o(i.fwdgt_window_value_config), (64 bytes).
    Removing gd32f1x0_fwdgt.o(i.fwdgt_write_disable), (12 bytes).
    Removing gd32f1x0_gpio.o(.rev16_text), (4 bytes).
    Removing gd32f1x0_gpio.o(.revsh_text), (4 bytes).
    Removing gd32f1x0_gpio.o(i.gpio_bit_reset), (4 bytes).
    Removing gd32f1x0_gpio.o(i.gpio_bit_set), (4 bytes).
    Removing gd32f1x0_gpio.o(i.gpio_bit_write), (10 bytes).
    Removing gd32f1x0_gpio.o(i.gpio_deinit), (148 bytes).
    Removing gd32f1x0_gpio.o(i.gpio_input_bit_get), (16 bytes).
    Removing gd32f1x0_gpio.o(i.gpio_input_port_get), (8 bytes).
    Removing gd32f1x0_gpio.o(i.gpio_output_bit_get), (16 bytes).
    Removing gd32f1x0_gpio.o(i.gpio_output_port_get), (8 bytes).
    Removing gd32f1x0_gpio.o(i.gpio_pin_lock), (18 bytes).
    Removing gd32f1x0_gpio.o(i.gpio_port_write), (4 bytes).
    Removing gd32f1x0_i2c.o(.rev16_text), (4 bytes).
    Removing gd32f1x0_i2c.o(.revsh_text), (4 bytes).
    Removing gd32f1x0_i2c.o(i.i2c_ack_config), (24 bytes).
    Removing gd32f1x0_i2c.o(i.i2c_ackpos_config), (22 bytes).
    Removing gd32f1x0_i2c.o(i.i2c_clock_config), (216 bytes).
    Removing gd32f1x0_i2c.o(i.i2c_data_receive), (8 bytes).
    Removing gd32f1x0_i2c.o(i.i2c_data_transmit), (6 bytes).
    Removing gd32f1x0_i2c.o(i.i2c_deinit), (64 bytes).
    Removing gd32f1x0_i2c.o(i.i2c_disable), (10 bytes).
    Removing gd32f1x0_i2c.o(i.i2c_dma_enable), (16 bytes).
    Removing gd32f1x0_i2c.o(i.i2c_dma_last_transfer_enable), (16 bytes).
    Removing gd32f1x0_i2c.o(i.i2c_dualaddr_enable), (24 bytes).
    Removing gd32f1x0_i2c.o(i.i2c_enable), (10 bytes).
    Removing gd32f1x0_i2c.o(i.i2c_flag_clear), (18 bytes).
    Removing gd32f1x0_i2c.o(i.i2c_flag_get), (50 bytes).
    Removing gd32f1x0_i2c.o(i.i2c_interrupt_disable), (8 bytes).
    Removing gd32f1x0_i2c.o(i.i2c_interrupt_enable), (8 bytes).
    Removing gd32f1x0_i2c.o(i.i2c_interrupt_flag_clear), (18 bytes).
    Removing gd32f1x0_i2c.o(i.i2c_interrupt_flag_get), (94 bytes).
    Removing gd32f1x0_i2c.o(i.i2c_master_addressing), (20 bytes).
    Removing gd32f1x0_i2c.o(i.i2c_mode_addr_config), (24 bytes).
    Removing gd32f1x0_i2c.o(i.i2c_pec_enable), (16 bytes).
    Removing gd32f1x0_i2c.o(i.i2c_pec_transfer_enable), (16 bytes).
    Removing gd32f1x0_i2c.o(i.i2c_pec_value_get), (10 bytes).
    Removing gd32f1x0_i2c.o(i.i2c_slave_response_to_gcall_config), (16 bytes).
    Removing gd32f1x0_i2c.o(i.i2c_smbus_arp_enable), (16 bytes).
    Removing gd32f1x0_i2c.o(i.i2c_smbus_issue_alert), (16 bytes).
    Removing gd32f1x0_i2c.o(i.i2c_smbus_type_config), (24 bytes).
    Removing gd32f1x0_i2c.o(i.i2c_software_reset_config), (16 bytes).
    Removing gd32f1x0_i2c.o(i.i2c_start_on_bus), (10 bytes).
    Removing gd32f1x0_i2c.o(i.i2c_stop_on_bus), (10 bytes).
    Removing gd32f1x0_i2c.o(i.i2c_stretch_scl_low_config), (16 bytes).
    Removing gd32f1x0_misc.o(.rev16_text), (4 bytes).
    Removing gd32f1x0_misc.o(.revsh_text), (4 bytes).
    Removing gd32f1x0_misc.o(i.nvic_irq_disable), (24 bytes).
    Removing gd32f1x0_misc.o(i.nvic_priority_group_set), (20 bytes).
    Removing gd32f1x0_misc.o(i.nvic_vector_table_set), (20 bytes).
    Removing gd32f1x0_misc.o(i.system_lowpower_reset), (16 bytes).
    Removing gd32f1x0_misc.o(i.system_lowpower_set), (16 bytes).
    Removing gd32f1x0_misc.o(i.systick_clksource_set), (40 bytes).
    Removing gd32f1x0_pmu.o(.rev16_text), (4 bytes).
    Removing gd32f1x0_pmu.o(.revsh_text), (4 bytes).
    Removing gd32f1x0_pmu.o(i.pmu_backup_write_disable), (20 bytes).
    Removing gd32f1x0_pmu.o(i.pmu_backup_write_enable), (20 bytes).
    Removing gd32f1x0_pmu.o(i.pmu_deinit), (20 bytes).
    Removing gd32f1x0_pmu.o(i.pmu_flag_clear), (48 bytes).
    Removing gd32f1x0_pmu.o(i.pmu_flag_get), (24 bytes).
    Removing gd32f1x0_pmu.o(i.pmu_lvd_disable), (20 bytes).
    Removing gd32f1x0_pmu.o(i.pmu_lvd_select), (48 bytes).
    Removing gd32f1x0_pmu.o(i.pmu_to_deepsleepmode), (196 bytes).
    Removing gd32f1x0_pmu.o(i.pmu_to_sleepmode), (28 bytes).
    Removing gd32f1x0_pmu.o(i.pmu_to_standbymode), (52 bytes).
    Removing gd32f1x0_pmu.o(i.pmu_wakeup_pin_disable), (16 bytes).
    Removing gd32f1x0_pmu.o(i.pmu_wakeup_pin_enable), (16 bytes).
    Removing gd32f1x0_pmu.o(.bss), (16 bytes).
    Removing gd32f1x0_rcu.o(.rev16_text), (4 bytes).
    Removing gd32f1x0_rcu.o(.revsh_text), (4 bytes).
    Removing gd32f1x0_rcu.o(i.rcu_adc_clock_config), (152 bytes).
    Removing gd32f1x0_rcu.o(i.rcu_ahb_clock_config), (28 bytes).
    Removing gd32f1x0_rcu.o(i.rcu_all_reset_flag_clear), (20 bytes).
    Removing gd32f1x0_rcu.o(i.rcu_apb1_clock_config), (28 bytes).
    Removing gd32f1x0_rcu.o(i.rcu_apb2_clock_config), (28 bytes).
    Removing gd32f1x0_rcu.o(i.rcu_bkp_reset_disable), (20 bytes).
    Removing gd32f1x0_rcu.o(i.rcu_bkp_reset_enable), (20 bytes).
    Removing gd32f1x0_rcu.o(i.rcu_cec_clock_config), (28 bytes).
    Removing gd32f1x0_rcu.o(i.rcu_ckout_config), (28 bytes).
    Removing gd32f1x0_rcu.o(i.rcu_deepsleep_voltage_set), (36 bytes).
    Removing gd32f1x0_rcu.o(i.rcu_deinit), (128 bytes).
    Removing gd32f1x0_rcu.o(i.rcu_flag_get), (36 bytes).
    Removing gd32f1x0_rcu.o(i.rcu_hxtal_clock_monitor_disable), (20 bytes).
    Removing gd32f1x0_rcu.o(i.rcu_hxtal_clock_monitor_enable), (20 bytes).
    Removing gd32f1x0_rcu.o(i.rcu_hxtal_prediv_config), (24 bytes).
    Removing gd32f1x0_rcu.o(i.rcu_interrupt_disable), (16 bytes).
    Removing gd32f1x0_rcu.o(i.rcu_interrupt_enable), (16 bytes).
    Removing gd32f1x0_rcu.o(i.rcu_interrupt_flag_clear), (16 bytes).
    Removing gd32f1x0_rcu.o(i.rcu_interrupt_flag_get), (24 bytes).
    Removing gd32f1x0_rcu.o(i.rcu_irc14m_adjust_value_set), (24 bytes).
    Removing gd32f1x0_rcu.o(i.rcu_irc8m_adjust_value_set), (24 bytes).
    Removing gd32f1x0_rcu.o(i.rcu_lxtal_drive_capability_config), (28 bytes).
    Removing gd32f1x0_rcu.o(i.rcu_osci_bypass_mode_disable), (100 bytes).
    Removing gd32f1x0_rcu.o(i.rcu_osci_bypass_mode_enable), (100 bytes).
    Removing gd32f1x0_rcu.o(i.rcu_osci_off), (32 bytes).
    Removing gd32f1x0_rcu.o(i.rcu_osci_on), (32 bytes).
    Removing gd32f1x0_rcu.o(i.rcu_osci_stab_wait), (268 bytes).
    Removing gd32f1x0_rcu.o(i.rcu_periph_clock_disable), (32 bytes).
    Removing gd32f1x0_rcu.o(i.rcu_periph_clock_sleep_disable), (32 bytes).
    Removing gd32f1x0_rcu.o(i.rcu_periph_clock_sleep_enable), (32 bytes).
    Removing gd32f1x0_rcu.o(i.rcu_pll_config), (36 bytes).
    Removing gd32f1x0_rcu.o(i.rcu_power_down_voltage_set), (36 bytes).
    Removing gd32f1x0_rcu.o(i.rcu_rtc_clock_config), (28 bytes).
    Removing gd32f1x0_rcu.o(i.rcu_system_clock_source_config), (28 bytes).
    Removing gd32f1x0_rcu.o(i.rcu_system_clock_source_get), (16 bytes).
    Removing gd32f1x0_rcu.o(i.rcu_usart_clock_config), (28 bytes).
    Removing gd32f1x0_rcu.o(i.rcu_usbd_clock_config), (28 bytes).
    Removing gd32f1x0_rcu.o(i.rcu_voltage_key_unlock), (40 bytes).
    Removing gd32f1x0_rtc.o(.rev16_text), (4 bytes).
    Removing gd32f1x0_rtc.o(.revsh_text), (4 bytes).
    Removing gd32f1x0_rtc.o(i.rtc_alarm_config), (84 bytes).
    Removing gd32f1x0_rtc.o(i.rtc_alarm_disable), (80 bytes).
    Removing gd32f1x0_rtc.o(i.rtc_alarm_enable), (40 bytes).
    Removing gd32f1x0_rtc.o(i.rtc_alarm_get), (56 bytes).
    Removing gd32f1x0_rtc.o(i.rtc_alarm_subsecond_config), (32 bytes).
    Removing gd32f1x0_rtc.o(i.rtc_alarm_subsecond_get), (16 bytes).
    Removing gd32f1x0_rtc.o(i.rtc_alter_output_config), (76 bytes).
    Removing gd32f1x0_rtc.o(i.rtc_bypass_shadow_disable), (40 bytes).
    Removing gd32f1x0_rtc.o(i.rtc_bypass_shadow_enable), (40 bytes).
    Removing gd32f1x0_rtc.o(i.rtc_calibration_config), (76 bytes).
    Removing gd32f1x0_rtc.o(i.rtc_current_time_get), (100 bytes).
    Removing gd32f1x0_rtc.o(i.rtc_deinit), (128 bytes).
    Removing gd32f1x0_rtc.o(i.rtc_flag_clear), (16 bytes).
    Removing gd32f1x0_rtc.o(i.rtc_flag_get), (20 bytes).
    Removing gd32f1x0_rtc.o(i.rtc_hour_adjust), (36 bytes).
    Removing gd32f1x0_rtc.o(i.rtc_init), (196 bytes).
    Removing gd32f1x0_rtc.o(i.rtc_init_mode_enter), (68 bytes).
    Removing gd32f1x0_rtc.o(i.rtc_init_mode_exit), (20 bytes).
    Removing gd32f1x0_rtc.o(i.rtc_interrupt_disable), (60 bytes).
    Removing gd32f1x0_rtc.o(i.rtc_interrupt_enable), (60 bytes).
    Removing gd32f1x0_rtc.o(i.rtc_refclock_detection_disable), (56 bytes).
    Removing gd32f1x0_rtc.o(i.rtc_refclock_detection_enable), (56 bytes).
    Removing gd32f1x0_rtc.o(i.rtc_register_sync_wait), (96 bytes).
    Removing gd32f1x0_rtc.o(i.rtc_second_ajust), (108 bytes).
    Removing gd32f1x0_rtc.o(i.rtc_subsecond_get), (20 bytes).
    Removing gd32f1x0_rtc.o(i.rtc_tamper_disable), (16 bytes).
    Removing gd32f1x0_rtc.o(i.rtc_tamper_enable), (164 bytes).
    Removing gd32f1x0_rtc.o(i.rtc_timestamp_disable), (40 bytes).
    Removing gd32f1x0_rtc.o(i.rtc_timestamp_enable), (48 bytes).
    Removing gd32f1x0_rtc.o(i.rtc_timestamp_get), (60 bytes).
    Removing gd32f1x0_rtc.o(i.rtc_timestamp_subsecond_get), (12 bytes).
    Removing gd32f1x0_spi.o(.rev16_text), (4 bytes).
    Removing gd32f1x0_spi.o(.revsh_text), (4 bytes).
    Removing gd32f1x0_spi.o(i.i2s_disable), (10 bytes).
    Removing gd32f1x0_spi.o(i.i2s_enable), (10 bytes).
    Removing gd32f1x0_spi.o(i.i2s_init), (28 bytes).
    Removing gd32f1x0_spi.o(i.i2s_psc_config), (164 bytes).
    Removing gd32f1x0_spi.o(i.spi_bidirectional_transfer_config), (26 bytes).
    Removing gd32f1x0_spi.o(i.spi_crc_error_clear), (10 bytes).
    Removing gd32f1x0_spi.o(i.spi_crc_get), (16 bytes).
    Removing gd32f1x0_spi.o(i.spi_crc_next), (10 bytes).
    Removing gd32f1x0_spi.o(i.spi_crc_off), (10 bytes).
    Removing gd32f1x0_spi.o(i.spi_crc_on), (10 bytes).
    Removing gd32f1x0_spi.o(i.spi_crc_polynomial_get), (8 bytes).
    Removing gd32f1x0_spi.o(i.spi_crc_polynomial_set), (4 bytes).
    Removing gd32f1x0_spi.o(i.spi_disable), (10 bytes).
    Removing gd32f1x0_spi.o(i.spi_dma_disable), (22 bytes).
    Removing gd32f1x0_spi.o(i.spi_dma_enable), (22 bytes).
    Removing gd32f1x0_spi.o(i.spi_enable), (10 bytes).
    Removing gd32f1x0_spi.o(i.spi_i2s_data_frame_format_config), (16 bytes).
    Removing gd32f1x0_spi.o(i.spi_i2s_data_receive), (8 bytes).
    Removing gd32f1x0_spi.o(i.spi_i2s_data_transmit), (4 bytes).
    Removing gd32f1x0_spi.o(i.spi_i2s_deinit), (88 bytes).
    Removing gd32f1x0_spi.o(i.spi_i2s_flag_get), (16 bytes).
    Removing gd32f1x0_spi.o(i.spi_i2s_interrupt_disable), (48 bytes).
    Removing gd32f1x0_spi.o(i.spi_i2s_interrupt_enable), (48 bytes).
    Removing gd32f1x0_spi.o(i.spi_i2s_interrupt_flag_get), (100 bytes).
    Removing gd32f1x0_spi.o(i.spi_init), (50 bytes).
    Removing gd32f1x0_spi.o(i.spi_nss_internal_high), (10 bytes).
    Removing gd32f1x0_spi.o(i.spi_nss_internal_low), (10 bytes).
    Removing gd32f1x0_spi.o(i.spi_nss_output_disable), (10 bytes).
    Removing gd32f1x0_spi.o(i.spi_nss_output_enable), (10 bytes).
    Removing gd32f1x0_syscfg.o(.rev16_text), (4 bytes).
    Removing gd32f1x0_syscfg.o(.revsh_text), (4 bytes).
    Removing gd32f1x0_syscfg.o(i.syscfg_deinit), (20 bytes).
    Removing gd32f1x0_syscfg.o(i.syscfg_dma_remap_disable), (16 bytes).
    Removing gd32f1x0_syscfg.o(i.syscfg_dma_remap_enable), (16 bytes).
    Removing gd32f1x0_syscfg.o(i.syscfg_exti_line_config), (160 bytes).
    Removing gd32f1x0_syscfg.o(i.syscfg_flag_clear), (16 bytes).
    Removing gd32f1x0_syscfg.o(i.syscfg_flag_get), (24 bytes).
    Removing gd32f1x0_syscfg.o(i.syscfg_high_current_disable), (20 bytes).
    Removing gd32f1x0_syscfg.o(i.syscfg_high_current_enable), (20 bytes).
    Removing gd32f1x0_syscfg.o(i.syscfg_lock_config), (16 bytes).
    Removing gd32f1x0_timer.o(.rev16_text), (4 bytes).
    Removing gd32f1x0_timer.o(.revsh_text), (4 bytes).
    Removing gd32f1x0_timer.o(i.timer_auto_reload_shadow_disable), (10 bytes).
    Removing gd32f1x0_timer.o(i.timer_auto_reload_shadow_enable), (10 bytes).
    Removing gd32f1x0_timer.o(i.timer_automatic_output_disable), (8 bytes).
    Removing gd32f1x0_timer.o(i.timer_automatic_output_enable), (10 bytes).
    Removing gd32f1x0_timer.o(i.timer_autoreload_value_config), (4 bytes).
    Removing gd32f1x0_timer.o(i.timer_break_config), (30 bytes).
    Removing gd32f1x0_timer.o(i.timer_break_disable), (8 bytes).
    Removing gd32f1x0_timer.o(i.timer_break_enable), (10 bytes).
    Removing gd32f1x0_timer.o(i.timer_channel_capture_value_register_read), (42 bytes).
    Removing gd32f1x0_timer.o(i.timer_channel_complementary_output_polarity_config), (70 bytes).
    Removing gd32f1x0_timer.o(i.timer_channel_complementary_output_state_config), (70 bytes).
    Removing gd32f1x0_timer.o(i.timer_channel_control_shadow_config), (22 bytes).
    Removing gd32f1x0_timer.o(i.timer_channel_control_shadow_update_config), (26 bytes).
    Removing gd32f1x0_timer.o(i.timer_channel_dma_request_source_select), (26 bytes).
    Removing gd32f1x0_timer.o(i.timer_channel_input_capture_prescaler_config), (90 bytes).
    Removing gd32f1x0_timer.o(i.timer_channel_output_clear_config), (90 bytes).
    Removing gd32f1x0_timer.o(i.timer_channel_output_config), (460 bytes).
    Removing gd32f1x0_timer.o(i.timer_channel_output_fast_config), (90 bytes).
    Removing gd32f1x0_timer.o(i.timer_channel_output_mode_config), (90 bytes).
    Removing gd32f1x0_timer.o(i.timer_channel_output_polarity_config), (92 bytes).
    Removing gd32f1x0_timer.o(i.timer_channel_output_pulse_value_config), (38 bytes).
    Removing gd32f1x0_timer.o(i.timer_channel_output_shadow_config), (90 bytes).
    Removing gd32f1x0_timer.o(i.timer_channel_output_state_config), (92 bytes).
    Removing gd32f1x0_timer.o(i.timer_channel_remap_config), (6 bytes).
    Removing gd32f1x0_timer.o(i.timer_counter_alignment), (16 bytes).
    Removing gd32f1x0_timer.o(i.timer_counter_down_direction), (18 bytes).
    Removing gd32f1x0_timer.o(i.timer_counter_read), (8 bytes).
    Removing gd32f1x0_timer.o(i.timer_counter_up_direction), (14 bytes).
    Removing gd32f1x0_timer.o(i.timer_counter_value_config), (4 bytes).
    Removing gd32f1x0_timer.o(i.timer_deinit), (220 bytes).
    Removing gd32f1x0_timer.o(i.timer_disable), (10 bytes).
    Removing gd32f1x0_timer.o(i.timer_dma_disable), (8 bytes).
    Removing gd32f1x0_timer.o(i.timer_dma_enable), (8 bytes).
    Removing gd32f1x0_timer.o(i.timer_dma_transfer_config), (24 bytes).
    Removing gd32f1x0_timer.o(i.timer_enable), (10 bytes).
    Removing gd32f1x0_timer.o(i.timer_event_software_generate), (8 bytes).
    Removing gd32f1x0_timer.o(i.timer_external_clock_mode0_config), (56 bytes).
    Removing gd32f1x0_timer.o(i.timer_external_clock_mode1_config), (32 bytes).
    Removing gd32f1x0_timer.o(i.timer_external_clock_mode1_disable), (10 bytes).
    Removing gd32f1x0_timer.o(i.timer_external_trigger_as_external_clock_config), (164 bytes).
    Removing gd32f1x0_timer.o(i.timer_external_trigger_config), (30 bytes).
    Removing gd32f1x0_timer.o(i.timer_flag_clear), (8 bytes).
    Removing gd32f1x0_timer.o(i.timer_flag_get), (18 bytes).
    Removing gd32f1x0_timer.o(i.timer_hall_mode_config), (26 bytes).
    Removing gd32f1x0_timer.o(i.timer_init), (148 bytes).
    Removing gd32f1x0_timer.o(i.timer_input_capture_config), (326 bytes).
    Removing gd32f1x0_timer.o(i.timer_input_pwm_capture_config), (352 bytes).
    Removing gd32f1x0_timer.o(i.timer_input_trigger_source_select), (16 bytes).
    Removing gd32f1x0_timer.o(i.timer_internal_clock_config), (8 bytes).
    Removing gd32f1x0_timer.o(i.timer_internal_trigger_as_external_clock_config), (32 bytes).
    Removing gd32f1x0_timer.o(i.timer_interrupt_disable), (8 bytes).
    Removing gd32f1x0_timer.o(i.timer_interrupt_enable), (8 bytes).
    Removing gd32f1x0_timer.o(i.timer_interrupt_flag_clear), (8 bytes).
    Removing gd32f1x0_timer.o(i.timer_interrupt_flag_get), (32 bytes).
    Removing gd32f1x0_timer.o(i.timer_master_output_trigger_source_select), (16 bytes).
    Removing gd32f1x0_timer.o(i.timer_master_slave_mode_config), (26 bytes).
    Removing gd32f1x0_timer.o(i.timer_ocpre_clear_source_config), (26 bytes).
    Removing gd32f1x0_timer.o(i.timer_prescaler_config), (14 bytes).
    Removing gd32f1x0_timer.o(i.timer_prescaler_read), (10 bytes).
    Removing gd32f1x0_timer.o(i.timer_primary_output_config), (22 bytes).
    Removing gd32f1x0_timer.o(i.timer_quadrature_decoder_mode_config), (64 bytes).
    Removing gd32f1x0_timer.o(i.timer_repetition_value_config), (4 bytes).
    Removing gd32f1x0_timer.o(i.timer_single_pulse_mode_config), (26 bytes).
    Removing gd32f1x0_timer.o(i.timer_slave_mode_select), (16 bytes).
    Removing gd32f1x0_timer.o(i.timer_update_event_disable), (10 bytes).
    Removing gd32f1x0_timer.o(i.timer_update_event_enable), (10 bytes).
    Removing gd32f1x0_timer.o(i.timer_update_source_config), (26 bytes).
    Removing gd32f1x0_tsi.o(.rev16_text), (4 bytes).
    Removing gd32f1x0_tsi.o(.revsh_text), (4 bytes).
    Removing gd32f1x0_tsi.o(i.tsi_analog_off), (16 bytes).
    Removing gd32f1x0_tsi.o(i.tsi_analog_on), (16 bytes).
    Removing gd32f1x0_tsi.o(i.tsi_channel_pin_disable), (16 bytes).
    Removing gd32f1x0_tsi.o(i.tsi_channel_pin_enable), (16 bytes).
    Removing gd32f1x0_tsi.o(i.tsi_deinit), (20 bytes).
    Removing gd32f1x0_tsi.o(i.tsi_disable), (20 bytes).
    Removing gd32f1x0_tsi.o(i.tsi_enable), (20 bytes).
    Removing gd32f1x0_tsi.o(i.tsi_extend_charge_config), (100 bytes).
    Removing gd32f1x0_tsi.o(i.tsi_group0_cycle_get), (12 bytes).
    Removing gd32f1x0_tsi.o(i.tsi_group1_cycle_get), (12 bytes).
    Removing gd32f1x0_tsi.o(i.tsi_group2_cycle_get), (12 bytes).
    Removing gd32f1x0_tsi.o(i.tsi_group3_cycle_get), (12 bytes).
    Removing gd32f1x0_tsi.o(i.tsi_group4_cycle_get), (12 bytes).
    Removing gd32f1x0_tsi.o(i.tsi_group5_cycle_get), (12 bytes).
    Removing gd32f1x0_tsi.o(i.tsi_group_disable), (16 bytes).
    Removing gd32f1x0_tsi.o(i.tsi_group_enable), (16 bytes).
    Removing gd32f1x0_tsi.o(i.tsi_group_status_get), (24 bytes).
    Removing gd32f1x0_tsi.o(i.tsi_hardware_mode_config), (56 bytes).
    Removing gd32f1x0_tsi.o(i.tsi_hysteresis_off), (16 bytes).
    Removing gd32f1x0_tsi.o(i.tsi_hysteresis_on), (16 bytes).
    Removing gd32f1x0_tsi.o(i.tsi_init), (48 bytes).
    Removing gd32f1x0_tsi.o(i.tsi_interrupt_disable), (16 bytes).
    Removing gd32f1x0_tsi.o(i.tsi_interrupt_enable), (16 bytes).
    Removing gd32f1x0_tsi.o(i.tsi_interrupt_flag_clear), (16 bytes).
    Removing gd32f1x0_tsi.o(i.tsi_interrupt_flag_get), (24 bytes).
    Removing gd32f1x0_tsi.o(i.tsi_max_number_config), (32 bytes).
    Removing gd32f1x0_tsi.o(i.tsi_pin_mode_config), (44 bytes).
    Removing gd32f1x0_tsi.o(i.tsi_plus_config), (48 bytes).
    Removing gd32f1x0_tsi.o(i.tsi_sample_pin_disable), (28 bytes).
    Removing gd32f1x0_tsi.o(i.tsi_sample_pin_enable), (28 bytes).
    Removing gd32f1x0_tsi.o(i.tsi_sofeware_mode_config), (28 bytes).
    Removing gd32f1x0_tsi.o(i.tsi_software_start), (20 bytes).
    Removing gd32f1x0_tsi.o(i.tsi_software_stop), (20 bytes).
    Removing gd32f1x0_usart.o(.rev16_text), (4 bytes).
    Removing gd32f1x0_usart.o(.revsh_text), (4 bytes).
    Removing gd32f1x0_usart.o(i.usart_address_config), (32 bytes).
    Removing gd32f1x0_usart.o(i.usart_address_detection_mode_config), (28 bytes).
    Removing gd32f1x0_usart.o(i.usart_autobaud_detection_disable), (10 bytes).
    Removing gd32f1x0_usart.o(i.usart_autobaud_detection_enable), (10 bytes).
    Removing gd32f1x0_usart.o(i.usart_autobaud_detection_mode_config), (16 bytes).
    Removing gd32f1x0_usart.o(i.usart_block_length_config), (24 bytes).
    Removing gd32f1x0_usart.o(i.usart_clock_disable), (18 bytes).
    Removing gd32f1x0_usart.o(i.usart_clock_enable), (18 bytes).
    Removing gd32f1x0_usart.o(i.usart_command_enable), (8 bytes).
    Removing gd32f1x0_usart.o(i.usart_data_first_config), (28 bytes).
    Removing gd32f1x0_usart.o(i.usart_depolarity_config), (28 bytes).
    Removing gd32f1x0_usart.o(i.usart_disable), (10 bytes).
    Removing gd32f1x0_usart.o(i.usart_dma_receive_config), (16 bytes).
    Removing gd32f1x0_usart.o(i.usart_dma_transmit_config), (16 bytes).
    Removing gd32f1x0_usart.o(i.usart_driver_assertime_config), (32 bytes).
    Removing gd32f1x0_usart.o(i.usart_driver_deassertime_config), (32 bytes).
    Removing gd32f1x0_usart.o(i.usart_flag_clear), (18 bytes).
    Removing gd32f1x0_usart.o(i.usart_flag_get), (30 bytes).
    Removing gd32f1x0_usart.o(i.usart_guard_time_config), (32 bytes).
    Removing gd32f1x0_usart.o(i.usart_halfduplex_disable), (18 bytes).
    Removing gd32f1x0_usart.o(i.usart_halfduplex_enable), (18 bytes).
    Removing gd32f1x0_usart.o(i.usart_hardware_flow_cts_config), (24 bytes).
    Removing gd32f1x0_usart.o(i.usart_hardware_flow_rts_config), (24 bytes).
    Removing gd32f1x0_usart.o(i.usart_interrupt_flag_clear), (18 bytes).
    Removing gd32f1x0_usart.o(i.usart_invert_config), (110 bytes).
    Removing gd32f1x0_usart.o(i.usart_irda_lowpower_config), (20 bytes).
    Removing gd32f1x0_usart.o(i.usart_irda_mode_disable), (18 bytes).
    Removing gd32f1x0_usart.o(i.usart_irda_mode_enable), (18 bytes).
    Removing gd32f1x0_usart.o(i.usart_lin_break_dection_length_config), (20 bytes).
    Removing gd32f1x0_usart.o(i.usart_lin_mode_disable), (18 bytes).
    Removing gd32f1x0_usart.o(i.usart_lin_mode_enable), (18 bytes).
    Removing gd32f1x0_usart.o(i.usart_mute_mode_disable), (10 bytes).
    Removing gd32f1x0_usart.o(i.usart_mute_mode_enable), (10 bytes).
    Removing gd32f1x0_usart.o(i.usart_mute_mode_wakeup_config), (24 bytes).
    Removing gd32f1x0_usart.o(i.usart_overrun_disable), (18 bytes).
    Removing gd32f1x0_usart.o(i.usart_overrun_enable), (18 bytes).
    Removing gd32f1x0_usart.o(i.usart_oversample_config), (24 bytes).
    Removing gd32f1x0_usart.o(i.usart_parity_config), (24 bytes).
    Removing gd32f1x0_usart.o(i.usart_prescaler_config), (24 bytes).
    Removing gd32f1x0_usart.o(i.usart_receiver_timeout_config), (16 bytes).
    Removing gd32f1x0_usart.o(i.usart_receiver_timeout_disable), (10 bytes).
    Removing gd32f1x0_usart.o(i.usart_receiver_timeout_enable), (10 bytes).
    Removing gd32f1x0_usart.o(i.usart_reception_error_dma_disable), (18 bytes).
    Removing gd32f1x0_usart.o(i.usart_reception_error_dma_enable), (18 bytes).
    Removing gd32f1x0_usart.o(i.usart_rs485_driver_disable), (18 bytes).
    Removing gd32f1x0_usart.o(i.usart_rs485_driver_enable), (18 bytes).
    Removing gd32f1x0_usart.o(i.usart_sample_bit_config), (24 bytes).
    Removing gd32f1x0_usart.o(i.usart_smartcard_autoretry_config), (32 bytes).
    Removing gd32f1x0_usart.o(i.usart_smartcard_mode_disable), (18 bytes).
    Removing gd32f1x0_usart.o(i.usart_smartcard_mode_enable), (18 bytes).
    Removing gd32f1x0_usart.o(i.usart_smartcard_mode_nack_disable), (18 bytes).
    Removing gd32f1x0_usart.o(i.usart_smartcard_mode_nack_enable), (18 bytes).
    Removing gd32f1x0_usart.o(i.usart_stop_bit_set), (24 bytes).
    Removing gd32f1x0_usart.o(i.usart_synchronous_clock_config), (50 bytes).
    Removing gd32f1x0_usart.o(i.usart_wakeup_disable), (10 bytes).
    Removing gd32f1x0_usart.o(i.usart_wakeup_enable), (10 bytes).
    Removing gd32f1x0_usart.o(i.usart_wakeup_mode_config), (28 bytes).
    Removing gd32f1x0_usart.o(i.usart_word_length_set), (24 bytes).
    Removing gd32f1x0_wwdgt.o(.rev16_text), (4 bytes).
    Removing gd32f1x0_wwdgt.o(.revsh_text), (4 bytes).
    Removing gd32f1x0_wwdgt.o(i.wwdgt_config), (56 bytes).
    Removing gd32f1x0_wwdgt.o(i.wwdgt_counter_update), (28 bytes).
    Removing gd32f1x0_wwdgt.o(i.wwdgt_deinit), (20 bytes).
    Removing gd32f1x0_wwdgt.o(i.wwdgt_enable), (20 bytes).
    Removing gd32f1x0_wwdgt.o(i.wwdgt_flag_clear), (20 bytes).
    Removing gd32f1x0_wwdgt.o(i.wwdgt_flag_get), (24 bytes).
    Removing gd32f1x0_wwdgt.o(i.wwdgt_interrupt_enable), (20 bytes).
    Removing gd32f1x0_eval.o(.rev16_text), (4 bytes).
    Removing gd32f1x0_eval.o(.revsh_text), (4 bytes).
    Removing gd32f1x0_eval.o(i.gd_eval_key_init), (128 bytes).
    Removing gd32f1x0_eval.o(i.gd_eval_key_state_get), (32 bytes).
    Removing gd32f1x0_eval.o(i.gd_eval_led_init), (84 bytes).
    Removing gd32f1x0_eval.o(i.gd_eval_led_off), (24 bytes).
    Removing gd32f1x0_eval.o(i.gd_eval_led_on), (24 bytes).
    Removing gd32f1x0_eval.o(i.gd_eval_led_toggle), (36 bytes).
    Removing chip_uip_interrupt.o(i.Chip_UIP_InterruptInit), (44 bytes).
    Removing chip_uip_interrupt.o(i.Chip_UIP_InterruptNullHandler), (4 bytes).
    Removing chip_uip_interrupt.o(i.Chip_UIP_InterruptRegisterHandler), (32 bytes).
    Removing chip_uip_interrupt.o(i.Chip_UIP_InterruptRemoveHandler), (24 bytes).
    Removing chip_uip_interrupt.o(i.Chip_UIP_Kernel_Tick_ISR_Handler), (12 bytes).
    Removing chip_uip_interrupt.o(i.Chip_UIP_Kernel_Tick_ISR_Handler_Callback), (6 bytes).
    Removing hardware_init.o(.rev16_text), (4 bytes).
    Removing hardware_init.o(.revsh_text), (4 bytes).
    Removing hardware_init.o(i.Hardware_Init), (2 bytes).
    Removing hardware_init.o(.bss), (10 bytes).
    Removing uip_kernel_common.o(i.ShutdownOS), (2 bytes).
    Removing uip_kernel_common.o(i.uipAlarmInfoInit), (20 bytes).
    Removing uip_kernel_common.o(i.uipMsgInfoInit), (20 bytes).
    Removing uip_kernel_common.o(i.uipResInfoInit), (20 bytes).
    Removing uip_kernel_common.o(i.uipTaskInfoInit), (20 bytes).
    Removing uip_kernel_event.o(i.UIP_GetEvent), (116 bytes).
    Removing uip_kernel_message.o(i.UIP_CloseCOM), (4 bytes).
    Removing uip_kernel_message.o(i.UIP_GetMessageStatus), (88 bytes).
    Removing uip_kernel_message.o(i.UIP_ReadFlag), (24 bytes).
    Removing uip_kernel_message.o(i.UIP_ResetFlag), (40 bytes).
    Removing uip_kernel_message.o(i.UIP_StartCOM), (12 bytes).
    Removing uip_kernel_message.o(i.UIP_StopCOM), (56 bytes).
    Removing uip_kernel_task.o(i.UIP_ChainTask), (388 bytes).
    Removing uip_kernel_task.o(i.UIP_GetTaskID), (28 bytes).
    Removing uip_kernel_task.o(i.UIP_GetTaskState), (68 bytes).
    Removing uip_kernel_task.o(i.UIP_Schedule), (272 bytes).
    Removing uip_kernel_time.o(i.UIP_CancelAlarm), (72 bytes).
    Removing uip_kernel_time.o(i.UIP_GetAlarm), (112 bytes).
    Removing uip_kernel_time.o(i.UIP_GetAlarmBase), (48 bytes).
    Removing uip_kernel_time.o(i.UIP_SetAbsAlarm), (136 bytes).
    Removing uip_kernel_time.o(i.UIP_SetRelAlarm), (180 bytes).
    Removing uip_kernel_time.o(i.uipGeneralCounterHandler), (88 bytes).
    Removing uip_kernel_time.o(i.uipGetCtrCurrentValue), (80 bytes).

612 unused section(s) (total 22180 bytes) removed from the image.

==============================================================================

Image Symbol Table

    Local Symbols

    Symbol Name                              Value     Ov Type        Size  Object(Section)

    ../clib/../cmprslib/zerorunl2.c          0x00000000   Number         0  __dczerorl2.o ABSOLUTE
    ../clib/microlib/init/entry.s            0x00000000   Number         0  entry2.o ABSOLUTE
    ../clib/microlib/init/entry.s            0x00000000   Number         0  entry5.o ABSOLUTE
    ../clib/microlib/init/entry.s            0x00000000   Number         0  entry7a.o ABSOLUTE
    ../clib/microlib/init/entry.s            0x00000000   Number         0  entry10a.o ABSOLUTE
    ../clib/microlib/init/entry.s            0x00000000   Number         0  entry10b.o ABSOLUTE
    ../clib/microlib/init/entry.s            0x00000000   Number         0  entry11a.o ABSOLUTE
    ../clib/microlib/init/entry.s            0x00000000   Number         0  entry11b.o ABSOLUTE
    ../clib/microlib/init/entry.s            0x00000000   Number         0  entry7b.o ABSOLUTE
    ../clib/microlib/init/entry.s            0x00000000   Number         0  entry8a.o ABSOLUTE
    ../clib/microlib/init/entry.s            0x00000000   Number         0  entry.o ABSOLUTE
    ../clib/microlib/init/entry.s            0x00000000   Number         0  entry8b.o ABSOLUTE
    ../clib/microlib/init/entry.s            0x00000000   Number         0  entry9b.o ABSOLUTE
    ../clib/microlib/init/entry.s            0x00000000   Number         0  entry9a.o ABSOLUTE
    ..\..\Examples\USART\Transmitter&receiver_interrupt\gd32f1x0_it.c 0x00000000   Number         0  gd32f1x0_it.o ABSOLUTE
    ..\..\Examples\USART\Transmitter&receiver_interrupt\main.c 0x00000000   Number         0  main.o ABSOLUTE
    ..\..\Firmware\CMSIS\GD\GD32F1x0\Source\ARM\startup_gd32f1x0.s 0x00000000   Number         0  startup_gd32f1x0.o ABSOLUTE
    ..\..\Firmware\CMSIS\GD\GD32F1x0\Source\system_gd32f1x0.c 0x00000000   Number         0  system_gd32f1x0.o ABSOLUTE
    ..\..\Firmware\GD32F1x0_standard_peripheral\Source\gd32f1x0_adc.c 0x00000000   Number         0  gd32f1x0_adc.o ABSOLUTE
    ..\..\Firmware\GD32F1x0_standard_peripheral\Source\gd32f1x0_can.c 0x00000000   Number         0  gd32f1x0_can.o ABSOLUTE
    ..\..\Firmware\GD32F1x0_standard_peripheral\Source\gd32f1x0_cec.c 0x00000000   Number         0  gd32f1x0_cec.o ABSOLUTE
    ..\..\Firmware\GD32F1x0_standard_peripheral\Source\gd32f1x0_cmp.c 0x00000000   Number         0  gd32f1x0_cmp.o ABSOLUTE
    ..\..\Firmware\GD32F1x0_standard_peripheral\Source\gd32f1x0_crc.c 0x00000000   Number         0  gd32f1x0_crc.o ABSOLUTE
    ..\..\Firmware\GD32F1x0_standard_peripheral\Source\gd32f1x0_dac.c 0x00000000   Number         0  gd32f1x0_dac.o ABSOLUTE
    ..\..\Firmware\GD32F1x0_standard_peripheral\Source\gd32f1x0_dbg.c 0x00000000   Number         0  gd32f1x0_dbg.o ABSOLUTE
    ..\..\Firmware\GD32F1x0_standard_peripheral\Source\gd32f1x0_dma.c 0x00000000   Number         0  gd32f1x0_dma.o ABSOLUTE
    ..\..\Firmware\GD32F1x0_standard_peripheral\Source\gd32f1x0_exti.c 0x00000000   Number         0  gd32f1x0_exti.o ABSOLUTE
    ..\..\Firmware\GD32F1x0_standard_peripheral\Source\gd32f1x0_fmc.c 0x00000000   Number         0  gd32f1x0_fmc.o ABSOLUTE
    ..\..\Firmware\GD32F1x0_standard_peripheral\Source\gd32f1x0_fwdgt.c 0x00000000   Number         0  gd32f1x0_fwdgt.o ABSOLUTE
    ..\..\Firmware\GD32F1x0_standard_peripheral\Source\gd32f1x0_gpio.c 0x00000000   Number         0  gd32f1x0_gpio.o ABSOLUTE
    ..\..\Firmware\GD32F1x0_standard_peripheral\Source\gd32f1x0_i2c.c 0x00000000   Number         0  gd32f1x0_i2c.o ABSOLUTE
    ..\..\Firmware\GD32F1x0_standard_peripheral\Source\gd32f1x0_ivref.c 0x00000000   Number         0  gd32f1x0_ivref.o ABSOLUTE
    ..\..\Firmware\GD32F1x0_standard_peripheral\Source\gd32f1x0_misc.c 0x00000000   Number         0  gd32f1x0_misc.o ABSOLUTE
    ..\..\Firmware\GD32F1x0_standard_peripheral\Source\gd32f1x0_opa.c 0x00000000   Number         0  gd32f1x0_opa.o ABSOLUTE
    ..\..\Firmware\GD32F1x0_standard_peripheral\Source\gd32f1x0_pmu.c 0x00000000   Number         0  gd32f1x0_pmu.o ABSOLUTE
    ..\..\Firmware\GD32F1x0_standard_peripheral\Source\gd32f1x0_rcu.c 0x00000000   Number         0  gd32f1x0_rcu.o ABSOLUTE
    ..\..\Firmware\GD32F1x0_standard_peripheral\Source\gd32f1x0_rtc.c 0x00000000   Number         0  gd32f1x0_rtc.o ABSOLUTE
    ..\..\Firmware\GD32F1x0_standard_peripheral\Source\gd32f1x0_slcd.c 0x00000000   Number         0  gd32f1x0_slcd.o ABSOLUTE
    ..\..\Firmware\GD32F1x0_standard_peripheral\Source\gd32f1x0_spi.c 0x00000000   Number         0  gd32f1x0_spi.o ABSOLUTE
    ..\..\Firmware\GD32F1x0_standard_peripheral\Source\gd32f1x0_syscfg.c 0x00000000   Number         0  gd32f1x0_syscfg.o ABSOLUTE
    ..\..\Firmware\GD32F1x0_standard_peripheral\Source\gd32f1x0_timer.c 0x00000000   Number         0  gd32f1x0_timer.o ABSOLUTE
    ..\..\Firmware\GD32F1x0_standard_peripheral\Source\gd32f1x0_tsi.c 0x00000000   Number         0  gd32f1x0_tsi.o ABSOLUTE
    ..\..\Firmware\GD32F1x0_standard_peripheral\Source\gd32f1x0_usart.c 0x00000000   Number         0  gd32f1x0_usart.o ABSOLUTE
    ..\..\Firmware\GD32F1x0_standard_peripheral\Source\gd32f1x0_wwdgt.c 0x00000000   Number         0  gd32f1x0_wwdgt.o ABSOLUTE
    ..\..\Utilities\gd32f1x0_eval.c          0x00000000   Number         0  gd32f1x0_eval.o ABSOLUTE
    ..\..\app\app_cfg.c                      0x00000000   Number         0  app_cfg.o ABSOLUTE
    ..\..\app\app_int_cfg.c                  0x00000000   Number         0  app_int_cfg.o ABSOLUTE
    ..\..\app\demo.c                         0x00000000   Number         0  demo.o ABSOLUTE
    ..\..\app\hook.c                         0x00000000   Number         0  hook.o ABSOLUTE
    ..\..\bsp\chip_uip_interrupt.c           0x00000000   Number         0  chip_uip_interrupt.o ABSOLUTE
    ..\..\bsp\hardware_init.c                0x00000000   Number         0  hardware_init.o ABSOLUTE
    ..\..\uipkernel\uip_kernel_common.c      0x00000000   Number         0  uip_kernel_common.o ABSOLUTE
    ..\..\uipkernel\uip_kernel_event.c       0x00000000   Number         0  uip_kernel_event.o ABSOLUTE
    ..\..\uipkernel\uip_kernel_isr_cm.s      0x00000000   Number         0  uip_kernel_isr_cm.o ABSOLUTE
    ..\..\uipkernel\uip_kernel_isr_engine.c  0x00000000   Number         0  uip_kernel_isr_engine.o ABSOLUTE
    ..\..\uipkernel\uip_kernel_message.c     0x00000000   Number         0  uip_kernel_message.o ABSOLUTE
    ..\..\uipkernel\uip_kernel_resource.c    0x00000000   Number         0  uip_kernel_resource.o ABSOLUTE
    ..\..\uipkernel\uip_kernel_scheduler.c   0x00000000   Number         0  uip_kernel_scheduler.o ABSOLUTE
    ..\..\uipkernel\uip_kernel_task.c        0x00000000   Number         0  uip_kernel_task.o ABSOLUTE
    ..\..\uipkernel\uip_kernel_time.c        0x00000000   Number         0  uip_kernel_time.o ABSOLUTE
    ..\\..\\Examples\\USART\\Transmitter&receiver_interrupt\\gd32f1x0_it.c 0x00000000   Number         0  gd32f1x0_it.o ABSOLUTE
    ..\\..\\Examples\\USART\\Transmitter&receiver_interrupt\\main.c 0x00000000   Number         0  main.o ABSOLUTE
    ..\\..\\Firmware\\CMSIS\\GD\\GD32F1x0\\Source\\system_gd32f1x0.c 0x00000000   Number         0  system_gd32f1x0.o ABSOLUTE
    ..\\..\\Firmware\\GD32F1x0_standard_peripheral\\Source\\gd32f1x0_adc.c 0x00000000   Number         0  gd32f1x0_adc.o ABSOLUTE
    ..\\..\\Firmware\\GD32F1x0_standard_peripheral\\Source\\gd32f1x0_cec.c 0x00000000   Number         0  gd32f1x0_cec.o ABSOLUTE
    ..\\..\\Firmware\\GD32F1x0_standard_peripheral\\Source\\gd32f1x0_cmp.c 0x00000000   Number         0  gd32f1x0_cmp.o ABSOLUTE
    ..\\..\\Firmware\\GD32F1x0_standard_peripheral\\Source\\gd32f1x0_crc.c 0x00000000   Number         0  gd32f1x0_crc.o ABSOLUTE
    ..\\..\\Firmware\\GD32F1x0_standard_peripheral\\Source\\gd32f1x0_dac.c 0x00000000   Number         0  gd32f1x0_dac.o ABSOLUTE
    ..\\..\\Firmware\\GD32F1x0_standard_peripheral\\Source\\gd32f1x0_dbg.c 0x00000000   Number         0  gd32f1x0_dbg.o ABSOLUTE
    ..\\..\\Firmware\\GD32F1x0_standard_peripheral\\Source\\gd32f1x0_dma.c 0x00000000   Number         0  gd32f1x0_dma.o ABSOLUTE
    ..\\..\\Firmware\\GD32F1x0_standard_peripheral\\Source\\gd32f1x0_exti.c 0x00000000   Number         0  gd32f1x0_exti.o ABSOLUTE
    ..\\..\\Firmware\\GD32F1x0_standard_peripheral\\Source\\gd32f1x0_fmc.c 0x00000000   Number         0  gd32f1x0_fmc.o ABSOLUTE
    ..\\..\\Firmware\\GD32F1x0_standard_peripheral\\Source\\gd32f1x0_fwdgt.c 0x00000000   Number         0  gd32f1x0_fwdgt.o ABSOLUTE
    ..\\..\\Firmware\\GD32F1x0_standard_peripheral\\Source\\gd32f1x0_gpio.c 0x00000000   Number         0  gd32f1x0_gpio.o ABSOLUTE
    ..\\..\\Firmware\\GD32F1x0_standard_peripheral\\Source\\gd32f1x0_i2c.c 0x00000000   Number         0  gd32f1x0_i2c.o ABSOLUTE
    ..\\..\\Firmware\\GD32F1x0_standard_peripheral\\Source\\gd32f1x0_misc.c 0x00000000   Number         0  gd32f1x0_misc.o ABSOLUTE
    ..\\..\\Firmware\\GD32F1x0_standard_peripheral\\Source\\gd32f1x0_pmu.c 0x00000000   Number         0  gd32f1x0_pmu.o ABSOLUTE
    ..\\..\\Firmware\\GD32F1x0_standard_peripheral\\Source\\gd32f1x0_rcu.c 0x00000000   Number         0  gd32f1x0_rcu.o ABSOLUTE
    ..\\..\\Firmware\\GD32F1x0_standard_peripheral\\Source\\gd32f1x0_rtc.c 0x00000000   Number         0  gd32f1x0_rtc.o ABSOLUTE
    ..\\..\\Firmware\\GD32F1x0_standard_peripheral\\Source\\gd32f1x0_spi.c 0x00000000   Number         0  gd32f1x0_spi.o ABSOLUTE
    ..\\..\\Firmware\\GD32F1x0_standard_peripheral\\Source\\gd32f1x0_syscfg.c 0x00000000   Number         0  gd32f1x0_syscfg.o ABSOLUTE
    ..\\..\\Firmware\\GD32F1x0_standard_peripheral\\Source\\gd32f1x0_timer.c 0x00000000   Number         0  gd32f1x0_timer.o ABSOLUTE
    ..\\..\\Firmware\\GD32F1x0_standard_peripheral\\Source\\gd32f1x0_tsi.c 0x00000000   Number         0  gd32f1x0_tsi.o ABSOLUTE
    ..\\..\\Firmware\\GD32F1x0_standard_peripheral\\Source\\gd32f1x0_usart.c 0x00000000   Number         0  gd32f1x0_usart.o ABSOLUTE
    ..\\..\\Firmware\\GD32F1x0_standard_peripheral\\Source\\gd32f1x0_wwdgt.c 0x00000000   Number         0  gd32f1x0_wwdgt.o ABSOLUTE
    ..\\..\\Utilities\\gd32f1x0_eval.c       0x00000000   Number         0  gd32f1x0_eval.o ABSOLUTE
    ..\\..\\app\\app_int_cfg.c               0x00000000   Number         0  app_int_cfg.o ABSOLUTE
    ..\\..\\app\\demo.c                      0x00000000   Number         0  demo.o ABSOLUTE
    ..\\..\\bsp\\hardware_init.c             0x00000000   Number         0  hardware_init.o ABSOLUTE
    dc.s                                     0x00000000   Number         0  dc.o ABSOLUTE
    handlers.s                               0x00000000   Number         0  handlers.o ABSOLUTE
    init.s                                   0x00000000   Number         0  init.o ABSOLUTE
    RESET                                    0x08000000   Section      360  startup_gd32f1x0.o(RESET)
    .ARM.Collect$$$$00000000                 0x08000168   Section        0  entry.o(.ARM.Collect$$$$00000000)
    .ARM.Collect$$$$00000001                 0x08000168   Section        4  entry2.o(.ARM.Collect$$$$00000001)
    .ARM.Collect$$$$00000004                 0x0800016c   Section        4  entry5.o(.ARM.Collect$$$$00000004)
    .ARM.Collect$$$$00000008                 0x08000170   Section        0  entry7b.o(.ARM.Collect$$$$00000008)
    .ARM.Collect$$$$0000000A                 0x08000170   Section        0  entry8b.o(.ARM.Collect$$$$0000000A)
    .ARM.Collect$$$$0000000B                 0x08000170   Section        8  entry9a.o(.ARM.Collect$$$$0000000B)
    .ARM.Collect$$$$0000000D                 0x08000178   Section        0  entry10a.o(.ARM.Collect$$$$0000000D)
    .ARM.Collect$$$$0000000F                 0x08000178   Section        0  entry11a.o(.ARM.Collect$$$$0000000F)
    .ARM.Collect$$$$00002712                 0x08000178   Section        4  entry2.o(.ARM.Collect$$$$00002712)
    __lit__00000000                          0x08000178   Data           4  entry2.o(.ARM.Collect$$$$00002712)
    .text                                    0x0800017c   Section       36  startup_gd32f1x0.o(.text)
    .text                                    0x080001a0   Section       36  init.o(.text)
    .text                                    0x080001c4   Section        0  __dczerorl2.o(.text)
    CODE                                     0x0800021c   Section       72  uip_kernel_isr_cm.o(CODE)
    i.ADC_CMP_IRQHandler                     0x08000264   Section        0  chip_uip_interrupt.o(i.ADC_CMP_IRQHandler)
    i.AppIdleTask                            0x08000278   Section        0  demo.o(i.AppIdleTask)
    i.BusFault_Handler                       0x080002a6   Section        0  gd32f1x0_it.o(i.BusFault_Handler)
    i.CAN0_RX0_IRQHandler                    0x080002ac   Section        0  chip_uip_interrupt.o(i.CAN0_RX0_IRQHandler)
    i.CAN0_RX1_IRQHandler                    0x080002c0   Section        0  chip_uip_interrupt.o(i.CAN0_RX1_IRQHandler)
    i.CAN0_SCE_IRQHandler                    0x080002d4   Section        0  chip_uip_interrupt.o(i.CAN0_SCE_IRQHandler)
    i.CAN0_TX_IRQHandler                     0x080002e8   Section        0  chip_uip_interrupt.o(i.CAN0_TX_IRQHandler)
    i.CAN1_RX0_IRQHandler                    0x080002fc   Section        0  chip_uip_interrupt.o(i.CAN1_RX0_IRQHandler)
    i.CAN1_RX1_IRQHandler                    0x08000310   Section        0  chip_uip_interrupt.o(i.CAN1_RX1_IRQHandler)
    i.CAN1_SCE_IRQHandler                    0x08000324   Section        0  chip_uip_interrupt.o(i.CAN1_SCE_IRQHandler)
    i.CAN1_TX_IRQHandler                     0x08000338   Section        0  chip_uip_interrupt.o(i.CAN1_TX_IRQHandler)
    i.CEC_IRQHandler                         0x0800034c   Section        0  chip_uip_interrupt.o(i.CEC_IRQHandler)
    i.Chip_GD32F1X0_USART0_ISR_Handler_Callback 0x08000360   Section        0  app_int_cfg.o(i.Chip_GD32F1X0_USART0_ISR_Handler_Callback)
    i.DMA_Channel0_IRQHandler                0x08000368   Section        0  chip_uip_interrupt.o(i.DMA_Channel0_IRQHandler)
    i.DMA_Channel1_2_IRQHandler              0x0800037c   Section        0  chip_uip_interrupt.o(i.DMA_Channel1_2_IRQHandler)
    i.DMA_Channel3_4_IRQHandler              0x08000390   Section        0  chip_uip_interrupt.o(i.DMA_Channel3_4_IRQHandler)
    i.DMA_Channel5_6_IRQHandler              0x080003a4   Section        0  chip_uip_interrupt.o(i.DMA_Channel5_6_IRQHandler)
    i.DebugMon_Handler                       0x080003b8   Section        0  gd32f1x0_it.o(i.DebugMon_Handler)
    i.EXTI0_1_IRQHandler                     0x080003bc   Section        0  chip_uip_interrupt.o(i.EXTI0_1_IRQHandler)
    i.EXTI2_3_IRQHandler                     0x080003d0   Section        0  chip_uip_interrupt.o(i.EXTI2_3_IRQHandler)
    i.EXTI4_15_IRQHandler                    0x080003e4   Section        0  chip_uip_interrupt.o(i.EXTI4_15_IRQHandler)
    i.FMC_IRQHandler                         0x080003f8   Section        0  chip_uip_interrupt.o(i.FMC_IRQHandler)
    i.HardFault_Handler                      0x0800040c   Section        0  gd32f1x0_it.o(i.HardFault_Handler)
    i.I2C0_ER_IRQHandler                     0x08000410   Section        0  chip_uip_interrupt.o(i.I2C0_ER_IRQHandler)
    i.I2C0_EV_IRQHandler                     0x08000424   Section        0  chip_uip_interrupt.o(i.I2C0_EV_IRQHandler)
    i.I2C1_ER_IRQHandler                     0x08000438   Section        0  chip_uip_interrupt.o(i.I2C1_ER_IRQHandler)
    i.I2C1_EV_IRQHandler                     0x0800044c   Section        0  chip_uip_interrupt.o(i.I2C1_EV_IRQHandler)
    i.I2C2_ER_IRQHandler                     0x08000460   Section        0  chip_uip_interrupt.o(i.I2C2_ER_IRQHandler)
    i.I2C2_EV_IRQHandler                     0x08000474   Section        0  chip_uip_interrupt.o(i.I2C2_EV_IRQHandler)
    i.InterruptHandler                       0x08000488   Section        0  chip_uip_interrupt.o(i.InterruptHandler)
    i.Kernel_System_Tick_Init                0x080004e4   Section        0  hardware_init.o(i.Kernel_System_Tick_Init)
    i.LVD_IRQHandler                         0x08000544   Section        0  chip_uip_interrupt.o(i.LVD_IRQHandler)
    i.MemManage_Handler                      0x08000558   Section        0  gd32f1x0_it.o(i.MemManage_Handler)
    i.NMI_Handler                            0x0800055c   Section        0  gd32f1x0_it.o(i.NMI_Handler)
    i.RCU_IRQHandler                         0x08000560   Section        0  chip_uip_interrupt.o(i.RCU_IRQHandler)
    i.RTC_IRQHandler                         0x08000574   Section        0  chip_uip_interrupt.o(i.RTC_IRQHandler)
    i.SLCD_IRQHandler                        0x08000588   Section        0  chip_uip_interrupt.o(i.SLCD_IRQHandler)
    i.SPI0_IRQHandler                        0x0800059c   Section        0  chip_uip_interrupt.o(i.SPI0_IRQHandler)
    i.SPI1_IRQHandler                        0x080005b0   Section        0  chip_uip_interrupt.o(i.SPI1_IRQHandler)
    i.SPI2_IRQHandler                        0x080005c4   Section        0  chip_uip_interrupt.o(i.SPI2_IRQHandler)
    i.SVC_Handler                            0x080005d8   Section        0  gd32f1x0_it.o(i.SVC_Handler)
    i.StartOS                                0x080005dc   Section        0  uip_kernel_common.o(i.StartOS)
    i.SystemInit                             0x0800060c   Section        0  system_gd32f1x0.o(i.SystemInit)
    i.TASK_0                                 0x08000694   Section        0  demo.o(i.TASK_0)
    i.TASK_1                                 0x080006d0   Section        0  demo.o(i.TASK_1)
    i.TASK_2                                 0x080006f4   Section        0  demo.o(i.TASK_2)
    i.TASK_3                                 0x08000714   Section        0  demo.o(i.TASK_3)
    i.TASK_4                                 0x08000730   Section        0  demo.o(i.TASK_4)
    i.TIMER0_BRK_UP_TRG_COM_IRQHandler       0x08000750   Section        0  chip_uip_interrupt.o(i.TIMER0_BRK_UP_TRG_COM_IRQHandler)
    i.TIMER0_Channel_IRQHandler              0x08000764   Section        0  chip_uip_interrupt.o(i.TIMER0_Channel_IRQHandler)
    i.TIMER13_IRQHandler                     0x08000778   Section        0  chip_uip_interrupt.o(i.TIMER13_IRQHandler)
    i.TIMER14_IRQHandler                     0x0800078c   Section        0  chip_uip_interrupt.o(i.TIMER14_IRQHandler)
    i.TIMER15_IRQHandler                     0x080007a0   Section        0  chip_uip_interrupt.o(i.TIMER15_IRQHandler)
    i.TIMER16_IRQHandler                     0x080007b4   Section        0  chip_uip_interrupt.o(i.TIMER16_IRQHandler)
    i.TIMER1_IRQHandler                      0x080007c8   Section        0  chip_uip_interrupt.o(i.TIMER1_IRQHandler)
    i.TIMER2_IRQHandler                      0x080007dc   Section        0  chip_uip_interrupt.o(i.TIMER2_IRQHandler)
    i.TIMER5_DAC_IRQHandler                  0x080007f0   Section        0  chip_uip_interrupt.o(i.TIMER5_DAC_IRQHandler)
    i.TSI_IRQHandler                         0x08000804   Section        0  chip_uip_interrupt.o(i.TSI_IRQHandler)
    i.UIP_ActivateTask                       0x08000818   Section        0  uip_kernel_task.o(i.UIP_ActivateTask)
    i.UIP_ClearEvent                         0x0800091c   Section        0  uip_kernel_event.o(i.UIP_ClearEvent)
    i.UIP_GetResource                        0x0800096c   Section        0  uip_kernel_resource.o(i.UIP_GetResource)
    i.UIP_ReceiveMessage                     0x08000a30   Section        0  uip_kernel_message.o(i.UIP_ReceiveMessage)
    i.UIP_ReleaseResource                    0x08000b08   Section        0  uip_kernel_resource.o(i.UIP_ReleaseResource)
    i.UIP_SendMessage                        0x08000c34   Section        0  uip_kernel_message.o(i.UIP_SendMessage)
    i.UIP_SetEvent                           0x08000d44   Section        0  uip_kernel_event.o(i.UIP_SetEvent)
    i.UIP_TerminateTask                      0x08000e7c   Section        0  uip_kernel_task.o(i.UIP_TerminateTask)
    i.UIP_WaitEvent                          0x08000f88   Section        0  uip_kernel_event.o(i.UIP_WaitEvent)
    i.USART0_IRQHandler                      0x08001010   Section        0  chip_uip_interrupt.o(i.USART0_IRQHandler)
    i.USART0_IRQHandler_Process              0x08001024   Section        0  gd32f1x0_it.o(i.USART0_IRQHandler_Process)
    i.USART1_IRQHandler                      0x080010c0   Section        0  chip_uip_interrupt.o(i.USART1_IRQHandler)
    i.USBDWakeUp_IRQHandler                  0x080010d4   Section        0  chip_uip_interrupt.o(i.USBDWakeUp_IRQHandler)
    i.USBD_HP_IRQHandler                     0x080010e8   Section        0  chip_uip_interrupt.o(i.USBD_HP_IRQHandler)
    i.USBD_LP_IRQHandler                     0x080010fc   Section        0  chip_uip_interrupt.o(i.USBD_LP_IRQHandler)
    i.UsageFault_Handler                     0x08001110   Section        0  gd32f1x0_it.o(i.UsageFault_Handler)
    i.WWDGT_IRQHandler                       0x08001114   Section        0  chip_uip_interrupt.o(i.WWDGT_IRQHandler)
    i.__scatterload_copy                     0x08001128   Section       14  handlers.o(i.__scatterload_copy)
    i.__scatterload_null                     0x08001136   Section        2  handlers.o(i.__scatterload_null)
    i.__scatterload_zeroinit                 0x08001138   Section       14  handlers.o(i.__scatterload_zeroinit)
    i.gd_eval_com_init                       0x08001148   Section        0  gd32f1x0_eval.o(i.gd_eval_com_init)
    i.gpio_af_set                            0x08001208   Section        0  gd32f1x0_gpio.o(i.gpio_af_set)
    i.gpio_mode_set                          0x08001266   Section        0  gd32f1x0_gpio.o(i.gpio_mode_set)
    i.gpio_output_options_set                0x080012b4   Section        0  gd32f1x0_gpio.o(i.gpio_output_options_set)
    i.main                                   0x080012f6   Section        0  main.o(i.main)
    i.nvic_irq_enable                        0x08001300   Section        0  gd32f1x0_misc.o(i.nvic_irq_enable)
    i.rcu_clock_freq_get                     0x080013a4   Section        0  gd32f1x0_rcu.o(i.rcu_clock_freq_get)
    i.rcu_periph_clock_enable                0x0800164c   Section        0  gd32f1x0_rcu.o(i.rcu_periph_clock_enable)
    i.rcu_periph_reset_disable               0x0800166c   Section        0  gd32f1x0_rcu.o(i.rcu_periph_reset_disable)
    i.rcu_periph_reset_enable                0x0800168c   Section        0  gd32f1x0_rcu.o(i.rcu_periph_reset_enable)
    i.system_clock_72m_hxtal                 0x080016ac   Section        0  system_gd32f1x0.o(i.system_clock_72m_hxtal)
    system_clock_72m_hxtal                   0x080016ad   Thumb Code   154  system_gd32f1x0.o(i.system_clock_72m_hxtal)
    i.system_clock_config                    0x08001750   Section        0  system_gd32f1x0.o(i.system_clock_config)
    system_clock_config                      0x08001751   Thumb Code     8  system_gd32f1x0.o(i.system_clock_config)
    i.uipAlarmHandler                        0x08001758   Section        0  uip_kernel_time.o(i.uipAlarmHandler)
    i.uipAlarmInitialize                     0x080017d4   Section        0  uip_kernel_common.o(i.uipAlarmInitialize)
    i.uipAppInitialize                       0x08001800   Section        0  demo.o(i.uipAppInitialize)
    i.uipClearPrioGrpAndArrayBit             0x08001860   Section        0  uip_kernel_scheduler.o(i.uipClearPrioGrpAndArrayBit)
    i.uipEnterKernel                         0x080018c8   Section        0  demo.o(i.uipEnterKernel)
    i.uipGetNextPriority                     0x080018e4   Section        0  uip_kernel_scheduler.o(i.uipGetNextPriority)
    i.uipGetNextTask                         0x0800193c   Section        0  uip_kernel_scheduler.o(i.uipGetNextTask)
    i.uipInterruptHandlingCallback           0x080019d0   Section        0  chip_uip_interrupt.o(i.uipInterruptHandlingCallback)
    i.uipInterruptServiceEngine              0x080019e8   Section        0  uip_kernel_isr_engine.o(i.uipInterruptServiceEngine)
    i.uipKernelInitialize                    0x08001b04   Section        0  uip_kernel_common.o(i.uipKernelInitialize)
    i.uipMsgInitialize                       0x08001c2c   Section        0  uip_kernel_common.o(i.uipMsgInitialize)
    i.uipPreContexSwitch                     0x08001c74   Section        0  uip_kernel_scheduler.o(i.uipPreContexSwitch)
    i.uipResInitialize                       0x08001cc8   Section        0  uip_kernel_common.o(i.uipResInitialize)
    i.uipResetPrioGrpAndArrayBit             0x08001d1c   Section        0  uip_kernel_scheduler.o(i.uipResetPrioGrpAndArrayBit)
    i.uipSystemCounterHandler                0x08001d6c   Section        0  uip_kernel_time.o(i.uipSystemCounterHandler)
    i.uipTaskInitialize                      0x08001dec   Section        0  uip_kernel_common.o(i.uipTaskInitialize)
    i.uipTaskStackInit                       0x08001ef8   Section        0  uip_kernel_common.o(i.uipTaskStackInit)
    i.usart_baudrate_set                     0x08001f44   Section        0  gd32f1x0_usart.o(i.usart_baudrate_set)
    i.usart_data_receive                     0x08001fc0   Section        0  gd32f1x0_usart.o(i.usart_data_receive)
    i.usart_data_transmit                    0x08001fca   Section        0  gd32f1x0_usart.o(i.usart_data_transmit)
    i.usart_deinit                           0x08001fd4   Section        0  gd32f1x0_usart.o(i.usart_deinit)
    i.usart_enable                           0x08002014   Section        0  gd32f1x0_usart.o(i.usart_enable)
    i.usart_interrupt_disable                0x0800201e   Section        0  gd32f1x0_usart.o(i.usart_interrupt_disable)
    i.usart_interrupt_enable                 0x08002038   Section        0  gd32f1x0_usart.o(i.usart_interrupt_enable)
    i.usart_interrupt_flag_get               0x08002052   Section        0  gd32f1x0_usart.o(i.usart_interrupt_flag_get)
    i.usart_receive_config                   0x0800208a   Section        0  gd32f1x0_usart.o(i.usart_receive_config)
    i.usart_transmit_config                  0x0800209a   Section        0  gd32f1x0_usart.o(i.usart_transmit_config)
    .data                                    0x20000000   Section       30  main.o(.data)
    .data                                    0x20000020   Section      453  app_cfg.o(.data)
    .data                                    0x200001e8   Section       37  app_int_cfg.o(.data)
    .data                                    0x20000210   Section        4  system_gd32f1x0.o(.data)
    .data                                    0x20000214   Section      105  gd32f1x0_eval.o(.data)
    GPIO_PORT                                0x20000214   Data          16  gd32f1x0_eval.o(.data)
    GPIO_PIN                                 0x20000224   Data          16  gd32f1x0_eval.o(.data)
    COM_CLK                                  0x20000234   Data           2  gd32f1x0_eval.o(.data)
    COM_TX_PIN                               0x20000238   Data           4  gd32f1x0_eval.o(.data)
    COM_RX_PIN                               0x2000023c   Data           4  gd32f1x0_eval.o(.data)
    GPIO_CLK                                 0x20000240   Data           8  gd32f1x0_eval.o(.data)
    KEY_PORT                                 0x20000248   Data          12  gd32f1x0_eval.o(.data)
    KEY_PIN                                  0x20000254   Data          12  gd32f1x0_eval.o(.data)
    KEY_CLK                                  0x20000260   Data           6  gd32f1x0_eval.o(.data)
    KEY_EXTI_LINE                            0x20000268   Data          12  gd32f1x0_eval.o(.data)
    KEY_PORT_SOURCE                          0x20000274   Data           3  gd32f1x0_eval.o(.data)
    KEY_PIN_SOURCE                           0x20000277   Data           3  gd32f1x0_eval.o(.data)
    KEY_IRQn                                 0x2000027a   Data           3  gd32f1x0_eval.o(.data)
    .data                                    0x20000280   Section       48  uip_kernel_common.o(.data)
    .data                                    0x200002b0   Section      290  uip_kernel_scheduler.o(.data)
    .bss                                     0x200003d4   Section       32  main.o(.bss)
    .bss                                     0x200003f4   Section     1600  app_cfg.o(.bss)
    .bss                                     0x20000a34   Section       32  demo.o(.bss)
    .bss                                     0x20000a54   Section     1304  uip_kernel_common.o(.bss)
    .bss                                     0x20000f6c   Section       32  uip_kernel_scheduler.o(.bss)
    STACK                                    0x20000f90   Section      512  startup_gd32f1x0.o(STACK)

    Global Symbols

    Symbol Name                              Value     Ov Type        Size  Object(Section)

    BuildAttributes$$THM_ISAv4$P$D$K$B$S$PE$A:L22UL41UL21$X:L11$S22US41US21$IEEE1$IW$USESV6$~STKCKD$USESV7$~SHL$OSPACE$EBA8$MICROLIB$REQ8$PRES8$EABIv2 0x00000000   Number         0  anon$$obj.o ABSOLUTE
    __ARM_use_no_argv                        0x00000000   Number         0  main.o ABSOLUTE
    __cpp_initialize__aeabi_                  - Undefined Weak Reference
    __cxa_finalize                            - Undefined Weak Reference
    _clock_init                               - Undefined Weak Reference
    _microlib_exit                            - Undefined Weak Reference
    __Vectors_Size                           0x00000168   Number         0  startup_gd32f1x0.o ABSOLUTE
    __Vectors                                0x08000000   Data           4  startup_gd32f1x0.o(RESET)
    __Vectors_End                            0x08000168   Data           0  startup_gd32f1x0.o(RESET)
    __main                                   0x08000169   Thumb Code     0  entry.o(.ARM.Collect$$$$00000000)
    _main_stk                                0x08000169   Thumb Code     0  entry2.o(.ARM.Collect$$$$00000001)
    _main_scatterload                        0x0800016d   Thumb Code     0  entry5.o(.ARM.Collect$$$$00000004)
    __main_after_scatterload                 0x08000171   Thumb Code     0  entry5.o(.ARM.Collect$$$$00000004)
    _main_clock                              0x08000171   Thumb Code     0  entry7b.o(.ARM.Collect$$$$00000008)
    _main_cpp_init                           0x08000171   Thumb Code     0  entry8b.o(.ARM.Collect$$$$0000000A)
    _main_init                               0x08000171   Thumb Code     0  entry9a.o(.ARM.Collect$$$$0000000B)
    __rt_final_cpp                           0x08000179   Thumb Code     0  entry10a.o(.ARM.Collect$$$$0000000D)
    __rt_final_exit                          0x08000179   Thumb Code     0  entry11a.o(.ARM.Collect$$$$0000000F)
    Reset_Handler                            0x0800017d   Thumb Code     8  startup_gd32f1x0.o(.text)
    PendSV_Handler                           0x08000193   Thumb Code     2  startup_gd32f1x0.o(.text)
    SysTick_Handler                          0x08000195   Thumb Code     2  startup_gd32f1x0.o(.text)
    __scatterload                            0x080001a1   Thumb Code    28  init.o(.text)
    __scatterload_rt2                        0x080001a1   Thumb Code     0  init.o(.text)
    __decompress                             0x080001c5   Thumb Code     0  __dczerorl2.o(.text)
    __decompress1                            0x080001c5   Thumb Code    86  __dczerorl2.o(.text)
    uipDisableAllInterrupts                  0x0800021d   Thumb Code     0  uip_kernel_isr_cm.o(CODE)
    uipIntMaskStateRestore                   0x08000225   Thumb Code     0  uip_kernel_isr_cm.o(CODE)
    uipPendSVHandler                         0x0800022b   Thumb Code     0  uip_kernel_isr_cm.o(CODE)
    ADC_CMP_IRQHandler                       0x08000265   Thumb Code    14  chip_uip_interrupt.o(i.ADC_CMP_IRQHandler)
    AppIdleTask                              0x08000279   Thumb Code    46  demo.o(i.AppIdleTask)
    BusFault_Handler                         0x080002a7   Thumb Code     4  gd32f1x0_it.o(i.BusFault_Handler)
    CAN0_RX0_IRQHandler                      0x080002ad   Thumb Code    14  chip_uip_interrupt.o(i.CAN0_RX0_IRQHandler)
    CAN0_RX1_IRQHandler                      0x080002c1   Thumb Code    14  chip_uip_interrupt.o(i.CAN0_RX1_IRQHandler)
    CAN0_SCE_IRQHandler                      0x080002d5   Thumb Code    14  chip_uip_interrupt.o(i.CAN0_SCE_IRQHandler)
    CAN0_TX_IRQHandler                       0x080002e9   Thumb Code    14  chip_uip_interrupt.o(i.CAN0_TX_IRQHandler)
    CAN1_RX0_IRQHandler                      0x080002fd   Thumb Code    14  chip_uip_interrupt.o(i.CAN1_RX0_IRQHandler)
    CAN1_RX1_IRQHandler                      0x08000311   Thumb Code    14  chip_uip_interrupt.o(i.CAN1_RX1_IRQHandler)
    CAN1_SCE_IRQHandler                      0x08000325   Thumb Code    14  chip_uip_interrupt.o(i.CAN1_SCE_IRQHandler)
    CAN1_TX_IRQHandler                       0x08000339   Thumb Code    14  chip_uip_interrupt.o(i.CAN1_TX_IRQHandler)
    CEC_IRQHandler                           0x0800034d   Thumb Code    14  chip_uip_interrupt.o(i.CEC_IRQHandler)
    Chip_GD32F1X0_USART0_ISR_Handler_Callback 0x08000361   Thumb Code     6  app_int_cfg.o(i.Chip_GD32F1X0_USART0_ISR_Handler_Callback)
    DMA_Channel0_IRQHandler                  0x08000369   Thumb Code    14  chip_uip_interrupt.o(i.DMA_Channel0_IRQHandler)
    DMA_Channel1_2_IRQHandler                0x0800037d   Thumb Code    14  chip_uip_interrupt.o(i.DMA_Channel1_2_IRQHandler)
    DMA_Channel3_4_IRQHandler                0x08000391   Thumb Code    14  chip_uip_interrupt.o(i.DMA_Channel3_4_IRQHandler)
    DMA_Channel5_6_IRQHandler                0x080003a5   Thumb Code    14  chip_uip_interrupt.o(i.DMA_Channel5_6_IRQHandler)
    DebugMon_Handler                         0x080003b9   Thumb Code     2  gd32f1x0_it.o(i.DebugMon_Handler)
    EXTI0_1_IRQHandler                       0x080003bd   Thumb Code    14  chip_uip_interrupt.o(i.EXTI0_1_IRQHandler)
    EXTI2_3_IRQHandler                       0x080003d1   Thumb Code    14  chip_uip_interrupt.o(i.EXTI2_3_IRQHandler)
    EXTI4_15_IRQHandler                      0x080003e5   Thumb Code    14  chip_uip_interrupt.o(i.EXTI4_15_IRQHandler)
    FMC_IRQHandler                           0x080003f9   Thumb Code    14  chip_uip_interrupt.o(i.FMC_IRQHandler)
    HardFault_Handler                        0x0800040d   Thumb Code     4  gd32f1x0_it.o(i.HardFault_Handler)
    I2C0_ER_IRQHandler                       0x08000411   Thumb Code    14  chip_uip_interrupt.o(i.I2C0_ER_IRQHandler)
    I2C0_EV_IRQHandler                       0x08000425   Thumb Code    14  chip_uip_interrupt.o(i.I2C0_EV_IRQHandler)
    I2C1_ER_IRQHandler                       0x08000439   Thumb Code    14  chip_uip_interrupt.o(i.I2C1_ER_IRQHandler)
    I2C1_EV_IRQHandler                       0x0800044d   Thumb Code    14  chip_uip_interrupt.o(i.I2C1_EV_IRQHandler)
    I2C2_ER_IRQHandler                       0x08000461   Thumb Code    14  chip_uip_interrupt.o(i.I2C2_ER_IRQHandler)
    I2C2_EV_IRQHandler                       0x08000475   Thumb Code    14  chip_uip_interrupt.o(i.I2C2_EV_IRQHandler)
    InterruptHandler                         0x08000489   Thumb Code    78  chip_uip_interrupt.o(i.InterruptHandler)
    Kernel_System_Tick_Init                  0x080004e5   Thumb Code    82  hardware_init.o(i.Kernel_System_Tick_Init)
    LVD_IRQHandler                           0x08000545   Thumb Code    14  chip_uip_interrupt.o(i.LVD_IRQHandler)
    MemManage_Handler                        0x08000559   Thumb Code     4  gd32f1x0_it.o(i.MemManage_Handler)
    NMI_Handler                              0x0800055d   Thumb Code     2  gd32f1x0_it.o(i.NMI_Handler)
    RCU_IRQHandler                           0x08000561   Thumb Code    14  chip_uip_interrupt.o(i.RCU_IRQHandler)
    RTC_IRQHandler                           0x08000575   Thumb Code    14  chip_uip_interrupt.o(i.RTC_IRQHandler)
    SLCD_IRQHandler                          0x08000589   Thumb Code    14  chip_uip_interrupt.o(i.SLCD_IRQHandler)
    SPI0_IRQHandler                          0x0800059d   Thumb Code    14  chip_uip_interrupt.o(i.SPI0_IRQHandler)
    SPI1_IRQHandler                          0x080005b1   Thumb Code    14  chip_uip_interrupt.o(i.SPI1_IRQHandler)
    SPI2_IRQHandler                          0x080005c5   Thumb Code    14  chip_uip_interrupt.o(i.SPI2_IRQHandler)
    SVC_Handler                              0x080005d9   Thumb Code     2  gd32f1x0_it.o(i.SVC_Handler)
    StartOS                                  0x080005dd   Thumb Code    38  uip_kernel_common.o(i.StartOS)
    SystemInit                               0x0800060d   Thumb Code   118  system_gd32f1x0.o(i.SystemInit)
    TASK_0                                   0x08000695   Thumb Code    54  demo.o(i.TASK_0)
    TASK_1                                   0x080006d1   Thumb Code    30  demo.o(i.TASK_1)
    TASK_2                                   0x080006f5   Thumb Code    32  demo.o(i.TASK_2)
    TASK_3                                   0x08000715   Thumb Code    26  demo.o(i.TASK_3)
    TASK_4                                   0x08000731   Thumb Code    24  demo.o(i.TASK_4)
    TIMER0_BRK_UP_TRG_COM_IRQHandler         0x08000751   Thumb Code    14  chip_uip_interrupt.o(i.TIMER0_BRK_UP_TRG_COM_IRQHandler)
    TIMER0_Channel_IRQHandler                0x08000765   Thumb Code    14  chip_uip_interrupt.o(i.TIMER0_Channel_IRQHandler)
    TIMER13_IRQHandler                       0x08000779   Thumb Code    14  chip_uip_interrupt.o(i.TIMER13_IRQHandler)
    TIMER14_IRQHandler                       0x0800078d   Thumb Code    14  chip_uip_interrupt.o(i.TIMER14_IRQHandler)
    TIMER15_IRQHandler                       0x080007a1   Thumb Code    14  chip_uip_interrupt.o(i.TIMER15_IRQHandler)
    TIMER16_IRQHandler                       0x080007b5   Thumb Code    14  chip_uip_interrupt.o(i.TIMER16_IRQHandler)
    TIMER1_IRQHandler                        0x080007c9   Thumb Code    14  chip_uip_interrupt.o(i.TIMER1_IRQHandler)
    TIMER2_IRQHandler                        0x080007dd   Thumb Code    14  chip_uip_interrupt.o(i.TIMER2_IRQHandler)
    TIMER5_DAC_IRQHandler                    0x080007f1   Thumb Code    14  chip_uip_interrupt.o(i.TIMER5_DAC_IRQHandler)
    TSI_IRQHandler                           0x08000805   Thumb Code    14  chip_uip_interrupt.o(i.TSI_IRQHandler)
    UIP_ActivateTask                         0x08000819   Thumb Code   220  uip_kernel_task.o(i.UIP_ActivateTask)
    UIP_ClearEvent                           0x0800091d   Thumb Code    68  uip_kernel_event.o(i.UIP_ClearEvent)
    UIP_GetResource                          0x0800096d   Thumb Code   162  uip_kernel_resource.o(i.UIP_GetResource)
    UIP_ReceiveMessage                       0x08000a31   Thumb Code   208  uip_kernel_message.o(i.UIP_ReceiveMessage)
    UIP_ReleaseResource                      0x08000b09   Thumb Code   252  uip_kernel_resource.o(i.UIP_ReleaseResource)
    UIP_SendMessage                          0x08000c35   Thumb Code   262  uip_kernel_message.o(i.UIP_SendMessage)
    UIP_SetEvent                             0x08000d45   Thumb Code   268  uip_kernel_event.o(i.UIP_SetEvent)
    UIP_TerminateTask                        0x08000e7d   Thumb Code   228  uip_kernel_task.o(i.UIP_TerminateTask)
    UIP_WaitEvent                            0x08000f89   Thumb Code   118  uip_kernel_event.o(i.UIP_WaitEvent)
    USART0_IRQHandler                        0x08001011   Thumb Code    14  chip_uip_interrupt.o(i.USART0_IRQHandler)
    USART0_IRQHandler_Process                0x08001025   Thumb Code   118  gd32f1x0_it.o(i.USART0_IRQHandler_Process)
    USART1_IRQHandler                        0x080010c1   Thumb Code    14  chip_uip_interrupt.o(i.USART1_IRQHandler)
    USBDWakeUp_IRQHandler                    0x080010d5   Thumb Code    14  chip_uip_interrupt.o(i.USBDWakeUp_IRQHandler)
    USBD_HP_IRQHandler                       0x080010e9   Thumb Code    14  chip_uip_interrupt.o(i.USBD_HP_IRQHandler)
    USBD_LP_IRQHandler                       0x080010fd   Thumb Code    14  chip_uip_interrupt.o(i.USBD_LP_IRQHandler)
    UsageFault_Handler                       0x08001111   Thumb Code     4  gd32f1x0_it.o(i.UsageFault_Handler)
    WWDGT_IRQHandler                         0x08001115   Thumb Code    14  chip_uip_interrupt.o(i.WWDGT_IRQHandler)
    __scatterload_copy                       0x08001129   Thumb Code    14  handlers.o(i.__scatterload_copy)
    __scatterload_null                       0x08001137   Thumb Code     2  handlers.o(i.__scatterload_null)
    __scatterload_zeroinit                   0x08001139   Thumb Code    14  handlers.o(i.__scatterload_zeroinit)
    gd_eval_com_init                         0x08001149   Thumb Code   176  gd32f1x0_eval.o(i.gd_eval_com_init)
    gpio_af_set                              0x08001209   Thumb Code    94  gd32f1x0_gpio.o(i.gpio_af_set)
    gpio_mode_set                            0x08001267   Thumb Code    78  gd32f1x0_gpio.o(i.gpio_mode_set)
    gpio_output_options_set                  0x080012b5   Thumb Code    66  gd32f1x0_gpio.o(i.gpio_output_options_set)
    main                                     0x080012f7   Thumb Code    10  main.o(i.main)
    nvic_irq_enable                          0x08001301   Thumb Code   156  gd32f1x0_misc.o(i.nvic_irq_enable)
    rcu_clock_freq_get                       0x080013a5   Thumb Code   646  gd32f1x0_rcu.o(i.rcu_clock_freq_get)
    rcu_periph_clock_enable                  0x0800164d   Thumb Code    28  gd32f1x0_rcu.o(i.rcu_periph_clock_enable)
    rcu_periph_reset_disable                 0x0800166d   Thumb Code    28  gd32f1x0_rcu.o(i.rcu_periph_reset_disable)
    rcu_periph_reset_enable                  0x0800168d   Thumb Code    28  gd32f1x0_rcu.o(i.rcu_periph_reset_enable)
    uipAlarmHandler                          0x08001759   Thumb Code   116  uip_kernel_time.o(i.uipAlarmHandler)
    uipAlarmInitialize                       0x080017d5   Thumb Code    34  uip_kernel_common.o(i.uipAlarmInitialize)
    uipAppInitialize                         0x08001801   Thumb Code    60  demo.o(i.uipAppInitialize)
    uipClearPrioGrpAndArrayBit               0x08001861   Thumb Code    96  uip_kernel_scheduler.o(i.uipClearPrioGrpAndArrayBit)
    uipEnterKernel                           0x080018c9   Thumb Code    22  demo.o(i.uipEnterKernel)
    uipGetNextPriority                       0x080018e5   Thumb Code    74  uip_kernel_scheduler.o(i.uipGetNextPriority)
    uipGetNextTask                           0x0800193d   Thumb Code   120  uip_kernel_scheduler.o(i.uipGetNextTask)
    uipInterruptHandlingCallback             0x080019d1   Thumb Code    20  chip_uip_interrupt.o(i.uipInterruptHandlingCallback)
    uipInterruptServiceEngine                0x080019e9   Thumb Code   252  uip_kernel_isr_engine.o(i.uipInterruptServiceEngine)
    uipKernelInitialize                      0x08001b05   Thumb Code   188  uip_kernel_common.o(i.uipKernelInitialize)
    uipMsgInitialize                         0x08001c2d   Thumb Code    62  uip_kernel_common.o(i.uipMsgInitialize)
    uipPreContexSwitch                       0x08001c75   Thumb Code    68  uip_kernel_scheduler.o(i.uipPreContexSwitch)
    uipResInitialize                         0x08001cc9   Thumb Code    76  uip_kernel_common.o(i.uipResInitialize)
    uipResetPrioGrpAndArrayBit               0x08001d1d   Thumb Code    62  uip_kernel_scheduler.o(i.uipResetPrioGrpAndArrayBit)
    uipSystemCounterHandler                  0x08001d6d   Thumb Code   116  uip_kernel_time.o(i.uipSystemCounterHandler)
    uipTaskInitialize                        0x08001ded   Thumb Code   236  uip_kernel_common.o(i.uipTaskInitialize)
    uipTaskStackInit                         0x08001ef9   Thumb Code    76  uip_kernel_common.o(i.uipTaskStackInit)
    usart_baudrate_set                       0x08001f45   Thumb Code   120  gd32f1x0_usart.o(i.usart_baudrate_set)
    usart_data_receive                       0x08001fc1   Thumb Code    10  gd32f1x0_usart.o(i.usart_data_receive)
    usart_data_transmit                      0x08001fcb   Thumb Code     8  gd32f1x0_usart.o(i.usart_data_transmit)
    usart_deinit                             0x08001fd5   Thumb Code    58  gd32f1x0_usart.o(i.usart_deinit)
    usart_enable                             0x08002015   Thumb Code    10  gd32f1x0_usart.o(i.usart_enable)
    usart_interrupt_disable                  0x0800201f   Thumb Code    26  gd32f1x0_usart.o(i.usart_interrupt_disable)
    usart_interrupt_enable                   0x08002039   Thumb Code    26  gd32f1x0_usart.o(i.usart_interrupt_enable)
    usart_interrupt_flag_get                 0x08002053   Thumb Code    56  gd32f1x0_usart.o(i.usart_interrupt_flag_get)
    usart_receive_config                     0x0800208b   Thumb Code    16  gd32f1x0_usart.o(i.usart_receive_config)
    usart_transmit_config                    0x0800209b   Thumb Code    16  gd32f1x0_usart.o(i.usart_transmit_config)
    Region$$Table$$Base                      0x080020ac   Number         0  anon$$obj.o(Region$$Table)
    Region$$Table$$Limit                     0x080020cc   Number         0  anon$$obj.o(Region$$Table)
    transmitter_buffer                       0x20000000   Data          25  main.o(.data)
    transfersize                             0x20000019   Data           1  main.o(.data)
    receivesize                              0x2000001a   Data           1  main.o(.data)
    txcount                                  0x2000001b   Data           1  main.o(.data)
    rxcount                                  0x2000001c   Data           2  main.o(.data)
    AppAlarmBase                             0x20000020   Data          24  app_cfg.o(.data)
    AppCounter                               0x20000038   Data          24  app_cfg.o(.data)
    AppAlarm                                 0x20000050   Data          48  app_cfg.o(.data)
    AppAlarmNumber                           0x20000080   Data           1  app_cfg.o(.data)
    AppRes                                   0x20000084   Data          20  app_cfg.o(.data)
    AppResNumber                             0x20000098   Data           1  app_cfg.o(.data)
    AppMsg                                   0x2000009c   Data          36  app_cfg.o(.data)
    AppMsgNumber                             0x200000c0   Data           1  app_cfg.o(.data)
    AppTask                                  0x200000c4   Data         288  app_cfg.o(.data)
    AppTaskNumber                            0x200001e4   Data           1  app_cfg.o(.data)
    Chip_GD32F1X0_USART_Int_Handling_Data    0x200001e8   Data           4  app_int_cfg.o(.data)
    UIP_Exc_VectorTable                      0x200001ec   Data          32  app_int_cfg.o(.data)
    AppIntNumber                             0x2000020c   Data           1  app_int_cfg.o(.data)
    SystemCoreClock                          0x20000210   Data           4  system_gd32f1x0.o(.data)
    uipLowPowerMode                          0x20000280   Data           1  uip_kernel_common.o(.data)
    uipTCBArray                              0x20000284   Data           4  uip_kernel_common.o(.data)
    uipTaskNumber                            0x20000288   Data           1  uip_kernel_common.o(.data)
    uipTaskIDNumber                          0x20000289   Data           1  uip_kernel_common.o(.data)
    uipRCBArray                              0x2000028c   Data           4  uip_kernel_common.o(.data)
    uipResNumber                             0x20000290   Data           1  uip_kernel_common.o(.data)
    uipACBArray                              0x20000294   Data           4  uip_kernel_common.o(.data)
    uipAlarmNumber                           0x20000298   Data           1  uip_kernel_common.o(.data)
    uipAlarmID                               0x20000299   Data           1  uip_kernel_common.o(.data)
    uipMCBArray                              0x2000029c   Data           4  uip_kernel_common.o(.data)
    uipMsgNumber                             0x200002a0   Data           1  uip_kernel_common.o(.data)
    uipOSSurport                             0x200002a1   Data           1  uip_kernel_common.o(.data)
    uipIdleTaskID                            0x200002a2   Data           1  uip_kernel_common.o(.data)
    uipIdleTaskTCBPtr                        0x200002a4   Data           4  uip_kernel_common.o(.data)
    uipIntTableID                            0x200002a8   Data           4  uip_kernel_common.o(.data)
    uipInSchedulerLoop                       0x200002ac   Data           4  uip_kernel_common.o(.data)
    uipByteValue                             0x200002b0   Data         256  uip_kernel_scheduler.o(.data)
    uipSchedulerLock                         0x200003b0   Data           1  uip_kernel_scheduler.o(.data)
    uipNestedInterrupts                      0x200003b4   Data           4  uip_kernel_scheduler.o(.data)
    uipSystemMode                            0x200003b8   Data           1  uip_kernel_scheduler.o(.data)
    uipPrioGroup                             0x200003bc   Data           4  uip_kernel_scheduler.o(.data)
    uipLowHalfByteValue                      0x200003c0   Data           1  uip_kernel_scheduler.o(.data)
    uipHighHalfByteValue                     0x200003c1   Data           1  uip_kernel_scheduler.o(.data)
    uipCurrentTaskTCBPtr                     0x200003c4   Data           4  uip_kernel_scheduler.o(.data)
    uipNextRunningTaskTCBPtr                 0x200003c8   Data           4  uip_kernel_scheduler.o(.data)
    uipSystemStackPtr                        0x200003cc   Data           4  uip_kernel_scheduler.o(.data)
    uipCurrentTaskPriority                   0x200003d0   Data           1  uip_kernel_scheduler.o(.data)
    uipNextRunningTaskPriority               0x200003d1   Data           1  uip_kernel_scheduler.o(.data)
    receiver_buffer                          0x200003d4   Data          32  main.o(.bss)
    AppMsgBuf                                0x200003f4   Data          64  app_cfg.o(.bss)
    Task_0_Stack                             0x20000434   Data         256  app_cfg.o(.bss)
    Task_1_Stack                             0x20000534   Data         256  app_cfg.o(.bss)
    Task_2_Stack                             0x20000634   Data         256  app_cfg.o(.bss)
    Task_3_Stack                             0x20000734   Data         256  app_cfg.o(.bss)
    Task_4_Stack                             0x20000834   Data         256  app_cfg.o(.bss)
    Task_App_Idle_Stack                      0x20000934   Data         256  app_cfg.o(.bss)
    appBuf                                   0x20000a34   Data          32  demo.o(.bss)
    uipPriorityToTaskID                      0x20000a54   Data         256  uip_kernel_common.o(.bss)
    uipInitTaskStackPtr                      0x20000b54   Data        1024  uip_kernel_common.o(.bss)
    uipSystemCounter                         0x20000f54   Data          12  uip_kernel_common.o(.bss)
    uipSystemAlarmBase                       0x20000f60   Data          12  uip_kernel_common.o(.bss)
    uipPrioGrpArray                          0x20000f6c   Data          32  uip_kernel_scheduler.o(.bss)
    __initial_sp                             0x20001190   Data           0  startup_gd32f1x0.o(STACK)



==============================================================================

Memory Map of the image

  Image Entry point : 0x08000169

  Load Region LR_IROM1 (Base: 0x08000000, Size: 0x000024a0, Max: 0x00010000, ABSOLUTE, COMPRESSED[0x000021e4])

    Execution Region ER_IROM1 (Exec base: 0x08000000, Load base: 0x08000000, Size: 0x000020cc, Max: 0x00010000, ABSOLUTE)

    Exec Addr    Load Addr    Size         Type   Attr      Idx    E Section Name        Object

    0x08000000   0x08000000   0x00000168   Data   RO          415    RESET               startup_gd32f1x0.o
    0x08000168   0x08000168   0x00000000   Code   RO         4654  * .ARM.Collect$$$$00000000  mc_w.l(entry.o)
    0x08000168   0x08000168   0x00000004   Code   RO         4657    .ARM.Collect$$$$00000001  mc_w.l(entry2.o)
    0x0800016c   0x0800016c   0x00000004   Code   RO         4660    .ARM.Collect$$$$00000004  mc_w.l(entry5.o)
    0x08000170   0x08000170   0x00000000   Code   RO         4662    .ARM.Collect$$$$00000008  mc_w.l(entry7b.o)
    0x08000170   0x08000170   0x00000000   Code   RO         4664    .ARM.Collect$$$$0000000A  mc_w.l(entry8b.o)
    0x08000170   0x08000170   0x00000008   Code   RO         4665    .ARM.Collect$$$$0000000B  mc_w.l(entry9a.o)
    0x08000178   0x08000178   0x00000000   Code   RO         4667    .ARM.Collect$$$$0000000D  mc_w.l(entry10a.o)
    0x08000178   0x08000178   0x00000000   Code   RO         4669    .ARM.Collect$$$$0000000F  mc_w.l(entry11a.o)
    0x08000178   0x08000178   0x00000004   Code   RO         4658    .ARM.Collect$$$$00002712  mc_w.l(entry2.o)
    0x0800017c   0x0800017c   0x00000024   Code   RO          416    .text               startup_gd32f1x0.o
    0x080001a0   0x080001a0   0x00000024   Code   RO         4671    .text               mc_w.l(init.o)
    0x080001c4   0x080001c4   0x00000056   Code   RO         4681    .text               mc_w.l(__dczerorl2.o)
    0x0800021a   0x0800021a   0x00000002   PAD
    0x0800021c   0x0800021c   0x00000048   Code   RO         4421    CODE                uip_kernel_isr_cm.o
    0x08000264   0x08000264   0x00000014   Code   RO         3937    i.ADC_CMP_IRQHandler  chip_uip_interrupt.o
    0x08000278   0x08000278   0x0000002e   Code   RO          251    i.AppIdleTask       demo.o
    0x080002a6   0x080002a6   0x00000004   Code   RO            3    i.BusFault_Handler  gd32f1x0_it.o
    0x080002aa   0x080002aa   0x00000002   PAD
    0x080002ac   0x080002ac   0x00000014   Code   RO         3938    i.CAN0_RX0_IRQHandler  chip_uip_interrupt.o
    0x080002c0   0x080002c0   0x00000014   Code   RO         3939    i.CAN0_RX1_IRQHandler  chip_uip_interrupt.o
    0x080002d4   0x080002d4   0x00000014   Code   RO         3940    i.CAN0_SCE_IRQHandler  chip_uip_interrupt.o
    0x080002e8   0x080002e8   0x00000014   Code   RO         3941    i.CAN0_TX_IRQHandler  chip_uip_interrupt.o
    0x080002fc   0x080002fc   0x00000014   Code   RO         3942    i.CAN1_RX0_IRQHandler  chip_uip_interrupt.o
    0x08000310   0x08000310   0x00000014   Code   RO         3943    i.CAN1_RX1_IRQHandler  chip_uip_interrupt.o
    0x08000324   0x08000324   0x00000014   Code   RO         3944    i.CAN1_SCE_IRQHandler  chip_uip_interrupt.o
    0x08000338   0x08000338   0x00000014   Code   RO         3945    i.CAN1_TX_IRQHandler  chip_uip_interrupt.o
    0x0800034c   0x0800034c   0x00000014   Code   RO         3946    i.CEC_IRQHandler    chip_uip_interrupt.o
    0x08000360   0x08000360   0x00000006   Code   RO          224    i.Chip_GD32F1X0_USART0_ISR_Handler_Callback  app_int_cfg.o
    0x08000366   0x08000366   0x00000002   PAD
    0x08000368   0x08000368   0x00000014   Code   RO         3953    i.DMA_Channel0_IRQHandler  chip_uip_interrupt.o
    0x0800037c   0x0800037c   0x00000014   Code   RO         3954    i.DMA_Channel1_2_IRQHandler  chip_uip_interrupt.o
    0x08000390   0x08000390   0x00000014   Code   RO         3955    i.DMA_Channel3_4_IRQHandler  chip_uip_interrupt.o
    0x080003a4   0x080003a4   0x00000014   Code   RO         3956    i.DMA_Channel5_6_IRQHandler  chip_uip_interrupt.o
    0x080003b8   0x080003b8   0x00000002   Code   RO            4    i.DebugMon_Handler  gd32f1x0_it.o
    0x080003ba   0x080003ba   0x00000002   PAD
    0x080003bc   0x080003bc   0x00000014   Code   RO         3957    i.EXTI0_1_IRQHandler  chip_uip_interrupt.o
    0x080003d0   0x080003d0   0x00000014   Code   RO         3958    i.EXTI2_3_IRQHandler  chip_uip_interrupt.o
    0x080003e4   0x080003e4   0x00000014   Code   RO         3959    i.EXTI4_15_IRQHandler  chip_uip_interrupt.o
    0x080003f8   0x080003f8   0x00000014   Code   RO         3960    i.FMC_IRQHandler    chip_uip_interrupt.o
    0x0800040c   0x0800040c   0x00000004   Code   RO            5    i.HardFault_Handler  gd32f1x0_it.o
    0x08000410   0x08000410   0x00000014   Code   RO         3961    i.I2C0_ER_IRQHandler  chip_uip_interrupt.o
    0x08000424   0x08000424   0x00000014   Code   RO         3962    i.I2C0_EV_IRQHandler  chip_uip_interrupt.o
    0x08000438   0x08000438   0x00000014   Code   RO         3963    i.I2C1_ER_IRQHandler  chip_uip_interrupt.o
    0x0800044c   0x0800044c   0x00000014   Code   RO         3964    i.I2C1_EV_IRQHandler  chip_uip_interrupt.o
    0x08000460   0x08000460   0x00000014   Code   RO         3965    i.I2C2_ER_IRQHandler  chip_uip_interrupt.o
    0x08000474   0x08000474   0x00000014   Code   RO         3966    i.I2C2_EV_IRQHandler  chip_uip_interrupt.o
    0x08000488   0x08000488   0x0000005c   Code   RO         3967    i.InterruptHandler  chip_uip_interrupt.o
    0x080004e4   0x080004e4   0x00000060   Code   RO         4275    i.Kernel_System_Tick_Init  hardware_init.o
    0x08000544   0x08000544   0x00000014   Code   RO         3968    i.LVD_IRQHandler    chip_uip_interrupt.o
    0x08000558   0x08000558   0x00000004   Code   RO            6    i.MemManage_Handler  gd32f1x0_it.o
    0x0800055c   0x0800055c   0x00000002   Code   RO            7    i.NMI_Handler       gd32f1x0_it.o
    0x0800055e   0x0800055e   0x00000002   PAD
    0x08000560   0x08000560   0x00000014   Code   RO         3969    i.RCU_IRQHandler    chip_uip_interrupt.o
    0x08000574   0x08000574   0x00000014   Code   RO         3970    i.RTC_IRQHandler    chip_uip_interrupt.o
    0x08000588   0x08000588   0x00000014   Code   RO         3971    i.SLCD_IRQHandler   chip_uip_interrupt.o
    0x0800059c   0x0800059c   0x00000014   Code   RO         3972    i.SPI0_IRQHandler   chip_uip_interrupt.o
    0x080005b0   0x080005b0   0x00000014   Code   RO         3973    i.SPI1_IRQHandler   chip_uip_interrupt.o
    0x080005c4   0x080005c4   0x00000014   Code   RO         3974    i.SPI2_IRQHandler   chip_uip_interrupt.o
    0x080005d8   0x080005d8   0x00000002   Code   RO            8    i.SVC_Handler       gd32f1x0_it.o
    0x080005da   0x080005da   0x00000002   PAD
    0x080005dc   0x080005dc   0x00000030   Code   RO         4306    i.StartOS           uip_kernel_common.o
    0x0800060c   0x0800060c   0x00000088   Code   RO          374    i.SystemInit        system_gd32f1x0.o
    0x08000694   0x08000694   0x0000003c   Code   RO          252    i.TASK_0            demo.o
    0x080006d0   0x080006d0   0x00000024   Code   RO          253    i.TASK_1            demo.o
    0x080006f4   0x080006f4   0x00000020   Code   RO          254    i.TASK_2            demo.o
    0x08000714   0x08000714   0x0000001a   Code   RO          255    i.TASK_3            demo.o
    0x0800072e   0x0800072e   0x00000002   PAD
    0x08000730   0x08000730   0x00000020   Code   RO          256    i.TASK_4            demo.o
    0x08000750   0x08000750   0x00000014   Code   RO         3975    i.TIMER0_BRK_UP_TRG_COM_IRQHandler  chip_uip_interrupt.o
    0x08000764   0x08000764   0x00000014   Code   RO         3976    i.TIMER0_Channel_IRQHandler  chip_uip_interrupt.o
    0x08000778   0x08000778   0x00000014   Code   RO         3977    i.TIMER13_IRQHandler  chip_uip_interrupt.o
    0x0800078c   0x0800078c   0x00000014   Code   RO         3978    i.TIMER14_IRQHandler  chip_uip_interrupt.o
    0x080007a0   0x080007a0   0x00000014   Code   RO         3979    i.TIMER15_IRQHandler  chip_uip_interrupt.o
    0x080007b4   0x080007b4   0x00000014   Code   RO         3980    i.TIMER16_IRQHandler  chip_uip_interrupt.o
    0x080007c8   0x080007c8   0x00000014   Code   RO         3981    i.TIMER1_IRQHandler  chip_uip_interrupt.o
    0x080007dc   0x080007dc   0x00000014   Code   RO         3982    i.TIMER2_IRQHandler  chip_uip_interrupt.o
    0x080007f0   0x080007f0   0x00000014   Code   RO         3983    i.TIMER5_DAC_IRQHandler  chip_uip_interrupt.o
    0x08000804   0x08000804   0x00000014   Code   RO         3984    i.TSI_IRQHandler    chip_uip_interrupt.o
    0x08000818   0x08000818   0x00000104   Code   RO         4552    i.UIP_ActivateTask  uip_kernel_task.o
    0x0800091c   0x0800091c   0x00000050   Code   RO         4391    i.UIP_ClearEvent    uip_kernel_event.o
    0x0800096c   0x0800096c   0x000000c4   Code   RO         4490    i.UIP_GetResource   uip_kernel_resource.o
    0x08000a30   0x08000a30   0x000000d8   Code   RO         4439    i.UIP_ReceiveMessage  uip_kernel_message.o
    0x08000b08   0x08000b08   0x0000012c   Code   RO         4491    i.UIP_ReleaseResource  uip_kernel_resource.o
    0x08000c34   0x08000c34   0x00000110   Code   RO         4441    i.UIP_SendMessage   uip_kernel_message.o
    0x08000d44   0x08000d44   0x00000138   Code   RO         4393    i.UIP_SetEvent      uip_kernel_event.o
    0x08000e7c   0x08000e7c   0x0000010c   Code   RO         4557    i.UIP_TerminateTask  uip_kernel_task.o
    0x08000f88   0x08000f88   0x00000088   Code   RO         4394    i.UIP_WaitEvent     uip_kernel_event.o
    0x08001010   0x08001010   0x00000014   Code   RO         3985    i.USART0_IRQHandler  chip_uip_interrupt.o
    0x08001024   0x08001024   0x0000009c   Code   RO            9    i.USART0_IRQHandler_Process  gd32f1x0_it.o
    0x080010c0   0x080010c0   0x00000014   Code   RO         3986    i.USART1_IRQHandler  chip_uip_interrupt.o
    0x080010d4   0x080010d4   0x00000014   Code   RO         3987    i.USBDWakeUp_IRQHandler  chip_uip_interrupt.o
    0x080010e8   0x080010e8   0x00000014   Code   RO         3988    i.USBD_HP_IRQHandler  chip_uip_interrupt.o
    0x080010fc   0x080010fc   0x00000014   Code   RO         3989    i.USBD_LP_IRQHandler  chip_uip_interrupt.o
    0x08001110   0x08001110   0x00000004   Code   RO           10    i.UsageFault_Handler  gd32f1x0_it.o
    0x08001114   0x08001114   0x00000014   Code   RO         3990    i.WWDGT_IRQHandler  chip_uip_interrupt.o
    0x08001128   0x08001128   0x0000000e   Code   RO         4675    i.__scatterload_copy  mc_w.l(handlers.o)
    0x08001136   0x08001136   0x00000002   Code   RO         4676    i.__scatterload_null  mc_w.l(handlers.o)
    0x08001138   0x08001138   0x0000000e   Code   RO         4677    i.__scatterload_zeroinit  mc_w.l(handlers.o)
    0x08001146   0x08001146   0x00000002   PAD
    0x08001148   0x08001148   0x000000c0   Code   RO         3881    i.gd_eval_com_init  gd32f1x0_eval.o
    0x08001208   0x08001208   0x0000005e   Code   RO         1615    i.gpio_af_set       gd32f1x0_gpio.o
    0x08001266   0x08001266   0x0000004e   Code   RO         1622    i.gpio_mode_set     gd32f1x0_gpio.o
    0x080012b4   0x080012b4   0x00000042   Code   RO         1624    i.gpio_output_options_set  gd32f1x0_gpio.o
    0x080012f6   0x080012f6   0x0000000a   Code   RO          177    i.main              main.o
    0x08001300   0x08001300   0x000000a4   Code   RO         1905    i.nvic_irq_enable   gd32f1x0_misc.o
    0x080013a4   0x080013a4   0x000002a8   Code   RO         2059    i.rcu_clock_freq_get  gd32f1x0_rcu.o
    0x0800164c   0x0800164c   0x00000020   Code   RO         2079    i.rcu_periph_clock_enable  gd32f1x0_rcu.o
    0x0800166c   0x0800166c   0x00000020   Code   RO         2082    i.rcu_periph_reset_disable  gd32f1x0_rcu.o
    0x0800168c   0x0800168c   0x00000020   Code   RO         2083    i.rcu_periph_reset_enable  gd32f1x0_rcu.o
    0x080016ac   0x080016ac   0x000000a4   Code   RO          375    i.system_clock_72m_hxtal  system_gd32f1x0.o
    0x08001750   0x08001750   0x00000008   Code   RO          376    i.system_clock_config  system_gd32f1x0.o
    0x08001758   0x08001758   0x0000007c   Code   RO         4599    i.uipAlarmHandler   uip_kernel_time.o
    0x080017d4   0x080017d4   0x0000002c   Code   RO         4308    i.uipAlarmInitialize  uip_kernel_common.o
    0x08001800   0x08001800   0x00000060   Code   RO          257    i.uipAppInitialize  demo.o
    0x08001860   0x08001860   0x00000068   Code   RO         4508    i.uipClearPrioGrpAndArrayBit  uip_kernel_scheduler.o
    0x080018c8   0x080018c8   0x0000001c   Code   RO          259    i.uipEnterKernel    demo.o
    0x080018e4   0x080018e4   0x00000058   Code   RO         4509    i.uipGetNextPriority  uip_kernel_scheduler.o
    0x0800193c   0x0800193c   0x00000094   Code   RO         4510    i.uipGetNextTask    uip_kernel_scheduler.o
    0x080019d0   0x080019d0   0x00000018   Code   RO         3991    i.uipInterruptHandlingCallback  chip_uip_interrupt.o
    0x080019e8   0x080019e8   0x0000011c   Code   RO         4424    i.uipInterruptServiceEngine  uip_kernel_isr_engine.o
    0x08001b04   0x08001b04   0x00000128   Code   RO         4309    i.uipKernelInitialize  uip_kernel_common.o
    0x08001c2c   0x08001c2c   0x00000048   Code   RO         4311    i.uipMsgInitialize  uip_kernel_common.o
    0x08001c74   0x08001c74   0x00000054   Code   RO         4511    i.uipPreContexSwitch  uip_kernel_scheduler.o
    0x08001cc8   0x08001cc8   0x00000054   Code   RO         4313    i.uipResInitialize  uip_kernel_common.o
    0x08001d1c   0x08001d1c   0x00000050   Code   RO         4512    i.uipResetPrioGrpAndArrayBit  uip_kernel_scheduler.o
    0x08001d6c   0x08001d6c   0x00000080   Code   RO         4602    i.uipSystemCounterHandler  uip_kernel_time.o
    0x08001dec   0x08001dec   0x0000010c   Code   RO         4315    i.uipTaskInitialize  uip_kernel_common.o
    0x08001ef8   0x08001ef8   0x0000004c   Code   RO         4316    i.uipTaskStackInit  uip_kernel_common.o
    0x08001f44   0x08001f44   0x0000007c   Code   RO         3408    i.usart_baudrate_set  gd32f1x0_usart.o
    0x08001fc0   0x08001fc0   0x0000000a   Code   RO         3414    i.usart_data_receive  gd32f1x0_usart.o
    0x08001fca   0x08001fca   0x00000008   Code   RO         3415    i.usart_data_transmit  gd32f1x0_usart.o
    0x08001fd2   0x08001fd2   0x00000002   PAD
    0x08001fd4   0x08001fd4   0x00000040   Code   RO         3416    i.usart_deinit      gd32f1x0_usart.o
    0x08002014   0x08002014   0x0000000a   Code   RO         3423    i.usart_enable      gd32f1x0_usart.o
    0x0800201e   0x0800201e   0x0000001a   Code   RO         3431    i.usart_interrupt_disable  gd32f1x0_usart.o
    0x08002038   0x08002038   0x0000001a   Code   RO         3432    i.usart_interrupt_enable  gd32f1x0_usart.o
    0x08002052   0x08002052   0x00000038   Code   RO         3434    i.usart_interrupt_flag_get  gd32f1x0_usart.o
    0x0800208a   0x0800208a   0x00000010   Code   RO         3450    i.usart_receive_config  gd32f1x0_usart.o
    0x0800209a   0x0800209a   0x00000010   Code   RO         3466    i.usart_transmit_config  gd32f1x0_usart.o
    0x080020aa   0x080020aa   0x00000002   PAD
    0x080020ac   0x080020ac   0x00000020   Data   RO         4673    Region$$Table       anon$$obj.o


    Execution Region RW_IRAM1 (Exec base: 0x20000000, Load base: 0x080020cc, Size: 0x00001190, Max: 0x00002000, ABSOLUTE, COMPRESSED[0x00000118])

    Exec Addr    Load Addr    Size         Type   Attr      Idx    E Section Name        Object

    0x20000000   COMPRESSED   0x0000001e   Data   RW          179    .data               main.o
    0x2000001e   COMPRESSED   0x00000002   PAD
    0x20000020   COMPRESSED   0x000001c5   Data   RW          209    .data               app_cfg.o
    0x200001e5   COMPRESSED   0x00000003   PAD
    0x200001e8   COMPRESSED   0x00000025   Data   RW          225    .data               app_int_cfg.o
    0x2000020d   COMPRESSED   0x00000003   PAD
    0x20000210   COMPRESSED   0x00000004   Data   RW          377    .data               system_gd32f1x0.o
    0x20000214   COMPRESSED   0x00000069   Data   RW         3888    .data               gd32f1x0_eval.o
    0x2000027d   COMPRESSED   0x00000003   PAD
    0x20000280   COMPRESSED   0x00000030   Data   RW         4318    .data               uip_kernel_common.o
    0x200002b0   COMPRESSED   0x00000122   Data   RW         4514    .data               uip_kernel_scheduler.o
    0x200003d2   COMPRESSED   0x00000002   PAD
    0x200003d4        -       0x00000020   Zero   RW          178    .bss                main.o
    0x200003f4        -       0x00000640   Zero   RW          208    .bss                app_cfg.o
    0x20000a34        -       0x00000020   Zero   RW          260    .bss                demo.o
    0x20000a54        -       0x00000518   Zero   RW         4317    .bss                uip_kernel_common.o
    0x20000f6c        -       0x00000020   Zero   RW         4513    .bss                uip_kernel_scheduler.o
    0x20000f8c   COMPRESSED   0x00000004   PAD
    0x20000f90        -       0x00000200   Zero   RW          413    STACK               startup_gd32f1x0.o


==============================================================================

Image component sizes


      Code (inc. data)   RO Data    RW Data    ZI Data      Debug   Object Name

         0          0          0        453       1600       1491   app_cfg.o
         6          0          0         37          0       1673   app_int_cfg.o
      1056        300          0          0          0      28099   chip_uip_interrupt.o
       356         62          0          0         32       4996   demo.o
       192         16          0        105          0       1751   gd32f1x0_eval.o
       238          0          0          0          0       2648   gd32f1x0_gpio.o
       178         38          0          0          0      42882   gd32f1x0_it.o
       164          8          0          0          0        922   gd32f1x0_misc.o
       776         54          0          0          0       4004   gd32f1x0_rcu.o
       356         10          0          0          0       7331   gd32f1x0_usart.o
        96         14          0          0          0      24625   hardware_init.o
        10          0          0         30         32       1897   main.o
        36         10        360          0        512        888   startup_gd32f1x0.o
       308         28          0          4          0       2263   system_gd32f1x0.o
       888        178          0         48       1304      14353   uip_kernel_common.o
       528         74          0          0          0       2700   uip_kernel_event.o
        72          4          0          0          0        384   uip_kernel_isr_cm.o
       284         32          0          0          0        824   uip_kernel_isr_engine.o
       488         18          0          0          0       2191   uip_kernel_message.o
       496         82          0          0          0       1988   uip_kernel_resource.o
       504         84          0        290         32      12148   uip_kernel_scheduler.o
       528         80          0          0          0       1743   uip_kernel_task.o
       252         20          0          0          0       1388   uip_kernel_time.o

    ----------------------------------------------------------------------
      7828       1112        392        980       3516     163189   Object Totals
         0          0         32          0          0          0   (incl. Generated)
        16          0          0         13          4          0   (incl. Padding)

    ----------------------------------------------------------------------

      Code (inc. data)   RO Data    RW Data    ZI Data      Debug   Library Member Name

        86          0          0          0          0          0   __dczerorl2.o
         0          0          0          0          0          0   entry.o
         0          0          0          0          0          0   entry10a.o
         0          0          0          0          0          0   entry11a.o
         8          4          0          0          0          0   entry2.o
         4          0          0          0          0          0   entry5.o
         0          0          0          0          0          0   entry7b.o
         0          0          0          0          0          0   entry8b.o
         8          4          0          0          0          0   entry9a.o
        30          0          0          0          0          0   handlers.o
        36          8          0          0          0         68   init.o

    ----------------------------------------------------------------------
       176         16          0          0          0         68   Library Totals
         4          0          0          0          0          0   (incl. Padding)

    ----------------------------------------------------------------------

      Code (inc. data)   RO Data    RW Data    ZI Data      Debug   Library Name

       172         16          0          0          0         68   mc_w.l

    ----------------------------------------------------------------------
       176         16          0          0          0         68   Library Totals

    ----------------------------------------------------------------------

==============================================================================


      Code (inc. data)   RO Data    RW Data    ZI Data      Debug   

      8004       1128        392        980       3516     157769   Grand Totals
      8004       1128        392        280       3516     157769   ELF Image Totals (compressed)
      8004       1128        392        280          0          0   ROM Totals

==============================================================================

    Total RO  Size (Code + RO Data)                 8396 (   8.20kB)
    Total RW  Size (RW Data + ZI Data)              4496 (   4.39kB)
    Total ROM Size (Code + RO Data + RW Data)       8676 (   8.47kB)

==============================================================================

